:100000000C94B40F0C94D50F0C94D50F0C94D50F01
:100010000C94D50F0C94D50F0C94D50F0C94D50FD0
:100020000C94D50F0C94D50F0C9476680C949368AF
:100030000C94D50F0C94D50F0C9454690C948169D1
:100040000C94AE690C94DB690C94086A0C94356AC4
:100050000C94626A0C948F6A0C94BC6A0C94E96AE2
:100060000C94D50F0D942C350D9463350C94D50F4D
:100070000C94D50F0C94D50F0C94D50F0C94D50F70
:100080000C94D50F0C94D50F0C94D50F0C94D50F60
:100090000C94D50F0C94D50F0C94D50F0D947A6059
:1000A0000D94AC600D94DE600D9410610D94C6103B
:1000B0000C94D50F0C94D50F0C94D50F0C94D86CD0
:1000C0000C94056D0C94326D0C945F6D0C948C6DDA
:1000D0000C94B96D0C94E66D0C94136E0C94406EF8
:1000E0000C946D6E0C94D50F0D9450340D94873490
:1000F0000C94D50F0C94D50F0C94D50F0C94D50FF0
:100100000C94D50F0C94D50F0D94A0150C94D50F0D
:100110000C94D50F0C94D50F0C94D50F0D94B25FA1
:100120000D94E45F0D9416600D9448600C94D50F07
:100130000C94D50F0C94166B0C94436B0C94706B51
:100140000C949D6B0C94CA6B0C94F76B0C94246C00
:100150000C94516C0C947E6C0C94AB6C0C94D50F7D
:100160000D94BE340D94F5340C94D50F0C94D50F2A
:100170000C94D50F0C94D50F0C94D50F0C94D50F6F
:100180000C94D50F0C94D50F0C94D50F0C94D50F5F
:100190000C94D50F0C94D50F0C94D50F0C94D50F4F
:1001A0000D9493100C94D50F0C94D50F0C94D50F7F
:1001B0000C949A6E0C94C76E0C94F46E0C94216F90
:1001C0000C944E6F0C947B6F0C94D50F0C94D50F40
:1001D0000C94D50F0C94D50F0C94D50F0D949A3523
:1001E0000D94D1350C94D50F0C94D50F0C94D50FDC
:1001F0000C94D50F0C94137B0C94CE7B8E101111A4
:10020000A0101111B2101111C410DE10C410F8109A
:10021000F810BF12D312E7120D133313AE139B1352
:10022000AE137513751376187618AE18EB182F19D0
:100230006C18181A341A711ACF19CF19341A181ADF
:100240002F19EB18AE187618761835223F2249225E
:1002500053225D226722712276227B22852285220B
:10026000762271225D22532249223F2235224D27D8
:100270004D275427542767278A274D278A27542735
:1002800054274D278A27542754274D274D27C32706
:10029000C327CB27CB27E0270728C3270728CB274F
:1002A000CB27C3270728CB27CB27C327C32717284C
:1002B000B8284028B828B8289128B828692869287B
:1002C0009128B8284028B8281728EB28F6280529AF
:1002D0002029362958299E29A729C2297E297E2925
:1002E000A7299E29362920290529F628EB288A6185
:1002F000016201621A6101620162016201620162CE
:1003000001620162016201620162016201620162D5
:1003100001622F6101620162016201620162016298
:1003200001628461E26101620162EF610162016266
:1003300001620162016201629D6101620162FB6111
:100340000162FE610162016201620162F8610162A3
:100350000162016201620162016201620162016285
:100360000162016201620162016201620162016275
:100370000162016201620162016201620162016265
:100380000162016201620162016201620162016255
:100390000162016201620162016201620162016245
:1003A00001628761E775EA75ED75F075F375F675AD
:1003B000F975667D797D8C7D9F7DB27DC57DD87D0B
:1003C000E082E0825D82A282A28215821582A282F0
:1003D000A282A282A282A282A282A282A282A282FD
:1003E000A282A282A282A282A282A2821582A2827A
:1003F000A282A282A282A282EC879389288859884D
:10040000938993899389938993899389938993890C
:1004100093899389938993899389938993899389FC
:1004200093899389938993899389938993899389EC
:1004300093899389938993899389938993899389DC
:1004400093899389938993899389938993899389CC
:100450009389938993899389938926899389948829
:1004600093899389558993899389938993899389EA
:100470009389938993899389D7889389A38893894A
:10048000B1889389058944937491AD91F7915D92F8
:10049000A892BD92EF9211933293F79484938C9328
:1004A000A993E893FB93459467947E949394F29474
:1004B000F294F294F294F294F294F294F294F2940C
:1004C000F294AA94B294BD94D294D894C8BDF9BDC4
:1004D000A4BDB0BDF9BDF9BDF9BDF9BDF9BDF9BD0A
:1004E000F9BDF9BDF9BDF9BDF9BDF9BDF9BDF9BD5C
:1004F000BCBDF9BDF9BDF9BDF9BDF9BDF9BDF9BD89
:10050000F9BDF9BDF9BDF9BDF9BDF9BDC8BDF9BD6C
:10051000A4BDB0BDF9BDF9BDF9BDF9BDF9BDF9BDC9
:10052000F9BDF9BDF9BDF9BDF9BDF9BDF9BDF9BD1B
:10053000BCBD61C964C9B5C9B5C9B5C9B5C9B5C975
:10054000B5C9B5C9B5C9B5C9B5C9B5C9B5C9B5C9BB
:10055000B5C9B5C9B5C9B5C9B5C9B5C99BC9B5C9C5
:10056000B5C9B5C9B5C9B5C9B5C981C9B5C9B5C9CF
:10057000B5C9B5C9B5C967C9B5C9B5C9B5C9B5C9D9
:10058000B5C9B5C9B5C9B5C9B5C9B5C9B5C9B5C97B
:10059000B5C9B5C9B5C9B5C9B5C9B5C99BC9B5C985
:1005A000B5C9B5C9B5C9B5C9B5C981C9B5C9B5C98F
:1005B000B5C9B5C9B5C967C95ECC5BCC70CC70CCC8
:1005C00070CC70CC70CC70CC70CC70CC70CC70CC4B
:1005D00070CC70CC70CC70CC70CCA7CB7ACB98CBD5
:1005E00070CC70CC1ECC61CB70CC70CC70CC70CC8D
:1005F00070CC89CB61CC70CC70CCB1CB70CC70CCD2
:1006000070CC70CC70CC70CC70CC70CC70CC70CC0A
:1006100070CC70CC70CC70CC70CCA7CB7ACB98CB94
:1006200070CC70CC1ECC61CB70CC70CC70CC70CC4C
:1006300070CC89CB61CC70CC70CCB1CB69CFACCF56
:10064000BBCFBBCFBBCFBBCFBBCFBBCFBBCFBBCF5A
:10065000BBCFBBCFBBCFBBCFBBCF96CEBBCF4DCFDE
:1006600047CFAFCE63CFBBCFBBCFBFCE96CEBBCF36
:100670005DCF78CFA3CE57CFB1CF53CFB5CE6ECF0E
:1006800041CFBACEBBCF73CF92CEB6CFBBCFBBCF0D
:10069000A9CEBBCFBBCFBBCFBBCFBBCFBBCF4DCF8B
:1006A00047CFAFCE63CFBBCFBBCFBFCE96CEBBCFF6
:1006B0005DCF78CFA3CE57CFB1CF53CFB5CE6ECFCE
:1006C00041CFBACEBBCF73CF92CEB6CFBBCFBBCFCD
:1006D000A9CE72CEDBD4CBD4CDD4CFD4D1D4D3D485
:1006E000D5D4D7D4F8D4E8D4EAD4ECD4EED4F0D42A
:1006F000F2D4F4D405D533D50DD533D50DD533D5B6
:100700000DD533D50DD533D50DD533D533D533D51B
:1007100033D533D533D533D514D51BD527D527D5E8
:1007200063E892E69EE6E9E61AE8FEE640E764E75B
:100730008DE7E8E70FF00FF099F0D1F1B1F2D9F3BE
:10074000C3F4B1F5C3F4FDF6FDF6B1F5C3F4B1F2AF
:10075000D1F199F00FF00FF033F933F974F9D2F9C0
:1007600011FA5FFA94FAD3FA94FA21FB21FBD3FA37
:1007700094FA11FAD2F974F933F933F97EFDE9FDEF
:1007800054FE0DFFB9FFD003DA03E003DA03D80308
:10079000D803E003DA03B9FF0DFF54FEE9FD7EFD47
:1007A0000D94A9000D9469200D942B210D949E2188
:1007B0000D944A030D9492010D9484220D941E22EF
:1007C0000D9449020D9406224E414E494E4954590A
:1007D000494E46CDCCCC3D0AD7233C17B7D138770C
:1007E000CC2B329595E6241FB14F0A000020410022
:1007F00000C84200401C4620BCBE4CCA1B0E5AAE6C
:10080000C59D74444D2E4D00444D53004444003268
:1008100035304D4F686D0032354D4F686D003630C4
:10082000487A003530487A004E6F6E2D496E74005C
:1008300048692D4C4F004750530054696D65004482
:10084000697374616E6365005075736820427574D6
:10085000746F6E00496D70657269616C004D6574EE
:1008600072696300494E4300444543004F4E004FB8
:100870004646007B0976096C096509590952094603
:10088000093509270914090109EC08DB08C808BA69
:1008900008AB08A1089708434950532641435647DF
:1008A0000044435647264143564700434950532688
:1008B00044435647264143564700327844435647FF
:1008C00026327841435647004349505326327844F4
:1008D00043564726327841435647003278496D7077
:1008E0002E20434950532641435647003278496DE4
:1008F000702E43495053264443564726414356479A
:1009000000327843495053263278444356472641B3
:10091000435647003278496D702E20434950532684
:1009200032784443564700506172616C6C656C20AC
:1009300043495053003278496D702E20434950533B
:100940002644435647003278496D702E2043495063
:100950005300347844435647004349505326327875
:100960004443564700327844435647004349505366
:1009700026444356470044435647004349505300DA
:100980004B128911C7100510430F810EBF0DFD0CCE
:100990003B0C790B180BFD0CBF0D430F0510C71056
:1009A00089114B12AC12EA1128116610A40FE20E45
:1009B000200E5E0D9C0CDA0B180B5E0D200EA40FA2
:1009C00066102811EA11AC1253616D706C652F73BB
:1009D00065633A004552524F5220202020202000CB
:1009E000432D434950532C20522D434950532C2022
:1009F00000000000000000000000000000000000F7
:100A000000000000000000000000000000000000E6
:100A100000000000000000000000000000000000D6
:100A200000000000000000000000000000000000C6
:100A300000000000000000000000000000000000B6
:100A4000004C6F2D434950532C2048692D43495089
:100A5000532C2000000000000000000000000000F7
:100A60000000000000000000000000000000000086
:100A70000000000000000000000000000000000076
:100A80000000000000000000000000000000000066
:100A90000000000000000000000000000000000056
:100AA0000000434950532C200000000000000000CB
:100AB0000000000000000000000000000000000036
:100AC0000000000000000000000000000000000026
:100AD0000000000000000000000000000000000016
:100AE0000000000000000000000000000000000006
:100AF00000000000000000000000000000000000F6
:100B00000000004143564752506F6C2C2041435621
:100B10004752526D732C2000414356474C506F6C26
:100B20002C20414356474C526D732C20414356476D
:100B300052506F6C2C204143564752526D732C20FB
:100B400000000000000000000000000000000000A5
:100B50000000000000000000000000000000000095
:100B60000000000000000000000000000000000085
:100B7000000000000000000000522D4443564720B2
:100B80004F6E2C204C2D44435647204F6E2C204C4A
:100B90006F2D43495053204F6E2C2048692D4349F7
:100BA0005053204F6E2C20522D44435647204F6601
:100BB000662C204C2D44435647204F66662C204C13
:100BC0006F2D43495053204F66662C2048692D43B2
:100BD000495053204F66662C2000522D44435647FF
:100BE000204F66662C204C2D44435647204F6666A6
:100BF0002C204C6F2D43495053204F66662C2048C3
:100C0000692D43495053204F66662C20522D444392
:100C10005647204F6E2C204C2D44435647204F6E94
:100C20002C204C6F2D43495053204F6E2C20486987
:100C30002D43495053204F6E2C2000432D434950E3
:100C400053204F6E2C20522D43495053204F6E2C71
:100C500020432D43495053204F66662C20522D438C
:100C6000495053204F66662C200000000000000011
:100C70000000000000000000000000000000000074
:100C80000000000000000000000000000000000064
:100C9000000000000000000000000000432D434958
:100CA0005053204F66662C20522D43495053204FFD
:100CB00066662C20432D43495053204F6E2C205202
:100CC0002D43495053204F6E2C200000000000009F
:100CD0000000000000000000000000000000000014
:100CE0000000000000000000000000000000000004
:100CF00000000000000000000000000000522D4431
:100D0000435647204F6E2C204C6F2D4349505320A3
:100D10004F6E2C2048692D43495053204F6E2C2094
:100D2000522D44435647204F66662C204C6F2D436E
:100D3000495053204F66662C2048692D4349505333
:100D4000204F66662C20000000000000000000001C
:100D50000000000000000000000000000000522D14
:100D600044435647204F66662C204C6F2D43495014
:100D700053204F66662C2048692D43495053204F1D
:100D800066662C20522D44435647204F6E2C204C33
:100D90006F2D43495053204F6E2C2048692D4349F5
:100DA0005053204F6E2C2000000000000000000077
:100DB0000000000000000000000000000000004CE7
:100DC0006F2D43495053204F6E2C2048692D4349C5
:100DD0005053204F6E2C204C6F2D43495053204FC1
:100DE00066662C2048692D43495053204F66662C77
:100DF00020000000000000000000000000000000D3
:100E000000000000000000000000000000000000E2
:100E100000000000000000000000000000000000D2
:100E20004C6F2D43495053204F66662C2048692D46
:100E300043495053204F66662C204C6F2D43495038
:100E400053204F6E2C2048692D43495053204F6E3C
:100E50002C20000000000000000000000000000046
:100E60000000000000000000000000000000000082
:100E70000000000000000000000000000000000072
:100E800000522D44435647204F6E2C204C2D444396
:100E90005647204F6E2C20462D44435647204F6E18
:100EA0002C20422D44435647204F6E2C20522D4477
:100EB000435647204F66662C204C2D44435647200E
:100EC0004F66662C20462D44435647204F66662CBD
:100ED00020422D44435647204F66662C20000000D8
:100EE0000000522D44435647204F66662C204C2D5F
:100EF00044435647204F66662C20462D44435647B0
:100F0000204F66662C20422D44435647204F66668C
:100F10002C20522D44435647204F6E2C204C2D44FC
:100F2000435647204F6E2C20462D44435647204FB2
:100F30006E2C20422D44435647204F6E2C2000003B
:100F4000000000522D44435647204F6E2C204C2D5C
:100F500044435647204F6E2C2043495053204F6E38
:100F60002C20522D44435647204F66662C204C2D92
:100F700044435647204F66662C2043495053204F28
:100F800066662C2000000000000000000000000049
:100F90000000000000000000000000000000000051
:100FA00000000000522D44435647204F66662C2017
:100FB0004C2D44435647204F66662C2043495053DE
:100FC000204F66662C20522D44435647204F6E2CEE
:100FD000204C2D44435647204F6E2C2043495053FC
:100FE000204F6E2C200000000000000000000000D8
:100FF00000000000000000000000000000000000F1
:101000000000000000522D44435647204F6E2C2014
:101010004C2D44435647204F6E2C20522D444356AE
:1010200047204F66662C204C2D44435647204F6680
:10103000662C2000000000000000000000000000FE
:1010400000000000000000000000000000000000A0
:101050000000000000000000000000000000000090
:10106000000000000000522D44435647204F6666A2
:101070002C204C2D44435647204F66662C20522D81
:1010800044435647204F6E2C204C2D444356472056
:101090004F6E2C2000000000000000000000000047
:1010A0000000000000000000000000000000000040
:1010B0000000000000000000000000000000000030
:1010C00000000000000000522D44435647204F6EA0
:1010D0002C2043495053204F6E2C20522D44435610
:1010E00047204F66662C2043495053204F66662C9C
:1010F00020000000000000000000000000000000D0
:1011000000000000000000000000000000000000DF
:1011100000000000000000000000000000000000CF
:101120000000000000000000522D44435647204FAD
:1011300066662C2043495053204F66662C20522D62
:1011400044435647204F6E2C2043495053204F6E46
:101150002C20000000000000000000000000000043
:10116000000000000000000000000000000000007F
:10117000000000000000000000000000000000006F
:10118000000000000000000000522D44435647209C
:101190004F6E2C20522D44435647204F66662C201C
:1011A000000000000000000000000000000000003F
:1011B000000000000000000000000000000000002F
:1011C000000000000000000000000000000000001F
:1011D000000000000000000000000000000000000F
:1011E00000000000000000000000522D444356475C
:1011F000204F66662C20522D44435647204F6E2CBC
:1012000020000000000000000000000000000000BE
:1012100000000000000000000000000000000000CE
:1012200000000000000000000000000000000000BE
:1012300000000000000000000000000000000000AE
:10124000000000000000000000000043495053204F
:101250004F6E2C2043495053204F66662C200000CF
:10126000000000000000000000000000000000007E
:10127000000000000000000000000000000000006E
:10128000000000000000000000000000000000005E
:10129000000000000000000000000000000000004E
:1012A000000000000000000000000000434950530F
:1012B000204F66662C2043495053204F6E2C20004F
:1012C000000000000000000000000000000000001E
:1012D000000000000000000000000000000000000E
:1012E00000000000000000000000000000000000FE
:1012F00000000000000000000000000000000000EE
:101300000000000000000000000000000044656CC8
:1013100061792054696D653B0046696C65204E61BA
:101320006D653A2000436861696E6167652C200035
:10133000004C6F63616C54696D652C204C6F636168
:101340006C444D592C204C61742D4465672C204C05
:1013500061742D4D696E2C204E532C204C6F6E2DD8
:101360004465672C204C6F6E2D4D696E2C204557BF
:101370002C20466978537461742C204E756D53612E
:10138000742C2050444F502C20416C745F4D2C2005
:1013900043686B2C20436F6D6D000000000000005F
:1013A00000000000000000000000000000004C6F82
:1013B00063616C54696D652C204C6F63616C444DA6
:1013C000592C204C61742D4465672C204E532C20E1
:1013D0004C6F6E2D4465672C2045572C204669784C
:1013E000537461742C204E756D5361742C205044DD
:1013F0004F502C20416C745F4D2C2043686B2C2087
:10140000436F6D6D00000000000000000000000050
:1014100000000000000000000000000000000000CC
:1014200000000000000000000000004C6F63616CD1
:1014300054696D652C204C6F63616C444D592C20B0
:101440004C61742D4465672C204C61742D4D696E80
:101450002C204C61742D5365632C204E532C204C52
:101460006F6E2D4465672C204C6F6E2D4D696E2C70
:10147000204C6F6E2D5365632C2045572C204669F8
:1014800078537461742C204E756D5361742C205008
:10149000444F502C20416C745F4D2C2043686B2CC2
:1014A00020436F6D6D000000484558434F5244453E
:1014B000522043414C4942482E5458540000007772
:1014C00077772E636174682D746563682E636F6D22
:1014D0000000000000004C494D495445442039307B
:1014E000352D3835372D313035300000004341542B
:1014F000484F44494320544543484E4F4C4F475969
:101500000000007B702C30302C662C007B702C305F
:10151000302C657D007B702C30302C6F7D00686333
:1015200069746F6F6C20706169722000456E74651C
:10153000722050494E203A2000686369636F6E66DE
:101540006967206E616D65200061742B6274642A86
:10155000007175697400736D6172745A0061742B47
:1015600072756E00456E746572204143564720289F
:1015700027462720666F722046726F6E742C2027D4
:10158000422720666F72204261636B290A0D206139
:101590006E6420737570706C79203332302B363462
:1015A000302073696E65776176652077697468208D
:1015B0005065616B546F5065616B20766F6C746120
:1015C0006765206F6620302E385600456E74657250
:1015D0002053434F504520766F6C746167652069D6
:1015E0006E206D5620284E4E4E4E4E2900456E748C
:1015F0006572204349505320766F6C746167652093
:10160000696E206D562A313020284E4E4E4E4E299E
:1016100000456E746572204443564720766F6C74A3
:1016200061676520696E206D562A313020284E4E44
:101630004E4E4E29004469736320434F55504F4E20
:10164000204F4E203D20004469736320434F555086
:101650004F4E204F4646203D2000494E5354414EA8
:1016600054204F4E203D2000494E5354414E5420AB
:101670004F4646203D2000AD16A616A2169E169A8D
:1016800016961687168716432D53474E44205B3512
:101690002D3430565D00432D4200432D4600432D2E
:1016A0005200432D4C00522D53474E4400432D53BE
:1016B000474E440020616E6420656E74657220762A
:1016C0006F6C7461676520696E206D562A31302019
:1016D000284E4E4E4E4E2900506C65617365206356
:1016E0006F6E6E65637420004572726F722C206D90
:1016F000697373696E6720414443206E756D2028BD
:10170000302D3729000A0D5363616C696E674361A0
:101710006C6962204F66667365743A200045727288
:101720006F722C20656E74657220766F6C746167C1
:101730006520696E206D562A313020284E4E4E4E5F
:101740004E2900F117D217BC17B0178C1779175113
:101750001743535B302F312F322F332F345D5B769D
:10176000767676765D202D204443205363616C6944
:101770006E672043616C6962004342202D20426104
:1017800074746572792043616C696200435A5B30FE
:101790002F312F322F332F345D202D204443205AF8
:1017A00065726F4F66667365742043616C69620091
:1017B00056202D20566E756D626572004C5B696E09
:1017C000785D5B4F4E2F4F46465D202D204C656463
:1017D0007300416E6E202D205265616420414443A8
:1017E0003120666F72206E6E207365636F6E647356
:1017F0000041202D20526561642041444331004561
:1018000052524F52004F4B004341544820544543DD
:101810004820484558434F52444552205630312EB7
:101820003233000100020003000400050006000A34
:10183000000C000F0014001E003C007800B400F003
:10184000002C01680100000000120002000100B835
:101850000B0F27010064006801100E010010271013
:101860002710271027102710270100010001000171
:1018700000F8010200010002000100F40100000074
:10188000000100000000000A00F1D8000001000182
:1018900000C8000000640064006400640064006428
:1018A00000000000000000000050FE0000000000EA
:1018B0000000000100000000000100000000000A1C
:1018C00000000001000100020058020000FA00FAC6
:1018D00000FA00FA00780078000000000000000123
:1018E00000000001000100000000000100010000F4
:1018F0008000190080001900800019008000190084
:101900008000190080001900800019008000190073
:10191000000100FF03E600E6004F19411933192CBE
:1019200019244A42494E2C39342C3100244A53415F
:10193000564500244A4153432C47504753412C31CC
:1019400000244A4153432C4750524D432C3100242C
:101950004A4153432C47504747412C310024504DB6
:10196000544B3636372A33350024504D544B3331DF
:10197000342C302C312C302C312C312C302C302C80
:10198000302C302C302C302C302C302C302C302C77
:10199000302C302C302C302A323900756E6C6F6749
:1019A000206C62616E64747261636B7374617461E4
:1019B000006C6F67206C62616E64747261636B733C
:1019C00074617461206F6E74696D652031300075CB
:1019D0006E6C6F6720707372706F7361006C6F67ED
:1019E00020707372706F7361206F6E74696D652003
:1019F000313000646174756D20757365720020303C
:101A00002E3020302E3020302E3020302E300075F9
:101A1000736572646174756D2000646174756D2006
:101A2000776773383400756E6C6F67206770616C10
:101A30006D006C6F67206770616C6D206F6E7469EC
:101A40006D6520313000AF1AA01A911A821A7A1AE5
:101A5000611A541A245047524D432C2C2C39362CE1
:101A600000245047524D432C412C2C3130302C2C2B
:101A70002C2C2C2C2C2C2C2C2C00245047524D433D
:101A80004500245047524D4F2C5047524D542C3056
:101A900000245047524D4F2C5047524D462C310098
:101AA000245047524D4F2C47504753562C3000245A
:101AB0005047524D4F2C2C3400101B011BF21AE3DF
:101AC0001AD41AC51A445A203D2000000000000014
:101AD000000000004459203D2000000000000000EC
:101AE0000000004458203D200000000000000000DD
:101AF0000000466C6174203D2000000000000000E2
:101B0000004D616A6F7241203D200000000000001E
:101B10005354505220444154554D2E545854005C57
:101B20001C4F1C421C351C281C1B1C0E1C011CF4C9
:101B30001BE71BDA1BCD1BC01BB31BA61B991B8C01
:101B40001B7F1B721B651B581B4B1B4143564732A7
:101B500020524D53203D2000414356473120524DE5
:101B600053203D200042415454202043616C203DCD
:101B7000200041432020205343616C203D20004140
:101B8000432020205A43616C203D200041444337CC
:101B9000205653636C203D200041444337205A4374
:101BA000616C203D200041444336205653636C2035
:101BB0003D200041444336205A43616C203D2000C3
:101BC00041444335205653636C203D20004144433B
:101BD00035205A43616C203D200041444334205657
:101BE00053636C203D200041444334205A43616CD0
:101BF000203D200041444333205653636C203D2058
:101C00000041444333205A43616C203D200041444D
:101C10004332205653636C203D2000414443322020
:101C20005A43616C203D20004144433120565363A8
:101C30006C203D200041444331205A43616C203DDB
:101C4000200041444330205653636C203D20004126
:101C5000444330205A43616C203D200046696C6546
:101C600020496E646578203D20000A1FF41EDE1EA8
:101C7000C81EB21E9C1E861E701E5A1E441E2E1E9C
:101C8000181E021EEC1DD61DC01DAA1D941D7E1D12
:101C9000681D521D3C1D261D101DFA1CE41CCE1C87
:101CA000B81C454E44000000000000000000000089
:101CB00000000000000000004443564720446566D1
:101CC0006563742056616C203D2000000000444391
:101CD00056472044656665637420456E203D2000AC
:101CE0000000000053796E632054797065203D2018
:101CF0000000000000000000000043495053205243
:101D0000616E6765202B2F2D3556203D2000000089
:101D100047505320436F6F726420666F726D617419
:101D2000203D200000004C6F63616C4750535469A4
:101D30006D654F6666736574203D20004143204603
:101D400072657175656E6379203D200000000000AA
:101D5000000042726F6B656E5769726520416C615D
:101D6000726D203D200000004C6F7720506F742072
:101D7000416C61726D203D20000000000000496E42
:101D800070757420496D706564616E6365203D20D7
:101D900000000000444356474D44656C4F4E203DC3
:101DA00020000000000000000000444356474D445E
:101DB000656C4F4646203D200000000000000000FA
:101DC00043495053324D44656C4F4E203D20000036
:101DD00000000000000043495053324D44656C4FF1
:101DE0004646203D200000000000000043495053BB
:101DF000314D44656C4F4E203D2000000000000036
:101E0000000043495053314D44656C4F4646203DD8
:101E10002000000000000000537461727457697460
:101E200068203D20000000000000000000004F6618
:101E30006654696D65205B6D7365635D203D2000B0
:101E400000000000546F74616C4379636C65205B23
:101E50007365635D203D2000000054696D65205668
:101E6000616C7565203D200000000000000000004E
:101E7000436861696E61676520446972656374696E
:101E80006F6E203D20005374617274204368616955
:101E90006E616765203D2000000000004469737496
:101EA000616E63652056616C7565203D2000000001
:101EB00000004D6561737572656D656E7420556EB9
:101EC000697473203D20000053746F726167652050
:101ED000416374696F6E203D20000000000053755F
:101EE000727665792054797065203D2000000000ED
:101EF000000000004F70657261746F72204E616D5A
:101F000065203D2000000000000053757276657961
:101F1000204E616D65203D200000000000000000A3
:101F200054532D5453204F4E203D200054532D54D4
:101F300053204F4646203D20004E45572054532005
:101F40004F4E203D20004E4557205453204F4646CB
:101F5000203D20005453204F4E203D20005453205C
:101F60004F4646203D20000011241FBECFEFCDBFBD
:101F7000DFE5DEBF00E00CBF1FE2A0E0B0E2E8E575
:101F8000F4ED02E00BBF02C007900D92AA3FB1072B
:101F9000D9F724E5AAEFBFE201C01D92A63BB20724
:101FA000E1F70E94743F0D942A6A0C940000CF93CD
:101FB000DF93CDB7DEB72B97CDBFDEBFBE016F5F1E
:101FC0007F4F80E092E00F949261AE01485F5F4FD7
:101FD00068E080E092E00F94EE618A819B819F78B7
:101FE0009B8395E09D83817E8A831C82BE016F5F07
:101FF0007F4F80E092E00F94426181E0888788E122
:102000008987AE01485F5F4F68E080E092E00F94FF
:10201000B56180E092E00F94A35F2B96CDBFDEBF49
:10202000DF91CF9108959FB7F894E0E0F2E08081CE
:10203000806280839FBF0895009781F020910602FF
:1020400023FF0EC020913C0230913D02FC01208311
:10205000318388E08093060281E0089580E008954E
:1020600080E00895CF92DF92EF92FF92CF93DF93BB
:102070000097D1F061157105C9F0EB01FC01A08159
:10208000B18128EE33E00F9442656B017C0183E15E
:102090000E94A6D09B01AC01C701B6010F94ED646C
:1020A0002883398381E003C080E001C080E0DF91B4
:1020B000CF91FF90EF90DF90CF900895EDE1F9E39D
:1020C0001082118214821582128213821682178264
:1020D0008BE00E94CAD0672B682B692B19F41092F1
:1020E000253903C081E080932539EDE1F9E31186BC
:1020F00012860895CF93DF93EC01892B09F491C0E8
:10210000862F90E0FC013197EB30F10508F089C093
:102110008827E250FF4F8F4F0D942B658091253912
:10212000811107C088819981809321399093223948
:1021300078C08A819B81809321399093223971C024
:1021400080912539811107C08A819B818093213933
:102150009093223966C08E819F818093213990931C
:1021600022395FC080912539811107C08C819D8102
:10217000809321399093223954C08A859B8580931E
:102180002139909322394DC08091253981110BC09E
:1021900088819981EDE1F9E3848395838A819B812C
:1021A000868397833EC08C819D81EDE1F9E3848332
:1021B00095838E819F818683978333C08091253953
:1021C00081110BC08A819B81EDE1F9E384839583C2
:1021D0008C819D818683978324C0EDE1F9E3888516
:1021E0009985848395838A859B858683978319C087
:1021F0008091253981110BC08C819D81EDE1F9E33E
:10220000848395838E819F81868397830AC0EDE1C5
:10221000F9E38C859D85848395838E859F85868350
:102220009783DF91CF910895EDE1F9E38481958162
:102230008083918386819781828393830895EDE1E2
:10224000F9E381E0818712860895EDE1F9E31186D3
:102250001286089580912739089583E10E94CAD09B
:10226000672B682B692B19F080912639089580E03F
:102270000895CF92DF92EF92FF926B01072E000C30
:10228000EE08FF08C216D306E406F5067CF48617AE
:102290009707E4F0092E000CAA0BBB0BE1E028170E
:1022A00039074A075B07ACF4E0E013C06C01092E64
:1022B000000CEE08FF08C216D306E406F50644F04B
:1022C000E1E0681779072CF4E0E003C0E0E001C02A
:1022D000E0E08E2FFF90EF90DF90CF900895FF9277
:1022E0000F931F93CF93DF93CDE1D9E301E219E37D
:1022F000F12CE991F991309719F1AF010F2E000CF3
:10230000660B770BDB01CA0177231CF40196A11D34
:10231000B11DB595A795979587959A01AB01280FA3
:10232000391F4A1F5B1FBF01FF2314F46F5F7F4FEC
:10233000759567958A819B819CDF813009F0F394C4
:10234000C017D107B1F6FF2011F079DF01C07DDFA2
:102350006BDFDF91CF911F910F91FF900895EDE119
:10236000F9E381E090E0A0E0B0E08787908BA18B5B
:10237000B28B838B948BA58BB68B178A13861486AE
:1023800015861686108E0895EDE1F9E381E0878BBE
:10239000108E0895EDE1F9E3178A108E089580916B
:1023A0003539089584E10E94CAD0672B682B692BC8
:1023B00019F080913439089580E00895EDE1F9E352
:1023C00087859089A189B289838B948BA58BB68BE5
:1023D00083859485A585B6858787908BA18BB28BE5
:1023E0000895609328397093293980932A399093FE
:1023F0002B3908958F929F92AF92BF92CF92DF9226
:10240000EF92FF92EDE1F9E3C388D488E588F6887E
:1024100087859089A189B289C816D906EA06FB0684
:1024200091F48090283990902939A0902A39B09061
:102430002B39C4DFC814D904EA04FB0411F4A4DF67
:1024400004C0A8DF02C0BADFFCCFFF90EF90DF909E
:10245000CF90BF90AF909F908F9008958BE10E9496
:10246000CAD0609336397093373980933839909356
:102470003939AAE3B9E3EDE1F9E385E299E31D9285
:1024800011A212A232968E179F07C9F7EDE1F9E368
:1024900011A612A6089581E090914639911101C0CC
:1024A00080E008958AE10E94CAD0672B682B692BCF
:1024B00039F081E090914639911103C080E0089590
:1024C00080E008950F931F938B019C018091363912
:1024D00090913739A0913839B09139390097A105D9
:1024E000B10529F1880F991FAA1FBB1FAC01BD01BF
:1024F000440F551F661F771F440F551F661F771F18
:10250000840F951FA61FB71FB901A80133233CF400
:1025100044275527BA01401B510B620B730B21E076
:1025200084179507A607B7071CF020E001C020E03C
:10253000822F1F910F9108950F931F93CF93DF93D5
:10254000009709F40BC1ADE1B9E35D961C925D976C
:102550005E961C925E975F961C925F9790961C9277
:10256000462F50E0FA013297EA30F10508F0F6C044
:10257000EC018827E75FFE4F8F4F0D942B6580910C
:102580002539811108C06C817D818E819F819ADF00
:1025900080933A39E3C0688179818A819B8192DF97
:1025A00080933A39DBC080912539811108C0688554
:1025B00079858A859B8586DF80933A39CFC068818B
:1025C00079818A819B817EDF80933A39C7C080916F
:1025D0002539811111C0688579858A859B8572DFCF
:1025E0000DE119E3F801858F6C857D858E859F85CA
:1025F00069DFF801868FB2C0688179818A819B8109
:1026000061DF0DE119E3F801858F6C817D818E8199
:102610009F8158DFF801868FA1C0809125398111F3
:1026200011C06C857D858E859F854CDF0DE119E39A
:10263000F801858F688979898A899B8943DFF80148
:10264000868F8CC0688179818A819B813BDF0DE117
:1026500019E3F801858F6C817D818E819F8132DF46
:10266000F801868F7BC08091253981111FC0688950
:1026700079898A899B8926DF0DE119E3F801858F25
:102680006C897D898E899F891DDFF801868F688D11
:10269000798D8A8D9B8D16DFF801878F6C8D7D8DEE
:1026A0008E8D9F8D0FDFF80180A358C068817981DE
:1026B0008A819B8107DF0DE119E3F801858F6C8129
:1026C0007D818E819F81FEDEF801868F6885798508
:1026D0008A859B85F7DEF801878F6C857D858E85E1
:1026E0009F85F0DEF80180A339C0809125398111E2
:1026F00011C0688979898A899B89E4DE0DE119E333
:10270000F801858F6C897D898E899F89DBDEF801D0
:10271000868F24C0688179818A819B81D3DE0DE117
:1027200019E3F801858F6C817D818E819F81CADEDE
:10273000F801868F13C080912539811108C06C85FE
:102740007D858E859F85BEDE80933A3907C068817E
:1027500079818A819B81B6DE80933A39DF91CF916E
:102760001F910F910895843040F5EDE1F9E341A503
:1027700052A5242F30E0082E02C0359527950A94E3
:10278000E2F720FF0AC0252F30E0082E02C0359561
:1027900027950A94E2F720FD10C021E030E0B9014E
:1027A00002C0660F771F8A95E2F7CB01EDE1F9E3EE
:1027B000462B41A78095852382A70895843090F405
:1027C00021E030E0A90102C0440F551F8A95E2F7CD
:1027D000CA018095EDE1F9E391A5982391A792A50F
:1027E000892382A70895BF92CF92DF92EF92FF9242
:1027F0000F931F93CF93DF930AE319E3CDE1D9E35E
:102800006E017801B12CF70181917F01F60121A1C0
:1028100090E0820F911D22A1820F911D039719F460
:102820008B2DA1DF02C08B2DC9DFB394F2E0CF0E58
:10283000D11C84E0B812E7CF25E239E389A18AA34D
:10284000F80181918F0189A32296C217D307B1F7AE
:10285000DF91CF911F910F91FF90EF90DF90CF907C
:10286000BF900895843060F42091463930E0A9018A
:1028700002C0559547958A95E2F7CA01817008957F
:1028800080E00895843060F42091473930E0A90158
:1028900002C0559547958A95E2F7CA01817008955F
:1028A00081E00895843000F5662379F0EDE1F9E3E5
:1028B00021E030E0A90102C0440F551F8A95E2F7DC
:1028C000CA0192A5892B82A70895EDE1F9E321E0E1
:1028D00030E0A90102C0440F551F8A95E2F7CA01F2
:1028E000809592A5892382A70895CF93833009F11B
:1028F00028F4813031F0823061F02CC0883008F14A
:1029000029C080913439882329F181E080933539B9
:1029100021C0C1DD8823F1F061E080E0C3DF61E028
:1029200081E0C0DF61E082E0BDDF61E083E0BADF2B
:1029300011C080912639882369F081E0809327397E
:1029400009C0CCEFC80F8C2F8DDF882319F061E010
:102950008C2FA8DFCF910895009781F0FC01DC0156
:10296000AD5BBD4F80818C936083643021F481E046
:102970000D945D16089580E00D945D1608950097FE
:1029800019F0FC018081089580E00895009741F0DE
:10299000613021F421E0FC0122AB0895FC0112AA70
:1029A0000895009719F0FC0182A9089580E0089528
:1029B000009741F0613021F421E0FC0123AB089540
:1029C000FC0113AA0895009719F0FC0183A908954A
:1029D00080E008958F929F92AF92BF92DF92EF9224
:1029E000FF920F931F93CF93DF934115510509F485
:1029F0006BC08A017B01C82F0E94C0D4D82F8C2FB6
:102A00000E94DDD4D82EDD2309F460C0882309F4A8
:102A10005FC08D2F0E94A6D04B015C018D2D0E94BE
:102A2000A6D0672B682B692B39F4F801108211822C
:102A30001282138280E04DC09701280D391D032EAC
:102A4000000C440B550BC63050F4A0E1B7E20F94D4
:102A50004865F801608371838283938309C0A8EE7F
:102A6000B3E00F944865F801608371838283938398
:102A70008D2D0E94A6D09B01AC01F801608171816F
:102A8000828193810F940F6588279927DC01821B2F
:102A9000930BA40BB50BF80180839183A283B383BE
:102AA0008C2F0E9483D8F80180809180A280B3800F
:102AB000DC01CB01880D991DAA1DBB1D808391836C
:102AC000A283B38381E005C080E003C080E001C041
:102AD00080E0DF91CF911F910F91FF90EF90DF90F9
:102AE000BF90AF909F908F900895CF93DF93009702
:102AF00009F460C0EC010F942E29813091F58C838C
:102B00000F9485118823F9F08091493F811119C0F4
:102B100089E0E4EEF0E2A0EDB4E401900D928A9534
:102B2000E1F7E0EDF4E401900020E9F73197AF011F
:102B3000405D544421E060ED74E48AEA99E30F9427
:102B4000F0310F94BE110F948811882399F18EEB08
:102B500098E40E94D1DE0F9482118A830F94CF11E2
:102B600029C01C820F945A298823F9F08091493F8B
:102B7000811119C089E0EDEEF0E2A0EDB4E401901E
:102B80000D928A95E1F7E0EDF4E401900020E9F779
:102B90003197AF01405D544421E060ED74E48AEA6E
:102BA00099E30F94F0310F945D290F944629811118
:102BB0000F944929DF91CF9108950F931F93CF93DD
:102BC000DF93009709F463C0EC010F94A52B8823D1
:102BD00081F18B8181115BC08091493F811126C0B9
:102BE0000F946E29182F0F9482111F921F931F921A
:102BF0008F938FEF90E29F938F9300ED14E41F93D8
:102C00000F930F945867F80101900020E9F731976E
:102C1000AF01405D544420E0B8018AEA99E30F9483
:102C2000F0318DB79EB708968DBF9EBF81E08B8334
:102C30002EC08B81813059F51B828091493F8111D3
:102C400026C00F946E29C82F0F9482111F92CF9324
:102C50001F928F9386EF90E29F938F93C0EDD4E401
:102C6000DF93CF930F94586709900020E9F72197DD
:102C7000AE01405D544420E060ED74E48AEA99E3DB
:102C80000F94F0318DB79EB708968DBF9EBFDF9130
:102C9000CF911F910F910895CF92DF92EF92FF9203
:102CA0000F931F93CF93DF93009709F4AAC0611588
:102CB000710509F4A6C08B01EC010E946FDE882328
:102CC00009F49FC00F94ED296B017C010F94922BA6
:102CD00086E10E94CAD0AB01BC0183E29DE30E9461
:102CE00005DFD701C6010197A109B109883E9340CC
:102CF000A105B10508F03FC00E94D9C8823088F113
:102D00008091493F81112DC00F9482111F928F93A2
:102D100080912B541F928F93FF92EF92DF92CF926C
:102D200082E191E29F938F930F2EF0EDEF2EF4E46A
:102D3000FF2EF02DFF92EF920F945867F70101904C
:102D40000020E9F73197AF01405D544421E0B7011D
:102D50008AEA99E30F94F0318DB79EB70C968DBF38
:102D60009EBF25ED35E44FEE57E469E277E4C801F4
:102D70000E94D3EA43C0D701C601895E9340A109EE
:102D8000B10984369105A105B105C0F58FEE95E432
:102D90000E9467DE811132C08091493F811125C0B8
:102DA000FF92EF92DF92CF928EE191E29F938F9309
:102DB0000F2EF0EDEF2EF4E4FF2EF02DFF92EF92A8
:102DC0000F945867F70101900020E9F73197AF01A0
:102DD000405D544421E0B7018AEA99E30F94F03151
:102DE0008DB79EB708968DBF9EBF25ED35E44FEE9B
:102DF00057E469E277E4C8010E94D3EACE010E9459
:102E000088DEDF91CF911F910F91FF90EF90DF90BF
:102E1000CF900895FC01892B39F0118689E0DF01FC
:102E20001D928A95E9F712860895FC01892B41F0DD
:102E3000118689E0DF011D928A95E9F712861386D3
:102E400008950F931F93CF93DF93CBE4D9E303EA65
:102E500019E3CE01DFDF2B96C017D107D1F78FED35
:102E60009CE3E3DF8BEE9CE3E0DF0F940B2EDF911E
:102E7000CF911F910F910895FC01892B31F081E0D2
:102E80009285913019F080E0089580E008951F93B5
:102E9000CF93DF93CDB7DEB76097CDBFDEBF9C0188
:102EA000FE013196AE014F5E5F4F21933193255F56
:102EB0003F4FE417F507C9F7892B31F110E010C037
:102EC000E12FF0E0EE0FFF1F81E090E08C0F9D1FDF
:102ED000E80FF91F80819181CFDF8823D1F01F5F38
:102EE0000F94922C181760F382E00E94CAD06B30C6
:102EF00068F08091EA3C882359F081E09091F63C9B
:102F0000911107C080E005C080E003C081E001C0EE
:102F100080E06096CDBFDEBFDF91CF911F91089515
:102F2000CF92DF92EF92FF920F931F93CF93DF9395
:102F3000CDB7DEB72597CDBFDEBF19821A821B82BF
:102F40001C824115510559F16A017B01182FCA01F4
:102F500061DFAE014F5F5F4FB701812F3BDD8823FB
:102F6000C9F009811A812B813C814BE0BE016B5F66
:102F70007F4FC6010F947439F60101900020E9F7E4
:102F80003197EC19FD09D6011996EC93199781E058
:102F90001A968C9369817A818B819C8103C060E051
:102FA00070E0CB012596CDBFDEBFDF91CF911F91A1
:102FB0000F91FF90EF90DF90CF9008958F929F92A6
:102FC000AF92BF92EF92FF920F931F93CF93DF9335
:102FD0000097A1F06115710589F0142F7B01EC01B8
:102FE0000F9490164B015C01113009F4FAD9950148
:102FF00084014BE0B701CE010F94C637DF91CF912A
:103000001F910F91FF90EF90BF90AF909F908F9086
:103010000895AF92BF92CF92DF92EF92FF920F93FB
:103020001F93CF93DF93CDB7DEB76097CDBFDEBFE1
:103030008C01CE0101967C014096F701619371935A
:10304000655F7F4FE817F907C9F70115110509F406
:1030500075C282E00E94CAD0D62E96E0D91206C070
:10306000C8010F94DC2781116FC243C38FEF8D0D10
:10307000823030F4C8010F94DC27811111C039C3AC
:103080008FEE8D0D823030F4C8010F94DC27811152
:1030900007C02FC3C8010F94DC27882309F429C374
:1030A00080E2E3E7F0E4DF011D928A95E9F780E131
:1030B000E8EBFBE3DF011D928A95E9F78D2D90E0A7
:1030C000FC013197E231F10508F03AC28827ED5E44
:1030D000FE4F8F4F0D942B6558010F2EF3E7CF2E27
:1030E000F0E4DF2EF02D01E010E00EC10F94D9279F
:1030F000C82E49815A81F8016081718111DF0F2E3C
:10310000F3E7EF2EF0E4FF2EF02DD7016D937D93C2
:103110008D939C9313974B815C81F801628173813D
:103120008C2DFEDED70114966D937D938D939C9329
:103130001797B2E0DB1206C2809173409091744001
:10314000A0917540B09176408093B83B9093B93B85
:10315000A093BA3BB093BB3B81E0CBC258010F2E8A
:10316000F3E7CF2EF0E4DF2EF02D01E010E00BC0EE
:103170001F5F0F5FE2E0EE0EF11CF2E0AF0EB11C3C
:1031800084E0C80ED11C112309F4FBC1123009F4EC
:10319000EAC1D7014D915C91F5016081718180E0B8
:1031A000BFDED6016D937D938D939C93139704306E
:1031B000F8F28091734090917440A0917540B09165
:1031C00076408093B83B9093B93BA093BA3BB093C1
:1031D000BB3B81E08EC258010F2EF3E7CF2EF0E407
:1031E000DF2EF02D01E010E00BC01F5F0F5FB2E09B
:1031F000EB0EF11CE2E0AE0EB11CF4E0CF0ED11CE0
:10320000112309F4DBC1123009F4CAC1D7014D9171
:103210005C91F5016081718182E082DED6016D935F
:103220007D938D939C9313970430F8F2E8EBFBE3C6
:10323000A3E7B0E44D915D916D917C91139740832C
:1032400051836283738314968D919D910D90BC91EF
:10325000A02D84839583A683B78381E04AC2580159
:103260000F2EF3E7CF2EF0E4DF2EF02D01E010E07B
:103270000BC01F5F0F5FB2E0EB0EF11CE2E0AE0E81
:10328000B11CF4E0CF0ED11C112309F4B8C11330E6
:1032900009F4A3C1113009F4A2C1143009F4A1C189
:1032A000D7014D915C91F5016081718180E038DE3C
:1032B000D6016D937D938D939C9313970630C8F23E
:1032C000E8EBFBE3A3E7B0E44D915D916D917C9158
:1032D0001397408351836283738314968D919D91DC
:1032E0000D90BC91A02D84839583A683B78381E044
:1032F00000C21F5F0F5FB2E0EB0EF11CE2E0AE0E0A
:10330000B11CF4E0CF0ED11C112309F487C1143095
:1033100009F492C1812F8B7F813009F48FC18230F3
:1033200009F48EC1D7014D915C91F50160817181E5
:1033300085E0F6DDD6016D937D938D939C93139775
:103340000830B8F2E8EBFBE3A3E7B0E44D915D9100
:103350006D917C911397408351836283738314969C
:103360004D915D916D917C91179744835583668350
:10337000778318964D915D916D917C911B97408755
:103380005187628773871C968D919D910D90BC919A
:10339000A02D84879587A687B78781E0AAC15801A9
:1033A0000F2EF3E7CF2EF0E4DF2EF02D01E010E03A
:1033B0000BC01F5F0F5FB2E0EB0EF11CE2E0AE0E40
:1033C000B11CF4E0CF0ED11C112309F458C1143004
:1033D00009F445C1812F8B7F813009F442C1D701A7
:1033E0004D915C91F5016081718180E099DDD6019C
:1033F0006D937D938D939C9313970830D0F2E8EBF7
:10340000FBE3A3E7B0E44D915D916D917C9113973F
:10341000408351836283738314968D919D910D90A7
:10342000BC91A02D84839583A683B78381E061C17D
:10343000680103E710E45E01B9E0AB0EB11CF701CF
:10344000419151917F01D6016D917D916D0180E097
:1034500067DDF80161937193819391938F01EA1471
:10346000FB0469F781E045C158010F2EF3E7CF2E29
:10347000F0E4DF2EF02D01E010E00BC01F5F0F5FC6
:10348000F2E0EF0EF11C82E0A80EB11C94E0C90E30
:10349000D11C112309F410C1133009F4FFC0D70166
:1034A0004D915C91F5016081718180E039DDD6013B
:1034B0006D937D938D939C9313970630F8F28091D2
:1034C000734090917440A0917540B0917640809384
:1034D000B83B9093B93BA093BA3BB093BB3B81E020
:1034E00008C158010F2EF3E7CF2EF0E4DF2EF02DA8
:1034F00001E010E00BC01F5F0F5FB2E0EB0EF11CAC
:10350000E2E0AE0EB11CF4E0CF0ED11C112309F4A1
:10351000E2C0D7014D915C91F5016081718181E03C
:10352000123009F480E0FCDCD6016D937D938D931D
:103530009C9313970430F8F281E0DBC080E0D9C09F
:1035400080E0D7C081E0D5C080E2E3E7F0E4DF01AE
:103550001D928A95E9F780E1E8EBFBE3DF011D921C
:103560008A95E9F7B9CDF70140815181D5016D9177
:103570007C9183E0D5DCF601608371838283938341
:10358000F7CDD7014D915C91F5016081718183E0A8
:10359000C7DCD6016D937D938D939C931397E8CDF3
:1035A000F70140815181D5016D917C9183E0B8DCB8
:1035B000F601608371838283938317CED7014D9187
:1035C0005C91F5016081718183E0AADCD6016D9385
:1035D0007D938D939C93139708CE83E003C082E084
:1035E00001C082E0F70140815181D5016D917C914C
:1035F00097DCF60160837183828393833ACED7018F
:103600004D915C91F5016081718183E089DCD60187
:103610006D937D938D939C9313972BCEF7014081EF
:103620005181D5016D917C9183E07ADCF601608354
:103630007183828393835DCE83E003C082E001C007
:1036400084E0D7014D915C91F5016081718168DC66
:10365000D6016D937D938D939C9313974ACE83E00F
:1036600001C082E0F70140815181D5016D917C91CB
:1036700057DCF60160837183828393839ACED701EE
:103680004D915C91F5016081718183E049DCD60147
:103690006D937D938D939C9313978BCEF70140810F
:1036A0005181D5016D917C9183E03ADCF601608314
:1036B000718382839383E2CED7014D915C91F501B2
:1036C0006081718183E02CDCD6016D937D938D93B5
:1036D0009C931397D3CEF70140815181D5016D9111
:1036E0007C9180E01DDCF60160837183828393838B
:1036F00002CF6096CDBFDEBFDF91CF911F910F91BA
:10370000FF90EF90DF90CF90BF90AF9008950F940F
:103710004225882329F00F94532584E080932706BF
:103720000895CF93DF93009799F1EC018881813060
:10373000A8F0833018F0863019F010C0E8DF25C0FB
:103740008091280682FD03C084E0809325060F94B3
:10375000DC248823D1F00F94ED2417C00F94DC24CF
:10376000882399F00F94ED2484E0809327060DC000
:103770008D8181110DC00F942025882349F00F946D
:10378000312584E08093270603C08881863081F745
:10379000DF91CF9108950E94A9E20F94722A20E14F
:1037A00037E240E050E00F94ED64672B682B692B03
:1037B000E1F40E94A9E2813019F40C94BDE108956E
:1037C0000E94A9E2823021F481E00C94ACE20895D9
:1037D0000E94A9E2833019F40C94B2E408950E9487
:1037E000A9E2843011F40C9406E508950F931F9319
:1037F000CF93DF931F921F92CDB7DEB719821A8243
:103800000097B9F08C010E94095790E006969E013E
:103810002F5F3F4F43E060E0800F911F0F942536EC
:10382000882339F049815A8160E070E080E00E948D
:10383000B5D00F900F90DF91CF911F910F91089508
:103840009F92AF92BF92CF92DF92EF92FF920F932F
:103850001F93CF93DF931F92CDB7DEB7009709F484
:103860004BC05C0182E00E94CAD0962E8501085DA3
:103870001F4FBE016F5F7F4FC8010E947CEF8823FE
:1038800091F0F501C0A4D1A4E2A4F3A489E00E94C0
:10389000CAD0AB01BC010AE619E42AE539E4898102
:1038A0000F948D2A17C0BE016F5F7F4FC8010E9421
:1038B000C8F8F501C0A4D1A4E2A4F3A489E00E9451
:1038C000D8D0AB01BC010AE619E42AE539E48981C4
:1038D0000F948D2AFAE0F91558F4F50140A551A589
:1038E00062A573A582E599E40F94722D81E005C06D
:1038F0000F94DC2D81E001C080E00F90DF91CF912B
:103900001F910F91FF90EF90DF90CF90BF90AF90FD
:103910009F900895CF92DF92EF92FF920F931F93A3
:10392000CF93DF931F92CDB7DEB7009779F18C016B
:10393000BE016F5F7F4F88960E94C3FB882399F07A
:10394000F801C0A4D1A4E2A4F3A489E00E94CAD0E3
:10395000AB01BC010AE619E42AE539E489810F9438
:103960008D2A81E014C0F801C0A4D1A4E2A4F3A47C
:1039700089E00E94D8D0AB01BC010AE619E42AE52F
:1039800039E489810F948D2A81E001C080E00F9095
:10399000DF91CF911F910F91FF90EF90DF90CF902B
:1039A000089589E10E94CAD0623059F482E00E94F1
:1039B000CAD0673041F0693031F0613021F081E0E8
:1039C000089580E0089580E0089589E10F948017BC
:1039D000623059F482E00F948017673041F069300B
:1039E00031F0613021F081E0089580E0089580E0B9
:1039F00008953F924F925F926F927F928F929F9223
:103A0000AF92BF92CF92DF92EF92FF920F931F93EC
:103A1000CF93DF93CDB7DEB76497CDBFDEBFB82EAF
:103A20008B017A0189E10E94CAD0A62E01151105E9
:103A300009F472C28091493F882339F00F2EFAEAC7
:103A4000CF2EF9E3DF2EF02D06C00F2EF1EBCF2E97
:103A5000FAE3DF2EF02D82E08A1508F4A12C8BE723
:103A6000F801808383E781838CE28283F2E3BF12D3
:103A700007C082E38A0DF80183838CE284830BC044
:103A8000F801B3828CE28483F0E3BF1609F4F1C13C
:103A900082E3B81218C28BE499E3FE0132969E01CC
:103AA0002E5E3F4F819391930B962E173F07D1F7D0
:103AB00088E08983E114F10469F086E0F701D80118
:103AC000159601900D928A95E1F70F2EFBE0FF2EDF
:103AD000F02D04C00F2EF5E0FF2EF02DF801EF0DB4
:103AE000F11D8CE2808382E00E94CAD0762E872D61
:103AF000072C000C990B9F937F928BE191E29F938F
:103B00008F93F394C8018F0D911D9F938F930F9402
:103B10005867F80101900020E9F73197E01BF10B9D
:103B20007F01FF24F801EE0DFF1D118221E0A701A6
:103B3000B801C6010F94F0310F900F900F900F90C5
:103B40000F900F908091493F811112C01A8A21E095
:103B500040E050E0BE016E5E7F4F8AEA99E30F9429
:103B6000F03120E0A701B8018AEA99E30F94F0311F
:103B700091E09A1508F402C11982912C0F2EFCE2F3
:103B80008F2EF02DF8013196EB8BFC8B0F2EF9E484
:103B90004F2EFFE35F2EF02D5BC00F94922C6980B7
:103BA000861509F45BC0F8018082E62CF12CF70140
:103BB000EE0FFF1F81E090E08C0F9D1FE80FF91FB3
:103BC000A180B280F501418550E0B5018B899C89C7
:103BD0000F942A67F50181856894332431F8380EF3
:103BE0008F5FF801E80FF11D8082F7013196EE0F2B
:103BF000FF1F81E090E08C0F9D1FE80FF91FA1804F
:103C0000B280F501418550E0B501C801830D911DD9
:103C10000F942A67F501E1843E0C639463946982F2
:103C2000E32CF12CF801EE0DFF1D118221E0A7011C
:103C3000B801C6010F94F031F2018081811107C0F3
:103C400020E0A701B8018AEA99E30F94F031939438
:103C50000F94922C8695981608F49FCFFAE0F715EA
:103C60000CF0D8C08CE078164CF09DE097150CF065
:103C700050C180EF870D833008F44BC1198280E07A
:103C80000F2EFCE23F2EF02D4801EFEF8E1A9E0A18
:103C90000F2EF9E44F2EFFE35F2EF02DF801308256
:103CA000E82EF12CF701EE0FFF1FEE0DFF1DEE0FBA
:103CB000FF1FEE0FFF1FE152F34C82858C3419F089
:103CC000823541F00EC080E39CE2F4018083918351
:103CD00012820FC081E39CE2F401808391831282FF
:103CE00008C085E0E0E3F1E2D40101900D928A95ED
:103CF000E1F7F80101900020E9F731975F01A01A80
:103D0000B10A3701660C771CB3016E0D7F1D660F7B
:103D1000771F660F771F6152734CFB01418550E09E
:103D2000C8018A0D911D0F942A67F301EE0DFF1D46
:103D3000EE0FFF1FEE0FFF1FE152F34C8185A80E1F
:103D4000B12CF801EA0DFB1D118221E0A501B8019B
:103D5000C6010F94F031F2018081811107C020E08B
:103D6000A501B8018AEA99E30F94F031E98081E076
:103D70008E0D8983823008F491CF4CC01982612C5A
:103D80000F2EFCE25F2EF02D4801FFEF8F1A9F0AE5
:103D90000F2EF9E4AF2EFFE3BF2EF02D36C00F94A7
:103DA000922C79808715B1F1F8015082E72DF0E06F
:103DB000EE0FFF1F81E090E08C0F9D1FE80FF91FB1
:103DC000E180F280F701418550E0B701C4010F9412
:103DD0002A67F701E184E39473947982F12CF80166
:103DE000EE0DFF1D118221E0A701B801C6010F945D
:103DF000F031F5018081811107C020E0A701B801F1
:103E00008AEA99E30F94F03163940F94922C86958B
:103E1000681628F20F2EFCE2FF2EF02DF801F0823A
:103E200084E00E94CAD0605DF8016183F28240E0C4
:103E3000BE016F5F7F4FC8010396C0D8898193E0B0
:103E4000980FF801E90FF11D9DE790838C5FE82E34
:103E5000F12CF801EE0DFF1D118221E0A701B80140
:103E6000C6010F94F0318091493F882309F445C081
:103E700053C00F2EF8E2EF2EF7E4FF2EF02DF701DE
:103E8000408150E061EF76E4C80105960F942A67FF
:103E9000F701808195E0980FF801E90FF11D9DE78A
:103EA00090838A5FE82EF12CF801EE0DFF1D118240
:103EB00021E0A701B801C6010F94F0318091493F7C
:103EC00081112AC011C021E045E050E0B801C601CF
:103ED0000F94F0318091493F81111EC0F0E3BF1271
:103EE0000FC045E050E002C04E2D5F2D20E0B8012C
:103EF0008AEA99E30F94F0310FC04E2D5F2D02C076
:103F000045E050E021E0B8018AEA99E30F94F031EE
:103F100003C081E08983B4CE6496CDBFDEBFDF915C
:103F2000CF911F910F91FF90EF90DF90CF90BF90B6
:103F3000AF909F908F907F906F905F904F903F9049
:103F40000895CF93892B81F00E941756CAE00E94F2
:103F5000DA560E941456882321F00E942A568111B5
:103F600005C0C150A1F703C0C0E001C0C1E08C2F63
:103F7000CF91089589E10E94CAD0611104C00F94C5
:103F80009911882371F081E040913054509131545F
:103F90006091325470913354452B462B472B09F0D6
:103FA00080E008958F929F92AF92BF92CF92DF925E
:103FB000EF92FF920F931F93CF93DF930097A9F196
:103FC000EC0186E00E94CAD04B015C0184E00E94B3
:103FD000CAD0162F87E00E94CAD0062F812F0F94D7
:103FE00074160F9490166B017C0186169706A8062E
:103FF000B906D9F0AB01BC0186E00E941ED6882329
:10400000A1F00F941D16B701A60186E00E94C0D052
:10401000B701A60186E00F949317602F812F0F94AC
:10402000741668E0CE010E94AC14DF91CF911F910D
:104030000F91FF90EF90DF90CF90BF90AF909F9047
:104040008F90089582E10E94CAD028E0E2E6F4E56C
:10405000DF01322F1D923A95E9F7EAE6F4E5DF0138
:104060001D922A95E9F721E030E0672B682B692B38
:1040700011F420E030E0F901E153FF4D80818560CB
:10408000E8E2F4E582AF83AF81E00895CF93DF9358
:104090000097A1F0613071F4EC01E3EBF0E4628190
:1040A0007381808191810F947958CA5CDD4F81E0E2
:1040B000888304C0FC01EA5CFD4F1082DF91CF9140
:1040C00008950097B1F0FC0180818430A1F40F9431
:1040D000C529823039F089E10E94CAD0672B682B4C
:1040E000692B59F00F94A22991E0811107C090E04B
:1040F00005C090E003C090E001C090E0892F0895D2
:104100000F931F93CF93DF938C01EB01209709F45A
:1041100042C01882892B19F189E10E94CAD0F801A6
:1041200080818130C0F0833018F08530D0F013C02A
:10413000611106C02097B9F087E4888380E02EC023
:104140006150623090F0209791F087E4888380E09E
:1041500025C0209771F082E4888380E01FC080E052
:104160001DC081E01BC080E019C081E017C080E065
:1041700015C080E013C081E011C080E00FC089E16C
:104180000E94CAD0F8018081813018F3833080F218
:10419000853088F3DECF892B91F7EFCFDF91CF9178
:1041A0001F910F910895009739F0FC018081815093
:1041B000843020F481E0089580E0089580E008953F
:1041C000009751F0FC018081813040F0843010F084
:1041D000853021F481E0089580E0089580E008951D
:1041E000CF92DF92EF92FF92CF93DF93009709F483
:1041F0005FC0EC0183E00E94CAD06B017C01AB017F
:10420000BC0155276627772783E00E941ED68823A6
:1042100009F44BC08C2DFE01E95CFD4FC08281305A
:1042200021F1823009F044C088E00E94CAD0FE012A
:10423000E75CFD4F6083AB01BC01552766277727FC
:1042400088E00E941ED6811105C081E0FE01E75C76
:10425000FD4F8083FE01E85CFD4F1082C65CDD4FA0
:10426000188219821A821B8223C087E00E94CAD05A
:10427000F62E84E00E94CAD0862F6F2D0F947416FC
:1042800085E00E94CAD00F942517FE01E25CFD4F25
:1042900060837183828393830F943D16C65CDD4FE8
:1042A000188219821A821B8203C0C95CDD4F1882F2
:1042B000DF91CF91FF90EF90DF90CF90089500971E
:1042C00061F1FC01E85CFD4F2081319630813217AD
:1042D00010F021111BC0FC01E85CFD4F3150308310
:1042E00032964081518162817381403821E55207C5
:1042F00021E06207710598F44F5F5F4F6F4F7F4F6A
:10430000408351836283738381E00895FC01E85CFC
:10431000FD4F2150208380E0089580E0089580E0E3
:1043200008950F931F93CF93DF93009741F1EC0112
:104330000F945416FE01E25CFD4F00811181228131
:1043400033816017710782079307D8F00F943D16E9
:10435000FE01E65CFD4F80819181A281B3818038AE
:1043600021E5920721E0A207B10568F40196A11D9D
:10437000B11D80839183A283B38381E005C080E077
:1043800003C080E001C080E0DF91CF911F910F91C9
:104390000895CF93DF93009709F43DC0FC01EA5CD8
:1043A000FD4F20812223B9F1EC018BDE813021F415
:1043B000CA5CDD4F18822FC089E10E94CAD061110A
:1043C0001AC00F94C529813031F1823089F4D2DDD1
:1043D000882309F10F947F29CA5CDD4F18828FEE84
:1043E00095E40E9461DE8EEB98E40E9488DE13C0A3
:1043F0000F94B32910C0BEDD882369F00F947F2984
:10440000CA5CDD4F18828FEE95E40E9461DE8EEB70
:1044100098E40E9488DEDF91CF910895FF920F9378
:104420001F93CF93DF936115710509F47CC041158B
:10443000510509F478C08A01EB01F82E82E10F944E
:10444000801721E0672B682B692B09F420E08F2D62
:1044500090E0FC013197E231F10508F05BC088275C
:10446000EB5DFE4F8F4F0D942B651882E22FF0E02D
:10447000E153FF4D80818560F801808354C083E063
:104480008883E22FF0E0E153FF4D8081F8018083C3
:104490004AC01882E22FF0E0E153FF4D8081816035
:1044A000F801808340C083E08883E22FF0E0E1538D
:1044B000FF4D8081F801808336C01882E22FF0E042
:1044C000E153FF4D80818160F80180832CC083E03F
:1044D0008883E22FF0E0E153FF4D8081F801808373
:1044E00022C0188285E0F80180831DC0188281E017
:1044F000F801808318C01882E22FF0E0E153FF4DED
:1045000080818160F80180830EC0188281E0F8010B
:10451000808309C01882E22FF0E0E153FF4D8081D3
:104520008560F8018083DF91CF911F910F91FF90FB
:1045300008958F929F92AF92BF92CF92DF92EF92A7
:10454000FF920F931F93CF93DF93892B09F486C0BB
:1045500089E00E94CAD09B01AC01A8EEB3E00F94A1
:1045600048656B017C010F94D629C616D706E8066C
:10457000F90609F475C0C701B60128EE33E040E042
:1045800050E00F94ED64F22ED22F2E3108F06AC065
:10459000213009F469C00F94D62928EE33E040E0B9
:1045A00050E00F94ED64822FF21638F46F2D0F94C3
:1045B000BA64C92F992309F45CC00F946E29E82EC0
:1045C0006D2F0F94BA64D92F892F90E08E0D911D15
:1045D000CA970CF04BC08D2E912CA12CB12C0F94AE
:1045E000ED29162F072FD82EC92EA8EEB3E0A5016E
:1045F00094010F9448654F2D0F941B2AC091493F99
:10460000C11136C00F94ED299F938F937F936F93C1
:10461000CF92DF920F931F931F92DF931F92EF921F
:1046200085E391E29F938F9300ED14E41F930F9322
:104630000F945867F80101900020E9F73197AF0116
:10464000405D544421E0B8018AEA99E30F94F031C7
:104650008DB79EB740968DBF9EBF0BC0C0E009C00E
:10466000C0E007C0C1E005C0C0E003C0C1E001C0B8
:10467000C0E08C2FDF91CF911F910F91FF90EF90B1
:10468000DF90CF90BF90AF909F908F900895EF9262
:10469000FF920F931F93CF93DF932091493F2223E3
:1046A00039F00F2EFAEAEF2EF9E3FF2EF02D06C0B7
:1046B0000F2EF1EBEF2EFAE3FF2EF02D0097D1F144
:1046C000EC018BE7888388E689838CE28A8392E613
:1046D0009B838C837F936F9380E791E29F938F936B
:1046E000CE0105969F938F930F945867FE0101901A
:1046F0000020E9F73197EC1BFD0B8F01112721E01A
:10470000A801BE01C7010F94F0310E94D9C80F90D3
:104710000F900F900F900F900F90873059F4809169
:10472000493F811107C021E0A801BE018AEA99E34F
:104730000F94F031DF91CF911F910F91FF90EF9087
:1047400008958F929F92AF92BF92CF92DF92EF9295
:10475000FF920F931F93CF93DF93009709F470C0DC
:104760002091493F222339F00F2EFAEAEF2EF9E388
:10477000FF2EF02D06C00F2EF1EBEF2EFAE3FF2EE9
:10478000F02DEC018BE7888388E689838CE28A83AD
:1047900093E79B838C8307EF1CE3F801848C0E94D2
:1047A00028A7982EA090483FB090453FF801C280BE
:1047B000D0800F9499111F928F921F929F921F92F7
:1047C000AF921F92BF921F92CF921F92DF921F92C1
:1047D0008F93F80185811F928F9384811F928F930D
:1047E00083811F928F9385E591E29F938F93CE01F2
:1047F00005969F938F930F945867FE0101900020B8
:10480000E9F73197EC1BFD0B8F01112721E0A8017F
:10481000BE01C7010F94F0318DB79EB748968DBF8A
:104820009EBF8091493F81110BC0A80142505109A0
:10483000BE016F5F7F4F21E08AEA99E30F94F03168
:10484000DF91CF911F910F91FF90EF90DF90CF906C
:10485000BF90AF909F908F900895DF92EF92FF925C
:104860000F931F93CF93DF9300D01F92CDB7DEB786
:104870008C010F946425882349F00F9475250E94BC
:10488000131089E493E45DDF80E066C0CE010196F9
:104890000E941C10882309F45FC0F090A806E090E5
:1048A0006806D0902806BE016D5F7F4FCE0101964D
:1048B0000E943210882309F44CC00E94E5C8882366
:1048C000C9F18091493F811135C0D0FADD24D0F87B
:1048D0001F92DF92E4FAEE24E0F81F92EF92F6FACC
:1048E000FF24F0F81F92FF928A818F9389818F9322
:1048F0008C818F938B818F9384E791E29F938F9329
:104900000F2EF0EDEF2EF4E4FF2EF02DFF92EF923C
:104910000F945867F70101900020E9F73197AF0134
:10492000405D544421E0B7018AEA99E30F94F031E5
:10493000CDBFDEBF6B817C8189E493E4A8DE0115E5
:10494000110549F08B819C81F8018083918381E07E
:1049500003C081E001C081E02496CDBFDEBFDF91BE
:10496000CF911F910F91FF90EF90DF9008958823D2
:1049700021F081E08093483F08951092483F0895C8
:104980000F931F93CF93DF936115710571F000971B
:1049900061F0EB018C010F948625882331F00F9490
:1049A0009725BE01C8010E942A91DF91CF911F91E6
:1049B0000F910895CF93DF93009751F0EC010F947E
:1049C000D225882329F0CE010E946C930F94E32511
:1049D000DF91CF910895009791F0FC01EC5BFD4FC2
:1049E0002FEF3FE720833183329620E030E82083A9
:1049F000318332961082118232961082118208958C
:104A00000F93CF93DF930097A1F0662371F0EA0133
:104A1000FC01E45BFD4F81E08083C9010F94E42B2E
:104A2000602FCE010E94CDA804C0FC01E45BFD4FC5
:104A30001082DF91CF910F910895EF92FF920F9323
:104A40001F93CF93DF931F921F92CDB7DEB70097CE
:104A500009F498C06115710509F494C0FC0122A9FC
:104A6000211104C023A9222309F48CC08B017C01ED
:104A7000FC0112AA13AA0E946F110E94FA110E944F
:104A8000F313F70144A955A9B7016A5C7F4F9E0152
:104A90002F5F3F4FC8010F944F5BC8010F94FD5C1F
:104AA000F701E75AFD4FD701AD5ABD4F8C91808376
:104AB000319611968C9180830F94ED299F938F935B
:104AC0007F936F9383E991E29F938F9300ED14E4BA
:104AD0001F930F930F945867F80101900020E9F796
:104AE0003197AF01405D544421E0B8018AEA99E36F
:104AF0000F94F031CDBFDEBFF70124A935A989811C
:104B00009A812817390719F1C70106969F938F9349
:104B10008FE991E29F938F931F930F930F945867A0
:104B2000F80101900020E9F73197AF01405D54444E
:104B300021E0B8018AEA99E30F94F0310E947AA942
:104B40000F900F900F900F900F900F9002C00E9447
:104B50000AA9E5E8F3E4808190E0DC01AB57BC4BA7
:104B600025853685880F991FFC01EB57FC4B418149
:104B700052811F960C9161E0C70142DF0E94D095DF
:104B80000F944A2C0F900F90DF91CF911F910F91AE
:104B9000FF90EF9008950F931F93CF93DF930097AB
:104BA00009F448C06115710509F444C08B01EC019A
:104BB000FC01E45BFD4F80818823C1F1DB018C9116
:104BC000882341F10F94002C8823A1F1F801608122
:104BD00061506083611108C00E943FA90E942CA906
:104BE000C45BDD4F188226C070E0F801E60FF71FA6
:104BF000D8011D962D913C911E97660F771FA60F29
:104C0000B71F11964D915C911297078561E0CE0117
:104C1000F7DE10C00F94002C882361F00E943FA99A
:104C20000E942CA9C45BDD4F188204C00E943FA9DA
:104C30000E942CA9DF91CF911F910F9108958F921F
:104C40009F92BF92CF92DF92FF920F931F93CF93C9
:104C5000DF93009709F4DAC06115710509F4D6C035
:104C60002091493F222309F4C0C0CAEAD9E3BFC05A
:104C70008B014C010E94D211B82E0E945212D82EE4
:104C80000E942D11C82E8D2D90E08B0D911D8C0D45
:104C9000911D892B71F4F401E35BFD4F808181301C
:104CA00009F4B4C081E0808380E090E00F94172C79
:104CB000ADC0F401E35BFD4F8081823009F43EC05A
:104CC000BB2051F00E94CF11811108C061E0CE01DC
:104CD0000E94A89501E003C000E001C000E0CC20E4
:104CE00009F48AC00E942A11811186C063E0CE01B6
:104CF0000E94A89501E080C0DD2081F0812F0E94F4
:104D00003214882359F0812F0E944214811106C069
:104D100064E0610FCE010E94A89501E01F5F14308E
:104D200059F7002309F472C0E401C35BDD4F82E050
:104D3000888384EF91E00F94172C68C00F94332C74
:104D4000882309F463C0BB2009F45DC00E94CF1121
:104D5000811159C00E9491A9CC2009F44FC0FF24B1
:104D6000F39401C0F12C0E942A11811149C00E94C4
:104D700091A916C0D0E0C0E0DD2069F08D2F0E941F
:104D80003214882341F08D2F0E944214811103C0F8
:104D90000E948FA9C1E0DF5FD43071F7CC23E1F02E
:104DA00084EF91E00F94172CD8018C9190E0F801DA
:104DB000E80FF91F1D962D913C911E97880F991FA2
:104DC000A80FB91F11964D915C911297078561E06C
:104DD00087EF9CE315DE1AC0F401E35BFD4F808191
:104DE0008230A1F481E0808311C0C1EBDAE3FC01E1
:104DF0002081243059F43CCF10E07ECFFF24F3947F
:104E0000F110CECFB7CFC110ADCFB4CFDF91CF91DE
:104E10001F910F91FF90DF90CF90BF909F908F9048
:104E20000895009721F0FC01E35BFD4F6083089536
:104E3000CF93DF930097C1F0EC01198218820E9492
:104E4000E51C813031F482E0888389E1898391E037
:104E500006C0CE010E94F6FC91E0811190E081E055
:104E6000992319F080E001C080E0DF91CF9108958F
:104E7000CF93892B09F44CC082E00E94CAD0862FC0
:104E800090E0FC013297E031F10508F043C088273B
:104E9000E95CFE4F8F4F0D942B6540E050E0BA0166
:104EA00080E00E9455D837C040E050E0BA0180E071
:104EB0000E9455D8C82F40E050E0BA0181E00E941E
:104EC00055D8C80F81E0C23031F180E024C040E005
:104ED00050E0BA0180E00E9455D8C82F40E050E071
:104EE000BA0181E00E9455D8C80F40E050E0BA01F5
:104EF00082E00E9455D8C80F40E050E0BA0183E03C
:104F00000E9455D8C80F81E0C43029F080E003C06A
:104F100080E001C080E0CF910895CF92DF92EF92C0
:104F2000FF92843098F4E82FF0E0EE0FFF1FEE0FB1
:104F3000FF1FE854F44CC080D180E280F3800E94CF
:104F400025D86C197D098E099F0903C060E070E0C7
:104F5000CB01FF90EF90DF90CF900895CF93892BF6
:104F600009F453C082E00E94CAD0862F90E0FC0171
:104F70003297E031F10508F04AC08827E95BFE4F1F
:104F80008F4F0D942B6580E0C8DFAB01BC0180E042
:104F90000E9455D83DC080E0C0DFAB01BC0180E07D
:104FA0000E9455D8C82F81E0B8DFAB01BC0181E079
:104FB0000E9455D8C80F81E0C23051F180E028C06E
:104FC00080E0ABDFAB01BC0180E00E9455D8C82F68
:104FD00081E0A3DFAB01BC0181E00E9455D8C80F7E
:104FE00082E09BDFAB01BC0182E00E9455D8C80F74
:104FF00083E093DFAB01BC0183E00E9455D8C80F6A
:1050000081E0C43029F080E003C080E001C080E08E
:10501000CF91089590E0FC013397EE30F10508F050
:10502000A7C08827E95AFE4F8F4F0D942B65E8E201
:10503000F4E5868D978DA0A1B1A1428D538D648D2D
:10504000758D841B950BA60BB70B86399105A105B1
:10505000B10508F48FC046A157A160A571A582A132
:1050600093A1A4A1B5A1481B590B6A0B7B0B81E04E
:10507000463951056105710508F483C080E0089543
:10508000E8E2F4E582A193A1A4A1B5A1468D578DD4
:1050900060A171A1841B950BA60BB70B86399105F6
:1050A000A105B10508F468C046A557A560A971A976
:1050B00082A593A5A4A5B5A5481B590B6A0B7B0B2C
:1050C00081E0463951056105710508F45AC080E058
:1050D0000895E8E2F4E582A193A1A4A1B5A1468DCB
:1050E000578D60A171A1841B950BA60BB70B863958
:1050F0009105A105B10508F441C042A953A964A9CD
:1051000075A986A597A5A0A9B1A9481B590B6A0B3B
:105110007B0B81E0463951056105710590F180E016
:105120000895E8E2F4E5868D978DA0A1B1A1428DA6
:10513000538D648D758D841B950BA60BB70B86392B
:105140009105A105B105E0F042A553A564A575A59B
:1051500086A197A1A0A5B1A5481B590B6A0B7B0B93
:1051600081E0463951056105710558F080E00895E8
:1051700080E0089581E0089581E0089581E0089538
:1051800081E00895CF9382E10E94CAD0C1E0672BED
:10519000682B692B09F4C0E082E00E94CAD088E045
:1051A000E2E6F4E5DF01982F1D929A95E9F7EAE629
:1051B000F4E5DF011D928A95E9F7862F90E0FC0166
:1051C0003197E231F10508F0EFC08827EB59FE4F27
:1051D0008F4F0D942B65EC2FF0E0E153FF4D808154
:1051E0008560E8E2F4E582AF83AFE8C0EC2FF0E041
:1051F000E153FF4D8081E8E2F4E582AF83AF83E0C5
:1052000080936A5480936B54D9C0862F03DFEC2FB0
:10521000F0E0E153FF4D908121E0811101C020E0D9
:10522000822F892BE8E2F4E582AF84AF83E080939C
:105230006A5480936C54892F816083AF85AFBEC060
:10524000EC2FF0E0E153FF4D8081E8E2F4E582AF1E
:1052500084AF93E090936A5490936C5483AF85AF7E
:1052600082E080936B5480936D54A8C0862FD2DE69
:10527000EC2FF0E0E153FF4D208191E0811101C05E
:1052800090E0892F822BE8E2F4E582AF85AF93E0CE
:1052900090936A5490936D5483AF86AF82E080936D
:1052A0006B5480936E54822F816084AF87AF86C029
:1052B000EC2FF0E0E153FF4D8081E8E2F4E582AFAE
:1052C00086AF93E090936A5490936E5483AF87AF08
:1052D00092E090936B5490936F5484AF8093685492
:1052E00094E090936C549093705485AF809369547C
:1052F00085E080936D548093715460C0862F8ADE60
:1053000091E0811101C090E0892F8F70E8E2F4E50F
:1053100082AF86AF93E090936A5490936E5483AFBC
:1053200087AF82E080936B5480936F5481E084AFA9
:105330008093685495AF9093695440C0E8E2F4E5D7
:1053400085E082AF84AF87E083AF85AF37C0862F1B
:1053500061DE91E0811101C090E0EC2FF0E0E153BB
:10536000FF4D8081892BE8E2F4E582AF85AF83E0D1
:1053700080936A5480936D5491E093AF96AF84AF5D
:1053800087AF1CC0EC2FF0E0E153FF4D80818160BE
:10539000E8E2F4E582AF84AF83AF85AF81E080932C
:1053A0006B5480936D540AC0EC2FF0E0E153FF4D35
:1053B00080818560E8E2F4E582AF83AF809162543A
:1053C00084700F949D1581E0CF9108951F93CF9322
:1053D000DF930097E9F1EC011AAA1BAA0E9421179A
:1053E00087E00E94CAD0162F84E00E94CAD0862F80
:1053F000612F0F94741689E10E94CAD06130710543
:105400008105910521F481E00F94042A03C080E016
:105410000F94042A0E94D11C813031F4CE010E94E5
:105420008A1C0E94222004C0CE010E94201CAADEF9
:105430000F94952C0F948015CE010E94F0200F94AC
:10544000202B0E945E100E94AF110E942E12198222
:10545000DF91CF911F910895CF93DF93009791F043
:10546000FC012081243071F4EC010E94D21FCE0196
:10547000ADDF0F9491291092443F63E0CE010E946A
:10548000AC141982DF91CF910895882321F081E037
:105490008093493F08951092493F08958091493F74
:1054A0000895AF92BF92CF92DF92EF92FF920F9347
:1054B0001F93CF93DF93DC01009709F45AC0411585
:1054C000510509F458C02115310509F456C0FA01F7
:1054D000C081D0E0F901008110E06115710561F033
:1054E000FC017C01E60EF71E9191C90FD11D0C0F36
:1054F0001D1FEE16FF06C1F7F9017B016D01DA01F0
:10550000CC930083F601E60FF71F8CE280838BE1DA
:1055100081835B01A2E0AA0EB11CAC0CBD1C8C2FD8
:1055200082958F700F940836F50180835701F3E060
:10553000AF0EB11CAC0CBD1C8C2F8F700F940836B5
:10554000D5018C93E7012496CC0DDD1D802F82952B
:105550008F700F9408368883D7011596E601CA0F1D
:10556000DB1F802F8F700F9408368883C701069643
:1055700005C0CB0103C0CB0101C0CB01DF91CF91AE
:105580001F910F91FF90EF90DF90CF90BF90AF9061
:1055900008953F924F925F926F927F928F929F9267
:1055A000AF92BF92CF92DF92EF92FF920F931F9331
:1055B000CF93DF93CDB7DEB76397CDBFDEBF7C015E
:1055C0006B013A01290189E10E94CAD0B62E82E01E
:1055D0000E94CAD0162FE114F10409F446C1C11487
:1055E000D10409F444C16B3008F449C16114710459
:1055F00009F43FC14114510409F43DC1FE01329642
:10560000CE014296C192D1922BE0C20ED11CE81776
:10561000F907C1F78DE0D701D6968C93D69782E033
:1056200090E0D4968D939C93D5978AE0D7968C93EF
:10563000F701F896EA8BFB8B41E0BE016F5F7F4F6D
:10564000CF010E94DE172981D701D4968D919C91BC
:10565000D597820F911D9C012F5F3F4FD4962D93BC
:105660003C93D597F701E80FF91F2CE226ABB1E088
:10567000BB1590F5B12C0F2EFCE2AF2EF02D61C0C2
:10568000EB2DF0E0EE0FFF1F81E090E08C0F9D1FEF
:10569000E80FF91FC180D280D701D4968D919C91DB
:1056A000D597C696F601418550E0B6018E0D9F1D37
:1056B0000F942A67D60119962C91F70184A995A910
:1056C000820F911D9C012F5F3F4F24AB35ABE80F3C
:1056D000F91FA6AAB39405C0B12C0F2EFCE2AF2E81
:1056E000F02D0F94922CB81658F230C0EB2DF0E04C
:1056F000EE0FFF1F81E090E08C0F9D1FE80FF91F58
:10570000C180D280D701D4968D919C91D597C696B1
:10571000F601418550E0B6018E0D9F1D0F942A675A
:10572000D60119962C91F70184A995A9820F911D94
:105730009C012F5F3F4F24AB35ABE80FF91FA6AAA2
:10574000B3940F94922C8695B81680F21B3008F40F
:1057500066C01C3028F01E3028F01051133010F0B5
:1057600010E001C011E00F2EF4EB8F2EF1E29F2E1E
:10577000F02D5701F6E3AF0EB11C0F2EFCE23F2EC9
:10578000F02DC12ED12CC601880F991FC80ED91E2D
:10579000CC0CDD1CCC0CDD1CC60CD71CD6011A961B
:1057A0008C911F928F939F928F92F70184A995A954
:1057B000C6968E0D9F1D9F938F930F945867F5018A
:1057C00001900020E9F73197EA19FB09D701D49637
:1057D000ED93FC93D597CF01C696F601418550E035
:1057E000B6018E0D9F1D0F942A67D60119962C9134
:1057F000F70184A995A9820F911D9C012F5F3F4F4E
:1058000024AB35ABE80FF91F36AA1F5F0F900F903E
:105810000F900F900F900F90123008F4B2CF01301C
:10582000D9F4D701D4968D919C91D597C6968201D3
:1058300001501F4FF801408150E0B2018E0D9F1DB5
:105840000F942A67D8012C91F70184A995A9820F9A
:10585000911D84AB95AB18C0D701D496ED91FC9106
:10586000D597EE0DFF1D16AA0FC080E02EC080E078
:105870002CC080E02AC080E028C080E026C041140F
:10588000510409F0BBCEF9CFA7014D5A5D4FF70186
:10589000E75AFD4F8081FA01808397012C5A3D4FD2
:1058A00037968081D9018C93F70164A975A962505C
:1058B00071098A899B89F5DD0296D701D4968D936B
:1058C0009C93D59781E0D2968C936396CDBFDEBF33
:1058D000DF91CF911F910F91FF90EF90DF90CF90CC
:1058E000BF90AF909F908F907F906F905F904F9000
:1058F0003F9008952F923F924F925F926F927F92C6
:105900008F929F92AF92BF92CF92DF92EF92FF92CF
:105910000F93CF93DF93CDB7DEB76097CDBFDEBFD8
:10592000009709F46EC06115710509F46AC09B0106
:10593000FE013196DE01519621933193255F3F4F51
:10594000EA17FB07C9F76A017B011C01B12C12C0E1
:10595000EB2DF0E0EE0FFF1F81E090E08C0F9D1F1C
:10596000E80FF91F808191810E943C17882309F478
:1059700048C0B3940F94922CB81650F30F94ED29AD
:105980004B015C010F94D6292B013C018FEE95E46D
:105990000E9467DE082F81110BC09EE1890E911CC9
:1059A000A11CB11C84149504A604B70450F115C0C1
:1059B00040E050E069E473E480E30E94F91C2FEEBC
:1059C00035E4A601B701C101E4DD41EF56E469E425
:1059D00073E482E30E94F91C0EC000E02FEE35E470
:1059E000A601B701C101D5DD40E050E069E473E4F0
:1059F00082E30E94F91C8FEE95E40E9461DE0E9412
:105A000021176096CDBFDEBFDF91CF910F91FF9040
:105A1000EF90DF90CF90BF90AF909F908F907F904E
:105A20006F905F904F903F902F900895009789F06E
:105A30006115710571F04115510559F021153105B8
:105A400041F0FC011082FB011082FA011082F90181
:105A5000108208952F923F924F925F926F927F92A1
:105A60008F929F92AF92BF92CF92DF92EF92FF926E
:105A70000F931F93CF93DF93CDB7DEB72597CDBF9D
:105A8000DEBF009709F461C04115510509F45FC0FC
:105A90002115310509F45DC0613BE4E07E0708F49F
:105AA0005AC02B01E0EB4E1AE4E05E0A612C712C27
:105AB000E2E04E165104610471040CF454C02C83CE
:105AC0003D831A018C01C12CD12C7601C3944B016A
:105AD000A12CB12CB501A4014C195D096E097F09F7
:105AE000C8010F944F5D9E012F5F3F4F41E050E092
:105AF000BE016D5F7F4FC8010F94035A81112DC005
:105B00008B818B3191F18FEFC81AD80AE80AF80A15
:105B1000C414D504E604F704ECF225C089819A8107
:105B20000497E8F0B10180ED94E40F94FA39982FCE
:105B3000882341F16C817D8182ED94E40F94FA39E0
:105B400091E081111FC090E01DC090E01BC090E06B
:105B500019C090E017C090E015C090E013C090E02D
:105B600011C090E00FC090E00DC09E012F5F3F4F2D
:105B700044E050E060ED74E4C8010F94035A8823B8
:105B800069F2EFCF892F2596CDBFDEBFDF91CF9190
:105B90001F910F91FF90EF90DF90CF90BF90AF904B
:105BA0009F908F907F906F905F904F903F902F903D
:105BB00008950097A9F061157105B1F0FC019C01F1
:105BC000260F371F60E070E0CB0141914D3021F48A
:105BD0006F5F7F4F8F4F9F4F2E173F07B1F708958D
:105BE00060E070E0CB01089560E070E0CB010895C3
:105BF0002F923F924F925F926F927F928F929F92DD
:105C0000AF92BF92CF92DF92EF92FF920F931F93CA
:105C1000CF93DF9300D01F92CDB7DEB7009709F482
:105C200055C00115110509F453C0613B7440C0F41F
:105C3000F801108211821282138280E04CC0098127
:105C40001A81B801C101B5DF460E571E681E791EC4
:105C50000815190500F1C00ED11EE11CF11C0BC086
:105C60000B831C8349011A015C01C12CD12C7601E4
:105C7000412C512C3201B701A601C5010F944F5D93
:105C80009E012F5F3F4FA401B101C5010F94035A3C
:105C90008823A9F21FC0F6E24F1651046104710473
:105CA00040F4EB81FC81108211821282138281E028
:105CB00012C0F5E24F1A510861087108EB81FC81AE
:105CC000408251826282738281E005C080E003C01D
:105CD00080E001C080E02496CDBFDEBFDF91CF9190
:105CE0001F910F91FF90EF90DF90CF90BF90AF90FA
:105CF0009F908F907F906F905F904F903F902F90EC
:105D00000895009741F0FC01EB5AFD4F60817181CD
:105D100082819381089560E070E0CB01089500973F
:105D200039F0FC01EB5AFD4F10821182128213826E
:105D30000895CF93DF93009781F12091493F21117E
:105D40002CC0EC010F946C26882339F1CE010E94FF
:105D50000C9A0F9445260F9482111F928F9388EB13
:105D600091E29F938F93C0EDD4E4DF93CF930F9490
:105D7000586709900020E9F72197AE01405D54442F
:105D800020E060ED74E48AEA99E30F94F0310F901B
:105D90000F900F900F900F900F90DF91CF9108957B
:105DA0002115310551F0505861097109F9014083FD
:105DB00051836283738381E0089580E008950097A2
:105DC00019F0FC01848D089580E008954F925F9250
:105DD0006F927F928F929F92AF92BF92EF92FF92BB
:105DE0000F931F93CF93DF931F92CDB7DEB7E114CC
:105DF000F10409F465C0480159012A013B01182F3B
:105E0000C7010E941517143031F484E10E94A6D016
:105E10009B01AC0105C085E10E94A6D09B01AC01AD
:105E20002115310541055105F9F084189508A6089A
:105E3000B708880C991CAA1CBB1CD501C401880F8B
:105E4000991FAA1FBB1F880F991FAA1FBB1FBC0148
:105E5000CD01680D791D8A1D9B1D0F940F65822E43
:105E6000932EA42EB52E0EC088248A940F2EF0EE09
:105E70009F2EF02D0F2EF5EFAF2EF02D0F2EF5E00B
:105E8000BF2EF02D082D192D2A2D3B2D4BE0BE01E4
:105E90006F5F7F4FC7010F947439F70101900020A5
:105EA000E9F73197EE19FF09D7011996EC93199785
:105EB00081E01B968C93682D792D8A2D9B2D04C033
:105EC00060E070E080E090E00F90DF91CF911F9153
:105ED0000F91FF90EF90BF90AF909F908F907F9029
:105EE0006F905F904F9008952F923F924F925F92E4
:105EF0006F927F928F929F92AF92BF92CF92DF92DA
:105F0000EF92FF920F931F93CF93DF93CDB7DEB73E
:105F10002A97CDBFDEBFC5016115710509F402C125
:105F20004115510509F400C1E114F10409F4FEC062
:105F3000802E912EA22EB32E25EB82169104A10461
:105F4000B10438F00F2EF4EB8F2E912CA12CB12C34
:105F5000F02D8B839C83CD82DE82EF82F88649838D
:105F60005A838B01FB01E453FD4F80819181A28113
:105F7000B381892B8A2B8B2B81F53497808191817A
:105F8000A281B38180324EE49407A105B1052CF1C2
:105F9000349680839183A283B383BF93AF939F93FF
:105FA0008F9383ED91E29F938F9380ED94E49F9381
:105FB0008F930F945867E0EDF4E401900020E9F727
:105FC0003197AF01405D544420E060ED74E48AEA0B
:105FD00099E30F94F031CDBFDEBFD801CD90DD90B5
:105FE000ED90FC90B0E8DB1AE108F108F801C082FE
:105FF000D182E282F38281E08093D132F2E08F1687
:106000009104A104B10408F46FC0F80161ED72E3DA
:1060100021E0821A20EC920A880C991C880C991CA9
:106020001801280C391C4601570100E010E09801C6
:1060300069877A8744815581668177812A013B018E
:1060400080E8581A61087108448255826682778216
:106050004191519161917191441A550A660A770AEA
:10606000141415041604170434F481E0A985BA85C4
:1060700011968C9304C0A985BA8511961C92A985A6
:10608000BA8511965C901197CD01019689879A8700
:106090009C91591691F0D801AA0FBB1FAA0FBB1FE4
:1060A00089819A81A80FB91F4D935D936D937C935D
:1060B00013970F5F1F4F2F4F3F4F408151816281D8
:1060C0007381C416D506E606F70614F46A017B014F
:1060D000481559056A057B0514F44A015B01E21570
:1060E000F30509F0A7CF05C04601570100E010E015
:1060F0009801AF81B8850D931D932D933C93139711
:10610000ED81FE81309721F080829182A282B3825C
:10611000EB81FC81309761F0C082D182E282F38210
:1061200081E007C080E005C080E003C080E001C0DE
:1061300081E02A96CDBFDEBFDF91CF911F910F91F5
:10614000FF90EF90DF90CF90BF90AF909F908F9097
:106150007F906F905F904F903F902F9008958F9217
:106160009F92AF92BF92CF92DF92EF92FF920F93E6
:106170001F93FC01892BA1F16115710599F1008133
:1061800011812281338184819581A681B78108178D
:1061900019072A073B0744F5C084D184E284F384BD
:1061A000C816D906EA06FB060CF584849584A684F5
:1061B000B784C814D904EA04FB04D4F488159905FB
:1061C000AA05BB05BCF40C151D052E053F0524F4DE
:1061D00081E0FB0180830FC0FB01108281E00BC0D6
:1061E00080E009C080E007C080E005C080E003C017
:1061F00080E001C080E01F910F91FF90EF90DF9051
:10620000CF90BF90AF909F908F9008953F924F9204
:106210005F926F927F928F929F92AF92BF92CF9236
:10622000DF92EF92FF920F931F93CF93DF9300972C
:1062300009F448C02115310509F446C04430510520
:106240006105710508F442C06A017B01E4E0CE1AE1
:10625000D108E108F108E1F159018C01912C312CB0
:10626000812C412C512C3201E501C90DD11DBE01FB
:10627000C201880F991F880F991F800F911F6FDF30
:10628000882379F08881882311F0839401C03394A6
:1062900083E0480E511C611C711C9394E2E0E915E7
:1062A00050F08FEF481A580A680A780A4C145D04B7
:1062B0006E047F04C8F2882069F081E0332059F031
:1062C00080E009C080E007C080E005C080E003C036
:1062D00081E001C081E0DF91CF911F910F91FF908C
:1062E000EF90DF90CF90BF90AF909F908F907F9076
:1062F0006F905F904F903F9008952F923F924F92F2
:106300005F926F927F928F929F92AF92BF92CF9245
:10631000DF92EF92FF920F931F93CF93DF93CDB74E
:10632000DEB76B97CDBFDEBF782ED92E662E798B68
:1063300019821A821B821C821D821E821F8218866D
:1063400019861A861B861C861D861E861F86188A3D
:1063500082E00E94CAD06B3008F4BBC00F94CB2DF2
:10636000882309F4CEC00F94BA2D8091133D82305A
:1063700009F0B1C083EB90E40F94FD5CACC08F8A50
:10638000988E530162010F2EFAEFEF2EFFE2FF2EDF
:10639000F02D04EB10E020E030E041E050E3B401E8
:1063A000832DA2DD882331F14091FA2F5091FB2FEC
:1063B0006091FC2F7091FD2F2EEF3FE281E090E382
:1063C00025DF882361F08091FE2F90E0A0E0B0E00F
:1063D000EF89F88D80839183A283B38314C08EEFFD
:1063E00090E0A0E0B0E0EF89F88D80839183A283F4
:1063F000B38309C08FEF90E0A0E0B0E0F4018083A8
:106400009183A283B3833394F0E38F1AFDEF9F0A45
:1064100084E0480E511C94E0690E711CA6E03A120B
:10642000AECF298C3A8C6B8C862C99886894552435
:1064300052F80F2EF5E44F2EF02D0F2EF2E5DF2E41
:10644000F02D0F2EFCE4CF2EF02DAB88BC886D888C
:106450007E88898A9A8AF301019111912191319163
:106460003F01D5014D915D916D917D915D0174016B
:10647000852DACDC65317105810591051CF4F401B5
:1064800042861AC0F10180819181A281B381009777
:10649000A105B10529F4A989BA891A96CC920CC034
:1064A0000197A105B10521F4E989FA89D28604C0D2
:1064B000A989BA891A964C925394BCE08B0E911C10
:1064C000E0E32E1AEDEF3E0AF6E05F12C2CF81E064
:1064D00018C080E016C0272C3D2CCE0101968B8B76
:1064E0009C8BDE011996AD8BBE8B2C01872C9D2CCD
:1064F0006894772472F8298E3A8E372C6B8E3D0182
:106500003ECF6B96CDBFDEBFDF91CF911F910F9134
:10651000FF90EF90DF90CF90BF90AF909F908F90C3
:106520007F906F905F904F903F902F900895CF9203
:10653000DF92EF92FF921F93CF93DF93009709F4BE
:1065400059C1EC018881843089F128F4813069F0E7
:106550008230E9F04FC1893009F40EC18A3009F464
:1065600022C1883009F046C11EC08B81813009F0FC
:1065700041C18C81813009F03DC10F94B329CE0116
:106580000E94E62962E0CE010E94AC1433C18091E2
:106590004A49813029F463E0CE010E94AC142AC13B
:1065A0000E94CB1B27C10E946B5124C1CE010E94C7
:1065B000C921898181111EC182E00E94CAD06B303D
:1065C00040F46BE479E38FEC9CE30E940918182FE8
:1065D00010C00F94CB2D8823E1F06BE479E38FECAE
:1065E0009CE30E940918182F6FED7CE388E89EE475
:1065F00084DE113071F482E00E94CAD0162F8FEC35
:106600009CE30E947A10612F83E790E40E949C1221
:1066100007C08BE499E30E944717882309F4DCC084
:106620004FED5CE36BE479E3CE0164D9D5C00F9400
:106630006517882309F4DBC082E00E94CAD0162FB8
:106640000F94ED291B3050F40F94312B63EB70E461
:10665000CE010E941D250F945417C9C0C0907B54D1
:10666000D0907C54E0907D54F0907E5424E6C20E8D
:10667000D11CE11CF11CC616D706E806F90650F03D
:10668000C8A4D9A4EAA4FBA46C157D058E059F05BA
:1066900008F0ADC00F94312B63EB70E4CE010E9483
:1066A0001D250F945417A3C089818111A3C0CE0169
:1066B0000E949121882341F00F94312B63EB70E409
:1066C000CE010E941D2596C01AAA81E08BAB92C014
:1066D0008AA9882309F48EC0898181118BC0CE01DB
:1066E0000E945F21882341F00F94312B63EB70E40B
:1066F000CE010E941D257EC01AAA7CC082E00E94A5
:10670000CAD0162F0F94ED296B017C010F946517E9
:10671000882309F46FC01B3050F40F94312B63EBC6
:1067200070E4CE010E941D250F94541763C0809120
:106730007B5490917C54A0917D54B0917E548C599F
:106740009F4FAF4FBF4F8C159D05AE05BF0550F055
:1067500088A599A5AAA5BBA5C816D906EA06FB0671
:1067600008F048C00F94312B63EB70E4CE010E9417
:106770001D250F9454173EC0CE010E94C9216BE421
:1067800079E38FEC9CE30F94AB1B813031F08BE409
:1067900099E30F94001C882369F16BE479E3CE013F
:1067A0000F94291F27C0CE010E94C921CE010E944B
:1067B000E6B44AE953E46BE479E38FEC9CE30E948E
:1067C00096B3CE010E94F7AD8831A1F46AE973E473
:1067D000CE010E947AB40EC0FE01E95CFD4F8081BB
:1067E000813009F424CF823009F088CF71CF8AA993
:1067F00081115ACFDF91CF911F91FF90EF90DF90E1
:10680000CF900895CF930E94C4D8C82F88E10E94EA
:10681000CAD0C61741F061E080E00F94821361E0B6
:1068200081E00F948213CF910895CF930E94C4D832
:10683000C82F88E10E94CAD0C61749F061E080E005
:106840000F94821361E081E00F94821308C060E02E
:1068500080E00F94821360E081E00F948213CF9167
:106860000895CF93DF93EC018091493F882319F07D
:10687000EAEAF9E302C0E1EBFAE3209729F18BE7BA
:10688000888388E689839CE29A8382E68B839C8353
:106890008CE68D838DE78E831F8221E047E050E0F8
:1068A000BE01CF010F94F0310E94D9C8873061F446
:1068B0008091493F811108C021E047E050E0BE01CE
:1068C0008AEA99E30F94F031DF91CF910895809196
:1068D000143D0895CF92DF92FF920F931F93CF93B1
:1068E000DF931F921F92CDB7DEB79FEF980F9230C4
:1068F00008F045C09091143D992309F443C08130BC
:1069000019F00CE61FE302C001EB1AE3F82E81E652
:10691000898384E78A8321E042E050E0BE016F5F13
:106920007F4FC8010F94F0310F945B2A0F94722AA5
:10693000643F714081059105C8F3C8010E942BA7EF
:106940000F945B2A0F94722A643F71408105910570
:10695000C8F38F2D0E9416D96C018F2D0E9416D975
:10696000FC0101900020E9F73197AF01481B590B5A
:1069700041F0B601C8010E949BA791E003C090E0DE
:1069800001C090E0892F0F900F90DF91CF911F9160
:106990000F91FF90DF90CF900895009791F0FC0148
:1069A000E15AFD4F108275961082749780599D4F61
:1069B000DC0111921192119211921D92E817F907C0
:1069C000C1F708950F931F93CF93DF931F92CDB715
:1069D000DEB7009709F4CAC08C0181E0D8018C931E
:1069E00011961C92119712961C92129713961C9254
:1069F000139714961C92149715961C921597169639
:106A000082E1E0E2F4E201900D928A95E1F7C8019B
:106A100048960E94F1D5F801808D8783818D80870B
:106A2000828D8187838D8287CE0101960E9412D646
:106A300089818C3438F4D8015C961C925C975D9601
:106A40001C9211C08C3431F482E0F801848F81E013
:106A5000858F09C08D3439F482E0D8015C968C931F
:106A60005C975D961C9280E00E94A6D0673EB3E0E2
:106A70007B0781059105BCF49F938F937F936F9360
:106A80008EEE91E29F938F93C801C6969F938F934A
:106A90000F945867F80186A9808B87A9818B80ADF8
:106AA000828BCDBFDEBFD8015E961C925E975F964B
:106AB0001C925F97D2961C92D297D3961C92F801A3
:106AC000EA5CFD4F10823196108231961082319629
:106AD00081E0808331961082118212821382349673
:106AE00081E090E0A0E0B0E080839183A283B38353
:106AF000349610823196D8018C918083E751F24010
:106B000086E0DF011D928A95E9F7E85EFD4F10826D
:106B10001182329610821182329610821182329640
:106B20001082118232961082319610823296108233
:106B300031961082319610823196108231961082F1
:106B4000319610823196108211821282138234960D
:106B500010823196108231961082319610823196D1
:106B600088E690E180839183C80117DF0F90DF9161
:106B7000CF911F910F910895EF92FF920F931F9362
:106B8000CF93DF93009709F43FC0FC01DC01A15AC9
:106B9000BD4F1C9255961C92EC01C05ADD4F84E10A
:106BA00090E0A0E0B0E088839983AA83BB836096DD
:106BB0001882289788839983AA83BB83DF01AE5804
:106BC000BD4F1C92E0A4F1A402A513A5D801C701F2
:106BD0004496A11DB11D249788839983AA83BB8302
:106BE0002D961882259788839983AA83BB83ED58B5
:106BF000FD4F108222E830E040E050E062E870E0B3
:106C000080E090E00F94232EDF91CF911F910F91A0
:106C1000FF90EF900895EF92FF920F931F93CF9301
:106C2000DF93CDB7DEB72797CDBFDEBF7C01FB0179
:106C300084818D8385818E8386818F8380819181FC
:106C4000A281B38189839A83AB83BC83870180EA65
:106C5000E81688E0F80629F460E183E00F945B44CD
:106C600014C080EBE81688E0F80629F460E283E0BF
:106C70000F945B4413C080EAE81689E0F80629F413
:106C800060E184E00F945B4412C0003B89E0180788
:106C900029F460E284E00F945B4412C0003A8AE079
:106CA000180729F460E185E00F945B4410C0003BB5
:106CB0008AE0180729F460E285E00F945B4407C07E
:106CC000003A1B4021F460E186E00F945B44BE0172
:106CD0006F5F7F4FC7010E94C9712796CDBFDEBF8E
:106CE000DF91CF911F910F91FF90EF900895DC01FC
:106CF000892BE1F0E62FE695E695E69580E2E89FA0
:106D0000F0011124FA5F8085677021E030E002C055
:106D1000220F331F6A95E2F7282381E009F480E00F
:106D20008C9311968C93119712961C920895CF9381
:106D3000DF93009709F4A5C06D3209F0A4C030912B
:106D4000A80621E0432F407235FF20E0FC0120839C
:106D50003181231709F499C0EC01442309F46BC075
:106D6000311169C00F94F4250097F9F40E944E2A5E
:106D7000811119C086E0E4EFF1E2A0EDB4E40190E6
:106D80000D928A95E1F7E0EDF4E401900020E9F737
:106D90003197AF01405D544421E060ED74E48AEA2C
:106DA00099E30F94F0311A8268C0803D974008F54E
:106DB0000E944E2A811119C086E0EAEFF1E2A0EDAF
:106DC000B4E401900D928A95E1F7E0EDF4E40190CE
:106DD0000020E9F73197AF01405D544421E060EDB8
:106DE00074E48AEA99E30F94F0310F9408261A822A
:106DF00044C081E08A830F9408260E944E2A8111A4
:106E00003CC086E0E0E0F2E2A0EDB4E401900D9237
:106E10008A95E1F7E0EDF4E401900020E9F731977D
:106E2000AF01405D544421E060ED74E48AEA99E3E7
:106E30000F94F03122C01A8281E090E00F941B265B
:106E40000E944E2A811119C086E0E6E0F2E2A0ED30
:106E5000B4E401900D928A95E1F7E0EDF4E401903D
:106E60000020E9F73197AF01405D544421E060ED27
:106E700074E48AEA99E30F94F031888189838A81E6
:106E800005C080E003C080E001C080E0DF91CF91C9
:106E900008958EEB98E40C9434E608950E944E2AEF
:106EA000811117C062E575E48AEA99E30F949C3179
:106EB0008091D445813029F542E555E464E575E4D7
:106EC0008AEA99E30E9446CE82E595E40D948D31DD
:106ED000089562E575E48AEA99E30E947AA48091B4
:106EE000D445813071F427EF3CE342E555E464E595
:106EF00075E48AEA99E30E946BA482E595E40D9417
:106F00008D3108950E94FF94882341F0E0DC8111C7
:106F100005C084E292E40C94DA2408950E944E2A7B
:106F200081112EC062E472E481EB9AE30E947AA49C
:106F30008091C442813021F50E944E2A811112C0F5
:106F400062E48091AA399091AB390E94AE70409171
:106F500042425091434221E064E472E48AEA99E3B8
:106F60000F94F03127EF3CE342E452E464E472E42E
:106F700081EB9AE30E946BA482E492E40D948D313C
:106F80000895CF92DF92EF92FF920F931F93CF93CA
:106F9000DF930E944E2A882319F00AEA19E302C0FF
:106FA00001EB1AE383E392E40E94A6A6882349F04A
:106FB0008EDC811106C063E372E4C8010E94C02424
:106FC0008BC2809141428150823008F057C10E94AB
:106FD00028A7811104C07BDC882309F414C36EEE5A
:106FE00070E48CE69FE30E941DA680911F428130D1
:106FF00009F072C2E090EE40F090EF4082E0E816B7
:10700000F10408F400C380914142813039F4809149
:10701000F3408F7D8C3409F0CBC00AC08091F340DF
:10702000843209F0C5C08091F440833509F0C0C0B6
:107030000E944E2A811156C087E0ECE0F2E2A0EDFA
:10704000B4E401900D928A95E1F7E0EDF4E401904B
:107050000020E9F73197AF01405D544420E060ED36
:1070600074E48AEA99E30F94F0311092F0401092A0
:10707000F140E114F104A1F080E090E0CEEED0E424
:10708000FC01E251FF4B65818AEA99E30F947C325F
:107090008A819B8101968A839B838E159F0580F34D
:1070A0000F94432B1F928F9383E192E29F938F93D0
:1070B000C0EDD4E4DF93CF930F945867099000207C
:1070C000E9F72197AE01405D544421E060ED74E49E
:1070D0008AEA99E30F94F0310F900F900F900F9080
:1070E0000F900F900F94432B882371F181E00E9441
:1070F0006D90813069F48EEE90E40E9473A68EEE5E
:1071000090E40E9485A60F94202B0E9419A902C02A
:107110000E947AA9E5E8F3E4808190E0DC01AB57B6
:10712000BC4B25853685880F991FFC01EB57FC4B1E
:10713000418152811F960C9161E087EF9CE30E9490
:1071400000250F944A2C93C0E0922242F0922342F1
:107150000F94432B682FC8010E944B930E944E2A24
:10716000811185C00F94432B1F928F9380914142D0
:107170001F928F9389E192E29F938F93C0EDD4E4A5
:10718000DF93CF930F94586709900020E9F7219778
:10719000AE01405D544421E060ED74E48AEA99E375
:1071A0000F94F031EDB7FEB73896EDBFFEBF5FC06C
:1071B0000E944E2A811157C080914142823049F489
:1071C0008091F340843229F48091F440873409F4AB
:1071D0004AC086E0E7E3F2E2A0EDB4E401900D924C
:1071E0008A95E1F7E0EDF4E401900020E9F73197AA
:1071F000AF01405D544420E060ED74E48AEA99E315
:107200000F94F031EEEEF0E41282138280819181CE
:10721000892BA9F080E090E0EF01FC01E251FF4BE7
:1072200065818AEA99E30F947C328A819B81019679
:107230008A839B83288139818217930770F3E0ED5D
:10724000F4E480E290E08083918301900020E9F7EC
:107250003197AF01405D544421E060ED74E48AEA67
:1072600099E30F94F0318EEE90E40E9485A68EEEA5
:1072700090E40E9473A60F94202B2EC10F947626C3
:107280006B017C016EEE70E48CE69FE30E94A1A589
:1072900080911F42813039F0F5E6CF16D104E10428
:1072A000F10408F419C10F948D2680911F4281309A
:1072B00079F48EEE90E40E94F6A6882321F0E09007
:1072C0002142F12C40C0E090EE40F090EF403BC0F6
:1072D0000F2EFEEEEF2EF0E4FF2EF02DF701818150
:1072E0008F9380818F938DE392E29F938F93C0ED74
:1072F000D4E4DF93CF930F94586709900020E9F707
:107300002197AE01405D544421E060ED74E48AEAC7
:1073100099E30F94F031109221420F900F900F904B
:107320000F900F900F90F70180819181873991051F
:1073300030F086E990E08093EE409093EF40E0904B
:10734000EE40F090EF400E944E2A81115DC0FF9206
:10735000EF928CE592E29F938F93C0EDD4E4DF939C
:10736000CF930F94586709900020E9F72197AE0159
:10737000405D544420E060ED74E48AEA99E30F94A0
:10738000F0311092F0401092F1400F900F900F905A
:107390000F900F900F90E114F104A1F080E090E0C5
:1073A000CEEED0E4FC01E251FF4B65818AEA99E31D
:1073B0000F947C328A819B8101968A839B838E15F0
:1073C0009F0580F30F94432B1F928F9383E192E2EA
:1073D0009F938F93C0EDD4E4DF93CF930F945867BE
:1073E00009900020E9F72197AE01405D544421E067
:1073F00060ED74E48AEA99E30F94F0310F900F90F6
:107400000F900F900F900F900F94432B882371F1E2
:1074100081E00E946D90813069F48EEE90E40E94CC
:1074200073A68EEE90E40E9485A60F94202B0E94F6
:1074300019A902C00E947AA9E5E8F3E4808190E0EE
:10744000DC01AB57BC4B25853685880F991FFC01A5
:10745000EB57FC4B418152811F960C9161E087EF05
:107460009CE30E9400250F944A2C30C0E0922242F7
:10747000F09223420F94432B682FC8010E944B9334
:107480000E944E2A811122C00F94432B1F928F938A
:1074900089E692E29F938F93C0EDD4E4DF93CF937C
:1074A0000F94586709900020E9F72197AE01405DDD
:1074B000544421E060ED74E48AEA99E30F94F031DA
:1074C0000F900F900F900F900F900F908EEE90E412
:1074D0000E9473A60F94202B0F94BF26693C710560
:1074E0008105910508F48FC00F94D6260E944E2A7C
:1074F00081114AC08AE0EDE7F2E2A0EDB4E4019028
:107500000D928A95E1F7E0EDF4E401900020E9F7AF
:107510003197AF01405D544420E060ED74E48AEAA5
:1075200099E30F94F031EEEEF0E412821382808141
:107530009181892BA9F080E090E0EF01FC01E251FC
:10754000FF4B65818AEA99E30F947C328A819B81A3
:1075500001968A839B83288139818217930770F370
:10756000E0EDF4E480E290E08083918301900020DC
:10757000E9F73197AF01405D544421E060ED74E4D8
:107580008AEA99E30F94F03183EF90E40E9404A813
:107590008823A9F18091414281110BC0E9E4F3E411
:1075A00081E3808382E3818383E3828384E3838333
:1075B00014C0813041F4E9E4F3E480E38083818303
:1075C000828383830AC0E9E4F3E481E3808382E376
:1075D000818383E3828384E3838321E044E050E07A
:1075E00069E473E48CE69FE30F94F03121E044E01A
:1075F00050E069E473E48AEA99E30F94F0318EEE87
:1076000090E40E9473A6DF91CF911F910F91FF909C
:10761000EF90DF90CF9008958F929F92AF92BF929C
:10762000CF92DF92EF920F931F93CF93DF93EC01F2
:1076300080E00E94A6D04B015C01209709F45CC158
:107640001F8EFE01E05BFD4F1082CE010E94A11F44
:10765000882309F451C16E0186E3C80ED11CBE0116
:10766000615E7F4FC6010F94210A8E8F81111FC06A
:107670000E944E2A811119C08BE1E7E8F2E2A0EDE9
:10768000B4E401900D928A95E1F7E0EDF4E4019005
:107690000020E9F73197AF01405D544421E060EDEF
:1076A00074E48AEA99E30F94F03181E08F8F6CE7FC
:1076B00077E4C6010F948E0FFE01E15BFD4F8083DE
:1076C0008CE797E40E948ED78823A1F181E0FE0128
:1076D000E05BFD4F80838CE797E40E942BD70E94EC
:1076E0004E2A811127C0FE01E05BFD4F80811F9271
:1076F0008F93319780811F928F9382EA92E29F93BA
:107700008F9300ED14E41F930F930F945867F801C3
:1077100001900020E9F73197AF01405D544421E02A
:10772000B8018AEA99E30F94F031ADB7BEB7189665
:10773000ADBFBEBF8F8D813039F0FE01E05BFD4FE4
:107740008081813009F05CC00E944E2A811119C0ED
:107750008CE1E5EBF2E2A0EDB4E401900D928A95A4
:10776000E1F7E0EDF4E401900020E9F73197AF0193
:10777000405D544421E060ED74E48AEA99E30F949B
:10778000F0316894EE24E2F801ED12E2A5019401D3
:10779000BE01685E7F4FCE0106960E94F3598D832D
:1077A00040E050E0BA01CE010E948F2E8D818823E7
:1077B00009F4A2C082E00E94CAD0062F8BE00E948A
:1077C000CAD021E0611120E0BE016C5C7F4F43EB29
:1077D00050E4C6010E94F652CE010E94F61B9E01A3
:1077E000265A3D4FAE01475A5D4FBE016C5A7D4F40
:1077F000CE018D5A9D4F0E94162D0F9459187CC0B2
:107800008E010A5F1F4FB80183EB90E40E94CB58B2
:107810008D83811139C0A5019401BE01685E7F4F3F
:10782000C8010E942D568D8340E050E0BA01CE0180
:107830000E948F2E8D81882309F45EC082E00E9411
:10784000CAD0062F8BE00E94CAD021E0611120E04F
:10785000BE016C5C7F4F43EB50E4C6010E94F652C0
:10786000CE010E94F61B9E01265A3D4FAE01475A9B
:107870005D4FBE016C5A7D4FCE018D5A9D4F0E94C7
:10788000162D0F94591838C08E010B5A1D4F0F2E0C
:10789000F3EBAF2EF0E4BF2EF02DF501628573857A
:1078A00020E032E0A601C5010E94F82D0150110927
:1078B0006E01FDEACF1AFDEFDF0AD5011A966D9130
:1078C0007C911B979801A601C5010E942A2DFE01FB
:1078D000E75AFD4FD6018C918083C65ADD4FF801DF
:1078E00080818883D5011A964D915D916D917C912F
:1078F0001D97C5010F944F5DDF91CF911F910F919F
:10790000EF90DF90CF90BF90AF909F908F900895B1
:107910006DE288E499E30BDA882309F467C080916B
:107920008533882309F446C00E94166484E080935E
:1079300026060F9431258CE797E40E94E5E487EF53
:107940009CE36ADE8091473F8823F1F00E94A9E220
:10795000813019F0823069F017C08091463F88234A
:1079600029F08CE797E40E9447E20EC00E941AE2D9
:107970000BC08091463F882329F08CE797E40E9452
:10798000C9E302C00E9494E3109285330F944A2CFD
:1079900087EF9CE30E94992281110F94B32987EF0E
:1079A0009CE30E94E62960913A3F87EF9CE30E94A6
:1079B000AC141CC00F944A2C0F94912966E087EFF9
:1079C0009CE30E94AC1461E08DEF9CE30E94995807
:1079D0000E9418560F941D3B0E94EC6381E0809337
:1079E000853384E0809325060F943125809185337B
:1079F000882331F00E946A628111FCCF8091853327
:107A000008954F925F926F927F928F929F92AF9262
:107A1000BF92CF92DF92EF92FF921F93CF93DF93AB
:107A2000CDB7DEB72797CDBFDEBF7C0110924B49A3
:107A300010E00F2E812CFBE49F2EA12CB12CF02DF9
:107A40000F2EF0EDCF2EF4E4DF2EF02D0F2EF0E808
:107A50004F2EF5E25F2E612C712CF02D111120C0FC
:107A600080E096E9A0E0B0E0F70180839183A283F3
:107A7000B3838AE0E6EDF2E2D60101900D928A9599
:107A8000E1F7F60101900020E9F73197AF01405D81
:107A9000544421E0B6018AEA99E30F94F0315CC0C6
:107AA000113001F580EC92E1A0E0B0E0F7018083B5
:107AB0009183A283B38389E0E0EEF2E2D6010190E4
:107AC0000D928A95E1F7F60101900020E9F73197D0
:107AD000AF01405D544421E0B6018AEA99E30F9476
:107AE000F0313AC01230E9F4D7014D925D926D92B7
:107AF0007C92139789E0E9EEF2E2D60101900D92B3
:107B00008A95E1F7F60101900020E9F73197AF017E
:107B1000405D544421E0B6018AEA99E30F94F031C4
:107B20001BC0F70180829182A282B38289E0E2EFDA
:107B3000F2E2D60101900D928A95E1F7F6010190EB
:107B40000020E9F73197AF01405D544421E0B601D0
:107B50008AEA99E30F94F031D70114968C91149727
:107B60008D8315968C9115978E8316968C9116970A
:107B70008F838D919D910D90BC91A02D89839A83C7
:107B8000AB83BC8360E185E00F945B44BE016F5F13
:107B90007F4F80EA9AE00E94C9710F94BD2B08C004
:107BA0008EEB98E40E9434E6813041F00E94871BFE
:107BB0000F94D02B803A9F4098F37AC011111DC0CA
:107BC0008CE0EBEFF2E2A0EDB4E401900D928A9527
:107BD000E1F7E0EDF4E401900020E9F73197AF011F
:107BE000405D544421E060ED74E48AEA99E30F9427
:107BF000F03182E080934B4978C01130E9F48BE09A
:107C0000E7E0F3E2A0EDB4E401900D928A95E1F78C
:107C1000E0EDF4E401900020E9F73197AF01405D19
:107C2000544421E060ED74E48AEA99E30F94F03162
:107C300081E080934B4959C01230E9F48BE0E2E1D6
:107C4000F3E2A0EDB4E401900D928A95E1F7E0ED46
:107C5000F4E401900020E9F73197AF01405D54440E
:107C600021E060ED74E48AEA99E30F94F03183E057
:107C700080934B493AC08BE0EDE1F3E2A0EDB4E430
:107C800001900D928A95E1F7E0EDF4E40190002077
:107C9000E9F73197AF01405D544421E060ED74E4B1
:107CA0008AEA99E30F94F03184E080934B491DC038
:107CB0001F5F143009F0D2CE89E0E8E2F3E2A0EDD4
:107CC000B4E401900D928A95E1F7E0EDF4E40190BF
:107CD0000020E9F73197AF01405D544421E060EDA9
:107CE00074E48AEA99E30F94F0312796CDBFDEBFA2
:107CF000DF91CF911F91FF90EF90DF90CF90BF90D9
:107D0000AF909F908F907F906F905F904F9008956D
:107D1000CF92DF92EF92FF920F931F93CF9387EF53
:107D20009CE30E94BF14883009F4D6C087EF9CE31F
:107D30000E94BF14863009F4CFC08091543F9091C7
:107D4000553F8E349C4008F4BEC00E94A6D88111D5
:107D5000B4C0C2C00F948B2C81111FC00F948E2C05
:107D60000E944E2A811119C088E1E1E3F3E2A0EDFF
:107D7000B4E401900D928A95E1F7E0EDF4E401900E
:107D80000020E9F73197AF01405D544421E060EDF8
:107D900074E48AEA99E30F94F0310F94772C8111FF
:107DA00029C09AC08CE1E9E4F3E2A0EDB4E40190CB
:107DB0000D928A95E1F7E0EDF4E401900020E9F7F7
:107DC0003197AF01405D544421E060ED74E48AEAEC
:107DD00099E30F94F0310F940F25C0E00F94FE2427
:107DE000882331F00F940F25CF5FCA30B9F702C056
:107DF000CA30A0F30F9491290E9418560E944E2A6F
:107E0000811119C08EE0E7E5F3E2A0EDB4E4019042
:107E10000D928A95E1F7E0EDF4E401900020E9F796
:107E20003197AF01405D544421E060ED74E48AEA8B
:107E300099E30F94F0310F940F2501E010E0C0E0BA
:107E40000F2EFDE0CF2EF1E2DF2EF02D0F2EF0ED04
:107E5000EF2EF4E4FF2EF02D0F94FE24882341F141
:107E60000F940F25CF5F0E944E2A81111CC01F93D3
:107E70000F93DF92CF92FF92EF920F945867F70122
:107E800001900020E9F73197AF01405D544421E0B3
:107E9000B7018AEA99E30F94F0310F900F900F9099
:107EA0000F900F900F900F5F1F4FC33019F0D4CF7A
:107EB000C33090F20F94C2100FC00F94812C88230E
:107EC00009F46BCF47CF89E493E40E9431340E94D8
:107ED0004E2A811180CF66CFCF911F910F91FF90D5
:107EE000EF90DF90CF900895F8940E941E670F9452
:107EF00006440F94E1130F94421460E080E00F9465
:107F0000DA140F941D3B0E9434A50F945E130E9457
:107F1000E3ED41E060EA78E081EB9AE30F945232BE
:107F200065E170E280EA98E00E940B36E0EAF8E052
:107F300083818F7C8061838382E492E40F948D310E
:107F400061E084E292E40E9496A641E060EA7BE070
:107F50008CE69FE30F9452326EE070E280EA9BE081
:107F60000E940B36E0EAFBE083818F7C8061838393
:107F70008EEE90E40E9473A68EEE90E40E9485A699
:107F800061E083E392E40E9496A61092414210922F
:107F9000484385EC92E40F948D3141E060EA7AE049
:107FA00088EC9BE30F94523267E070E280EA9AE03B
:107FB0000E940B36E0EAFAE083818F7C8061838344
:107FC00041E060EA79E08AEA99E30F94523260E096
:107FD00070E280EA99E00E940B36E0EAF9E08381E2
:107FE0008F7C8061838382E595E40F948D310F94BB
:107FF00099240F9408270F94BD280F94592B0F94A0
:108000002E270F94292D0F9471110F94E4160E94BE
:10801000D70FC0E060E08C2F0F948213CF5FC83081
:10802000C9F787E08093A2007894E0E2F6E082E06E
:10803000868384E086830E9462D0811116C00E94EC
:1080400068D10E9492D10E94E2D50E947FD70E94FF
:1080500077D80E94BED881E00E946BD982E00E944E
:108060006BD981E08093453F27C00E9455D5882376
:1080700009F181E08093453F0E944E2A81111CC086
:108080008DE1E5E6F3E2A0EDB4E401900D928A956E
:10809000E1F7E0EDF4E401900020E9F73197AF015A
:1080A000405D544421E060ED74E48AEA99E30F9462
:1080B000F03102C01092453F0E940BD70F9459181F
:1080C0000E9435D581E00F946F286DE288E499E332
:1080D0000E9477360E942CA96FEE75E48EEB98E42F
:1080E0000E94A8DE8EEB98E40E948AD987EF9CE379
:1080F0000E94E23480E00F945D168CE797E40E94C2
:10810000E5E40F94921587EF9CE386DA81E00E9404
:10811000DCC880E00E94D6C880E00E94DFC880E012
:108120000E94E2C80E9421170E9402340E9438A5D2
:108130008EEB98E40E948AD987E090E262DC0E948C
:10814000A9E2813029F48091463F0E9477E825C05A
:108150000E94A9E2823091F481E00E94ACE2809119
:10816000463F882329F08CE797E40E94C9E302C0C8
:108170000E9494E381E00E945EE30FC00E94A9E2A6
:10818000833029F480ED94E40E948EE406C00E94BE
:10819000A9E2843011F40E94B5E884E080932606B9
:1081A0000E94EFED81E00E946A3482E00E946A340E
:1081B00087EF9CE30E94E6298AEA99E30E941ABAB3
:1081C0000E9413100F940B2E02E813E2C0EDD4E4CA
:1081D0000E9449376FEE75E48EEB98E40E944C16CE
:1081E00087EF9CE30E94DD1587EF9CE30E947515E5
:1081F00087EF9CE30E94992E87EF9CE30E949732C1
:108200000E944E3785DB0E9482370E94C13787EF7C
:108210009CE30E94911B0E941CEE0E94D9C88330EF
:1082200031F50E94BA1F882311F10E944E2A811154
:108230001EC00F946E291F928F931F930F93DF938D
:10824000CF930F945867FE0101900020E9F7319712
:10825000AF01405D544421E0BE018AEA99E30F94E6
:10826000F0310F900F900F900F900F900F9084E5CA
:108270009FE30E942D2465E873E487EF9CE30E944E
:10828000CB2565E873E487EF9CE30E941F260F94DB
:1082900068173EDD0FB607FC9BCF80E00E94C57CCF
:1082A0000E94D97CFFCFEF92FF920F931F93CF9341
:1082B000DF93009749F16115710541F141155105B1
:1082C00039F18A017B01EC010F94DF66F8018083AC
:1082D0009183892B89F0D70120E030E0FE01E20F85
:1082E000F31FE491ED932F5F3F4FF801808191815F
:1082F0002817390798F302C020E030E0F701E20FB9
:10830000F31F108281E005C080E003C080E001C05F
:1083100080E0DF91CF911F910F91FF90EF90089532
:108320000F931F93CF93DF930097C9F061157105E9
:10833000C1F041155105B9F0EA018B01FC016591CD
:108340007491C8010F94D866F80101900020E9F7F4
:108350003197E01BF10BE883F98381E005C080E0F1
:1083600003C080E001C080E0DF91CF911F910F91A9
:1083700008957F928F929F92AF92BF92CF92DF9299
:10838000EF92FF920F931F93CF93DF931F921F9251
:10839000CDB7DEB7009709F49BC06115710509F4EC
:1083A00097C0D42E7B018C01AE014F5F5F4FBC01A3
:1083B0008DEE94E178DF882309F48AC089819A815F
:1083C0005C012FEFA21AB20AF801E80FF91F20E2B0
:1083D0002083B8016A0D7B1DAE014F5F5F4F86EDB4
:1083E00094E161DF882309F473C089819A81A80E22
:1083F000B91EF801EA0DFB1D8DE0808382E0A80E16
:10840000B11C8AE08183B8016A0D7B1DAE014F5F0C
:108410005F4F8FEB94E147DF882309F459C0A981AE
:10842000BA81AA0EBB1E48018A0C9B1C0F2EFDE0D0
:108430007F2EF02DF40170820F2EFAE0CF2EF02D5A
:10844000C182C5010296800F911F0E9488D0F4015D
:10845000748ED5015E96C58EDD2059F1A00FB11F37
:108460008AE0EAE8F3E201900D928A95E1F7F7E2FB
:10847000AF0EB11C0E94B5D5BC01C8018A0D9B1D71
:108480000F943A670E94B5D5FC0101900020E9F7EE
:108490003197E81BF90BE131F10518F4E983FA8310
:1084A00004C080E190E089839A83A981BA81AA0DF2
:1084B000BB1DF801EA0FFB1F8DE0808312968AE056
:1084C0008183F801EA0FFB1F1082F701A083B183BB
:1084D0000F900F90DF91CF911F910F91FF90EF9030
:1084E000DF90CF90BF90AF909F908F907F90089536
:1084F000CF92DF92EF92FF920F931F93CF93DF9370
:108500001F921F92CDB7DEB76115710591F141152C
:10851000510579F1009769F17A016B018C0119829B
:108520001A82AE014F5F5F4F89E193E1BCDE882381
:1085300001F1C80106969F938F9384E993E29F937C
:108540008F9389819A818C0D9D1D9F938F930F949A
:108550005867F60101900020E9F73197EC19FD0901
:10856000D701ED93FC930F900F900F900F900F9009
:108570000F900F900F90DF91CF911F910F91FF906F
:10858000EF90DF90CF900895BF92CF92DF92EF925D
:10859000FF920F931F93CF93DF931F921F92CDB73C
:1085A000DEB7009709F482C06115710509F47EC039
:1085B0006B018C0119821A82DB011D921C92AE01A3
:1085C0004F5F5F4FBC018DE093E16DDE882309F4BE
:1085D0006DC0E8E2F4E587858F9386858F93858566
:1085E0008F9384858F9380E59BE29F938F938981FE
:1085F0009A81800F911F9F938F930F945867F80172
:1086000001900020E9F73197E01BF10BE983FA8331
:10861000CDBFDEBFB12C0F2EF9E9EF2EF3E2FF2E16
:10862000F02D2DC0EB2DF0E0EE0FFF1FEE0FFF1F22
:10863000E85DFB4ADF015A9613968C9113978F934E
:1086400012968C9112978F9311968C918F93828DA5
:108650008F93FF92EF9289819A81800F911F9F9350
:108660008F930F945867F80101900020E9F7319734
:10867000E01BF10BE983FA83B394CDBFDEBF0F9407
:10868000922CB81678F2E981FA81E00FF11F8DE0A3
:108690009AE0808391831282F80101900020E9F72B
:1086A0003197E01BF10BD601ED93FC930F900F90E7
:1086B000DF91CF911F910F91FF90EF90DF90CF90BE
:1086C000BF900895BF92CF92DF92EF92FF920F93E7
:1086D0001F93CF93DF9300D01F92CDB7DEB71982DF
:1086E0001A821B821C82009709F4CDC061157105A6
:1086F00009F4C9C0022FB42E6B017C011FEF120FC9
:10870000123108F0B5C0AE014F5F5F4FBC0185E28A
:1087100093E1C9DD882309F4B6C01A3079F5BB208E
:1087200069F069817A816E0D7F1DAE014D5F5F4FEB
:1087300086EB99E0F5DD81110EC0A5C069817A81D3
:108740006E0D7F1DAE014D5F5F4F82E999E0E8DD60
:10875000882309F498C069817A818B819C81680F94
:10876000791F69837A836E0D7F1DAE014D5F5F4F68
:1087700088E19BE098DD811171C085C084EF800F96
:10878000873008F046C0BB2089F069817A816E0D80
:108790007F1D812F90E0880F991FAE014D5F5F4FC5
:1087A0008C55964FBDDD811112C06DC069817A81F3
:1087B0006E0D7F1D812F90E0880F991FAE014D5FD8
:1087C0005F4F8058964FACDD882309F45CC0698107
:1087D0007A818B819C81680F791F69837A8322EF6C
:1087E000200F223058F46E0D7F1DAE014D5F5F4F9C
:1087F00084E999E095DD811131C045C06E0D7F1D82
:10880000AE014D5F5F4F83E09BE04DDD811126C0DF
:108810003AC0BB2091F069817A816E0D7F1D212FB6
:1088200030E0C901880F991FAE014D5F5F4F8C5535
:10883000964F76DD811112C026C069817A816E0D56
:108840007F1D212F30E0C901880F991FAE014D5FB8
:108850005F4F8058964F64DD8823A9F029813A81C3
:108860008B819C81820F931FF601808391830BC0C3
:10887000AE014F5F5F4FBC0185E293E114DD8823B9
:1088800011F010E0C6CF2496CDBFDEBFDF91CF91AF
:108890001F910F91FF90EF90DF90CF90BF900895C0
:1088A00089E10E94CAD081E0623009F080E0089539
:1088B000CF92DF92EF92FF921F93CF93DF9300D07E
:1088C0001F92CDB7DEB719821A821B821C820097D5
:1088D00009F453C06115710509F44FC0142F6B01E1
:1088E0007C01AE014F5F5F4FBC0185E293E1DBDCB1
:1088F000882309F442C0173089F01930E1F01130B3
:1089000039F569817A816E0D7F1DAE014D5F5F4F34
:1089100082EA9AE0C8DC811127C02FC069817A8180
:108920006E0D7F1DAE014D5F5F4F81E49AE0BBDCB1
:1089300081111AC022C069817A816E0D7F1DAE013E
:108940004D5F5F4F80EE99E0AEDC81110DC015C028
:1089500069817A816E0D7F1DAE014D5F5F4F82EAA6
:108960009AE0A1DC882349F029813A818B819C819E
:10897000820F931FF601808391832496CDBFDEBFC3
:10898000DF91CF911F91FF90EF90DF90CF900895EE
:10899000EF92FF920F931F93CF93DF931F921F923B
:1089A000CDB7DEB719821A820097B1F16115710552
:1089B00099F17B018C0187E10E94CAD0613051F4AA
:1089C000AE014F5F5F4FB8018BE294E16CDC811127
:1089D00016C022C061110AC0AE014F5F5F4FB801DF
:1089E0008EEA93E160DC81110AC016C0AE014F5FD0
:1089F0005F4FB80181E393E156DC882369F08981F8
:108A00009A81F801E80FF91F2DE020832AE02183E5
:108A10000296F701808391830F900F90DF91CF91A1
:108A20001F910F91FF90EF900895EF92FF920F9397
:108A30001F93CF93DF931F921F92CDB7DEB700979E
:108A400009F47EC04115510509F47CC0F22E8A015B
:108A5000E62EAE014F5F5F4FB80162DC811102C0AC
:108A600019821A8283E0E81629F18E1538F091E018
:108A7000E91659F082E0E81699F03AC094E0E91658
:108A800019F185E0E81651F133C0ECE7F7E4019005
:108A90000020E9F73197EC57F7446CE777E42BC0F7
:108AA000E3E9F7E401900020E9F7E459F74463E9CA
:108AB00077E421C0EAEAF7E401900020E9F7EB5AF5
:108AC000F7446AEA77E417C0E1ECF7E4019000208C
:108AD000E9F7E25CF74461EC77E40DC0E8EDF7E418
:108AE00001900020E9F7E95DF74468ED77E403C001
:108AF0006CE777E4E0E0EF3008F0EEE0CB018E0FBA
:108B0000911DFC01108289819A81800F911F0F9421
:108B10003A67F80101900020E9F73197E01BF10B6B
:108B2000FF2091F0C8018E0F911DFC018CE29DE0A9
:108B3000808391838AE090E08283938381E005C003
:108B400080E003C080E001C081E00F900F90DF91D2
:108B5000CF911F910F91FF90EF9008958F929F9268
:108B6000AF92BF92CF92DF92EF92FF920F931F933B
:108B7000CF93DF931F921F92CDB7DEB73091463F60
:108B8000311104C0FB011082118236C00097A1F19F
:108B9000672B91F14115510579F1022F4A016C01C2
:108BA0000F2EFBEBEF2EFAE1FF2EF02D11E0202F20
:108BB000A601612FC70139DF8823A9F0F6010190D2
:108BC0000020E9F731975F01AC18BD089E012F5FC7
:108BD0003F4FA501B601C4010F944F5B89819A8173
:108BE000A816B90631F41F5FF2E0EF0EF11C163043
:108BF000F1F6C4010F94FD5C0F900F90DF91CF91BF
:108C00001F910F91FF90EF90DF90CF90BF90AF90AA
:108C10009F908F9008958F929F92AF92BF92DF9214
:108C2000EF92FF920F931F93CF93DF93CDB7DEB7F1
:108C30002597CDBFDEBF009709F421C54115510529
:108C400009F41FC5D22E7A01162FAE014F5F5F4F78
:108C5000B70166DB811102C019821A82163109F050
:108C60006DC00F94D9054B015C01672B682B692BF4
:108C7000E1F486E10E94CAD020E13EE040E050E00D
:108C80000F940F655F934F933F932F9384EA93E282
:108C90009F938F9389819A818E0D9F1D9F938F93B0
:108CA0000F945867CDBFDEBFD3C486E10E94CAD0FF
:108CB000992324F586E10E94CAD020E13EE040E0FD
:108CC00050E00F940F65CA01B9010F946D37BF9240
:108CD000AF929F928F929F938F937F936F938FE921
:108CE00093E29F938F9389819A818E0D9F1D9F930D
:108CF0008F930F945867CDBFDEBFAAC486E10E9450
:108D0000CAD0BF92AF929F928F9220E13EE040E0A6
:108D100050E00F940F655F934F933F932F9380EA3A
:108D200093E29F938F9389819A818E0D9F1D9F93CC
:108D30008F930F945867CDBFDEBF8AC4123060F4A2
:108D4000812F0E942FD129813A81BC01C701820F56
:108D5000931F0F943A677CC4163081F486E00E941A
:108D6000CAD08B019C0189819A814BE0BE016B5F67
:108D70007F4F8E0D9F1D0F94C6376AC4153081F446
:108D800085E00E94CAD08B019C0189819A814BE0C9
:108D9000BE016B5F7F4F8E0D9F1D0F94123958C41B
:108DA000123009F06EC082E00E94CAD063317105B2
:108DB0008105910524F061E070E080E090E00130F1
:108DC00009F049C029813A812E0D3F1DDC01CB01FC
:108DD0000197A109B109880F991FAE014D5F5F4F3F
:108DE000B9018D58974F9CDA8130F9F4F701019061
:108DF0000020E9F73197EE19FF09E983FA8382E051
:108E00000E94CAD09F938F937F936F9389EA93E2D6
:108E10009F938F9389819A818E0D9F1D9F938F932E
:108E20000F945867CDBFDEBF13C482E00E94CAD042
:108E30009F938F937F936F938AEA93E29F938F938D
:108E400089819A818E0D9F1D9F938F930F945867F0
:108E5000CDBFDEBFFDC382E00E94CAD09F938F9337
:108E60007F936F9381E59BE29F938F9389819A8192
:108E70008E0D9F1D9F938F930F945867CDBFDEBFBC
:108E8000E7C3173109F086C087E10E94CAD04B01C1
:108E90005C01011113C0BF92AF929F926F9381E565
:108EA0009BE29F938F9389819A818E0D9F1D9F9343
:108EB0008F930F945867CDBFDEBFCAC391E0891668
:108EC0009104A104B10439F082E088169104A10450
:108ED000B10409F140C069817A816E0D7F1DAE0138
:108EE0004D5F5F4F88E098E0DED98111B1C31F92DA
:108EF0001F921F9281E08F9381E59BE29F938F9356
:108F000089819A818E0D9F1D9F938F930F9458672F
:108F1000CDBFDEBF9DC369817A816E0D7F1DAE011D
:108F20004D5F5F4F83E098E0BED9811191C31F92DE
:108F30001F921F9282E08F9381E59BE29F938F9314
:108F400089819A818E0D9F1D9F938F930F945867EF
:108F5000CDBFDEBF7DC369817A816E0D7F1DAE01FD
:108F60004D5F5F4F8CE098E09ED9811171C3BF9235
:108F7000AF929F928F9281E59BE29F938F9389811D
:108F80009A818E0D9F1D9F938F930F945867CDBF2D
:108F9000DEBF5EC31B3049F08DEE810F823028F0BA
:108FA000812F8D7F883109F05CC0812F0E94CAD04B
:108FB0004B015C01011113C0BF92AF929F926F935E
:108FC00081E59BE29F938F9389819A818E0D9F1DEE
:108FD0009F938F930F945867CDBFDEBF39C3672B24
:108FE000682B692BF9F469817A816E0D7F1DAE01C2
:108FF0004D5F5F4F8FE698E056D9811129C31F92CC
:109000001F921F921F9281E59BE29F938F9389810C
:109010009A818E0D9F1D9F938F930F945867CDBF9C
:10902000DEBF16C369817A816E0D7F1DAE014D5F73
:109030005F4F8CE698E037D981110AC3BF92AF9297
:109040009F928F9281E59BE29F938F9389819A8172
:109050008E0D9F1D9F938F930F945867CDBFDEBFDA
:10906000F7C2173009F05CC087E00E94CAD04B01FC
:109070005C01011113C0BF92AF929F926F9381E583
:109080009BE29F938F9389819A818E0D9F1D9F9361
:109090008F930F945867CDBFDEBFDAC2672B682B62
:1090A000692BF9F469817A816E0D7F1DAE014D5FE8
:1090B0005F4F88E698E0F7D88111CAC21F921F92CD
:1090C0001F921F9281E59BE29F938F9389819A81E2
:1090D0008E0D9F1D9F938F930F945867CDBFDEBF5A
:1090E000B7C269817A816E0D7F1DAE014D5F5F4F02
:1090F00084E698E0D8D88111ABC2BF92AF929F921C
:109100008F9281E59BE29F938F9389819A818E0D47
:109110009F1D9F938F930F945867CDBFDEBF98C25A
:10912000143009F05CC084E00E94CAD04B015C019D
:10913000011113C0BF92AF929F926F9381E59BE2A2
:109140009F938F9389819A818E0D9F1D9F938F93FB
:109150000F945867CDBFDEBF7BC2672B682B692B8E
:10916000F9F469817A816E0D7F1DAE014D5F5F4F0D
:109170008DE598E098D881116BC21F921F921F92C3
:109180001F9281E59BE29F938F9389819A818E0D37
:109190009F1D9F938F930F945867CDBFDEBF58C21A
:1091A00069817A816E0D7F1DAE014D5F5F4F84E551
:1091B00098E079D881114CC2BF92AF929F928F9262
:1091C00081E59BE29F938F9389819A818E0D9F1DEC
:1091D0009F938F930F945867CDBFDEBF39C2133072
:1091E00009F0ADC083E00E94CAD04B015C010111BF
:1091F00013C0BF92AF929F926F9381E59BE29F93C2
:109200008F9389819A818E0D9F1D9F938F930F94C9
:109210005867CDBFDEBF1CC291E089169104A1043E
:10922000B10461F182E088169104A104B10409F44B
:1092300045C081149104A104B10409F060C06981A2
:109240007A816E0D7F1DAE014D5F5F4F88E498E01F
:109250002AD88111FDC11F921F921F921F9281E592
:109260009BE29F938F9389819A818E0D9F1D9F937F
:109270008F930F945867CDBFDEBFEAC169817A81B1
:109280006E0D7F1DAE014D5F5F4F8FE398E00BD8F1
:109290008111DEC11F921F921F9281E08F9381E5A1
:1092A0009BE29F938F9389819A818E0D9F1D9F933F
:1092B0008F930F945867CDBFDEBFCAC169817A8191
:1092C0006E0D7F1DAE014D5F5F4F8AE398E00E94F7
:1092D00053418111BDC11F921F921F9282E08F9353
:1092E00081E59BE29F938F9389819A818E0D9F1DCB
:1092F0009F938F930F945867CDBFDEBFA9C169813B
:109300007A816E0D7F1DAE014D5F5F4F88E498E05E
:109310000E94534181119CC1BF92AF929F928F9244
:1093200081E59BE29F938F9389819A818E0D9F1D8A
:109330009F938F930F945867CDBFDEBF89C11931BA
:1093400009F0AFC089E10E94CAD04B015C01011154
:1093500013C0BF92AF929F926F9381E59BE29F9360
:109360008F9389819A818E0D9F1D9F938F930F9468
:109370005867CDBFDEBF6CC191E089169104A1048E
:10938000B10469F182E088169104A104B10409F4E2
:1093900047C081149104A104B10409F062C069813D
:1093A0007A816E0D7F1DAE014D5F5F4F86E398E0C1
:1093B0000E94534181114CC11F921F921F921F9214
:1093C00081E59BE29F938F9389819A818E0D9F1DEA
:1093D0009F938F930F945867CDBFDEBF39C16981CA
:1093E0007A816E0D7F1DAE014D5F5F4F80E398E087
:1093F0000E94534181112CC11F921F921F9281E044
:109400008F9381E59BE29F938F9389819A818E0D43
:109410009F1D9F938F930F945867CDBFDEBF18C1D8
:1094200069817A816E0D7F1DAE014D5F5F4F88E2CD
:1094300098E00E94534181110BC11F921F921F920D
:1094400082E08F9381E59BE29F938F9389819A813C
:109450008E0D9F1D9F938F930F945867CDBFDEBFD6
:10946000F7C069817A816E0D7F1DAE014D5F5F4F40
:1094700086E398E00E9453418111EAC0BF92AF9207
:109480009F928F9281E59BE29F938F9389819A812E
:109490008E0D9F1D9F938F930F945867CDBFDEBF96
:1094A000D7C0123109F05EC082E10E94CAD04B01E0
:1094B0005C01011113C0BF92AF929F926F9381E53F
:1094C0009BE29F938F9389819A818E0D9F1D9F931D
:1094D0008F930F945867CDBFDEBFBAC0672B682B40
:1094E000692B01F569817A816E0D7F1DAE014D5F9B
:1094F0005F4F87E198E00E9453418111A9C01F92FC
:109500001F921F921F9281E59BE29F938F93898107
:109510009A818E0D9F1D9F938F930F945867CDBF97
:10952000DEBF96C069817A816E0D7F1DAE014D5FF1
:109530005F4F8FE098E00E945341811189C0BF9234
:10954000AF929F928F9281E59BE29F938F93898147
:109550009A818E0D9F1D9F938F930F945867CDBF57
:10956000DEBF76C0153109F05EC085E10E94CAD029
:109570004B015C01011113C0BF92AF929F926F9398
:1095800081E59BE29F938F9389819A818E0D9F1D28
:109590009F938F930F945867CDBFDEBF59C0672B41
:1095A000682B692B01F569817A816E0D7F1DAE01F3
:1095B0004D5F5F4F83E298E00E945341811148C0A4
:1095C0001F921F921F921F9281E59BE29F938F93A0
:1095D00089819A818E0D9F1D9F938F930F94586759
:1095E000CDBFDEBF35C069817A816E0D7F1DAE01B2
:1095F0004D5F5F4F8EE198E00E945341811128C07A
:10960000BF92AF929F928F9281E59BE29F938F933F
:1096100089819A818E0D9F1D9F938F930F94586718
:10962000CDBFDEBF15C0812F0E94CAD09F938F93FC
:109630007F936F9381E59BE29F938F9389819A81BA
:109640008E0D9F1D9F938F930F945867CDBFDEBFE4
:10965000F70101900020E9F73197EE19FF09DD20AD
:1096600091F0C7018E0F911DFC018CE29DE080837B
:1096700091838AE090E08283938381E005C080E05B
:1096800003C080E001C081E02596CDBFDEBFDF9141
:10969000CF911F910F91FF90EF90DF90BF90AF900F
:1096A0009F908F9008956F927F928F929F92AF922A
:1096B000BF92CF92DF92EF92FF920F931F93CF93BF
:1096C000DF931F921F92CDB7DEB70097B1F1672BE2
:1096D000A1F14115510589F1802E922E3A016C01BC
:1096E0000F2EFAE6EF2EFCE1FF2EF02D10E0082DF4
:1096F000292DA601612FC7018EDA8823A9F0F60172
:1097000001900020E9F731975F01AC18BD089E0178
:109710002F5F3F4FA501B601C3010F944F5B8981B5
:109720009A81A816B90631F41F5F82E0E80EF11C99
:109730001C31E9F6C3010F94FD5C0F900F90DF918F
:10974000CF911F910F91FF90EF90DF90CF90BF903E
:10975000AF909F908F907F906F9008958F929F927F
:10976000AF92BF92DF92EF92FF920F931F93CF932E
:10977000DF931F921F92CDB7DEB7009709F48FC019
:109780006115710509F48BC04B017C010E94B5D5B0
:109790009F938F9380EB93E29F938F93FF92EF922F
:1097A0000F945867F70101900020E9F73197AF0156
:1097B0004E195F094231510510F041E150E09E0120
:1097C0002F5F3F4FB701C4010F944F5B0F900F9075
:1097D0000F900F900F900F90D12C0F2EFBE0AF2E1B
:1097E000FAE2BF2EF02D8D2D0E94A6D09F938F936D
:1097F0007F936F93BF92AF92FF92EF920F9458674F
:10980000F70101900020E9F731978F010E191F0928
:109810009E012F5F3F4FA801B701C4010F944F5B1A
:10982000CDBFDEBF89819A810817190731F4D3941F
:1098300096E1D912D8CF11E001C011E00F2EF0EB64
:10984000AF2EF3E2BF2EF02D812F0E9416D99F93E9
:109850008F93BF92AF92FF92EF920F945867F701E8
:1098600001900020E9F73197AF014E195F094231AD
:10987000510510F041E150E09E012F5F3F4FB701CD
:10988000C4010F944F5B1F5F0F900F900F900F90CC
:109890000F900F901330C1F6C4010F94FD5C0F9030
:1098A0000F90DF91CF911F910F91FF90EF90DF907C
:1098B000BF90AF909F908F9008952F923F924F92BC
:1098C0005F926F927F928F929F92AF92BF92CF9250
:1098D000DF92EF92FF920F931F93CF93DF93CDB759
:1098E000DEB7E197CDBFDEBF91E09BA761157105A3
:1098F00009F4EAC34115510509F4E8C38A017B0163
:1099000089AB0F944A2C29A9213089F4A80166E873
:1099100073E3CE010B960E943E57182F86E08BA76B
:109920000F9407196DA77EA78FA798AB1AC0A8013F
:1099300066E873E3CE010B960E94B357182F0F947D
:1099400007196DA77EA78FA798AB82E00F948017A9
:10995000862FAE01445D5F4FBE01655D7F4F0E9463
:109960000E22112309F4B4C341E0BE01675F7F4FAB
:10997000C7010E94B94149855A85CA01A0E0B0E0FB
:1099800089839A83AB83BC839E01275F3F4FB701D6
:10999000CE010B960F944F5BCE010B960F94FD5C9E
:1099A000BE01655F7F4FC701D9DE0DE0D7010C9383
:1099B0001AE011961C939E01275F3F4F42E050E052
:1099C000B701CE010B960F944F5BCE010B960F940F
:1099D000FD5CE6E8F3E3018B128B9E01275F3F4FAE
:1099E00043E150E0BF01CE010B960F944F5BCE01D7
:1099F0000B960F94FD5CB9A9B1116EC30F945C195D
:109A00000F94451969C301E021E0A701612FC60148
:109A100002D9882381F0F70101900020E9F73197FE
:109A2000AF014E195F099E01275F3F4FB701CE017D
:109A30000B960F944F5BE2E0CE0ED11C1F5F1330EC
:109A400011F70F2EFCE7CF2EFCE1DF2EF02D19E0F1
:109A500001E021E0A701612FC601DDD8882381F054
:109A6000F70101900020E9F73197AF014E195F0926
:109A70009E01275F3F4FB701CE010B960F944F5BBE
:109A8000F2E0CF0ED11C1F5F1B3011F70F2EF2E159
:109A90008F2E912CA12CB12CF02D28E1821691044F
:109AA000A104B10451F401E021E0A70169E18CE9CE
:109AB0009CE1B1D881110EC030C001E021E0A701C6
:109AC000682DC401880F991F8659934EA4D8882306
:109AD000C1F007C00F2EF9E18F2E912CA12CB12CD3
:109AE000F02DF70101900020E9F73197AF014E19F1
:109AF0005F099E01275F3F4FB701CE010B960F9480
:109B00004F5B33E0830E911CA11CB11C4AE184160B
:109B10009104A104B10408F4C0CFCE010B960F94B8
:109B2000FD5C89E00E94CAD06F3171058105910505
:109B3000C0F4DC01CB01072E7CE0880F991FAA1F1F
:109B4000BB1F7A95D1F7702D89839A83AB83BC8331
:109B500080E090E1A0E0B0E08D839E83AF83B88782
:109B600017C0DC01CB01072E79E0880F991FAA1FCF
:109B7000BB1F7A95D1F7702D89839A83AB83BC8301
:109B800080E092E0A0E0B0E08D839E83AF83B88751
:109B90008DA59EA5AFA5B8A98115904EA140B10590
:109BA00089F489E00E94CAD06E3171058105910562
:109BB00049F080E090E1A0E0B0E08D839E83AF8328
:109BC000B88741C089819A81AB81BC812DA53EA512
:109BD0004FA558A9281739074A075B07A1F1AE011D
:109BE000475F5F4FB70184ED99E00E945341813098
:109BF00081F4F70101900020E9F73197AF014E1988
:109C00005F099E01275F3F4FB701CE010B960F946E
:109C10004F5BCE010B960F94FD5CCE010B960F941B
:109C2000445D39A9311156C20F94D31987EF9CE3D3
:109C30000E94992281110F94B32987EF9CE30E941F
:109C4000E62980E051C2AE01475F5F4FB70188EC63
:109C500099E00E945341813081F4F7010190002086
:109C6000E9F73197AF014E195F099E01275F3F4F1A
:109C7000B701CE010B960F944F5B48A94F935FA598
:109C80005F938EA58F939DA59F9388858F938F81DA
:109C90008F938E818F938D818F9384EB93E29F932B
:109CA0008F93FF92EF920F945867F7010190002075
:109CB000E9F73197AF014E195F099E01275F3F4FCA
:109CC000B701CE010B960F944F5B88E290E0898735
:109CD0009A8768E2C7010E9454B9482F50E060E0BB
:109CE00070E049835A836B837C83682F70E0C701DF
:109CF0000F945639CDBFDEBF8823C9F049815A8100
:109D00009E01275F3F4FB701CE010B960F944F5B2B
:109D10008DE0F70180838AE081839E01275F3F4FBA
:109D200042E050E0B701CE010B960F944F5BBE01AD
:109D30006F5F7F4FC7010E94C84449815A819E01CD
:109D4000275F3F4FB701CE010B960F944F5B6BE33C
:109D500070E0C7010E94A7B8A0E0B0E089839A83B1
:109D6000AB83BC830E944E2A81110EC0F701019083
:109D70000020E9F73197AF014E195F0920E0B701E4
:109D80008AEA99E30F94F03149815A816B817C8191
:109D90004115510561057105C1F09E01275F3F4FD7
:109DA000B701CE010B960F944F5B8DE0D7018C93DA
:109DB0008AE011968C939E01275F3F4F42E050E06E
:109DC000B701CE010B960F944F5BCE010B960F940B
:109DD000FD5C0E94D25B19821A821B821C822DA517
:109DE0003EA54FA558A9232B242B252B09F433C1BD
:109DF00080E090E0DC010F2EFDEE2F2EF3E23F2EEF
:109E0000F02D0F2EFFEB8F2EF3E29F2EF02D880FFB
:109E1000991FAA1FBB1FBC01CD017E5F8F4F9F4FB3
:109E20000E94DA5B0E94655E8111FCCF80E091E0C8
:109E3000E6ECF3E4DF019C011D9221503040E1F794
:109E40006F010F2EF6ECAF2EF4E4BF2EF02D8F0134
:109E50000E9468B8D8018D939D938D01AA16BB0608
:109E6000B9F70E94A55C0F941D3BCE010B960F9491
:109E7000FD5C412C512C3201F601619171916F0111
:109E8000AE014B5F5F4F8BA50E94EA14882309F453
:109E900096C088858F938F818F938E818F938D81CC
:109EA0008F9389819A81AB81BC81840D951DA61DFC
:109EB000B71DBF93AF939F938F939F928F92FF9203
:109EC000EF920F945867F70101900020E9F731975E
:109ED000AF014E195F099E01275F3F4FB701CE01C9
:109EE0000B960F944F5B182FCDBFDEBF882309F46C
:109EF0008CC00E944E2A811126C089819A81AB8133
:109F0000BC81840D951DA61DB71DBF93AF939F9374
:109F10008F931F921F9349EC53E25F934F93FF92ED
:109F2000EF920F945867F70101900020E9F73197FD
:109F3000AF014E195F0920E0B7018AEA99E30F9457
:109F4000F031CDBFDEBFF70101900020E9F7319776
:109F5000AF014E195F099E01275F3F4FB701CE0148
:109F60000B960F944F5B182F0E944E2A81114DC003
:109F700089819A81AB81BC81840D951DA61DB71D79
:109F8000BF93AF939F938F931F921F93EAEDF3E2DA
:109F9000FF93EF93FF92EF920F945867F7010190B0
:109FA0000020E9F73197AF014E195F0920E0B701B2
:109FB0008AEA99E30F94F031CDBFDEBF26C00E943C
:109FC0004E2A811122C089819A81AB81BC81840D86
:109FD000951DA61DB71DBF93AF939F938F933F927F
:109FE0002F92FF92EF920F945867F7010190002093
:109FF000E9F73197AF014E195F0920E0B7018AEA0E
:10A0000099E30F94F031CDBFDEBF9FEF491A590A93
:10A01000690A790AA0E84A1651046104710409F03A
:10A020002BCFCE010B960F94FD5C89819A81AB8179
:10A03000BC8180589F4FAF4FBF4F89839A83AB83BA
:10A04000BC832DA53EA54FA558A982179307A40749
:10A05000B50708F4DCCECE010B960F94FD5CCE0163
:10A060000B960F94445D1092973386E893E30E9419
:10A07000925839A931110DC00F94D31987EF9CE381
:10A080000E94992281110F94B32987EF9CE30E94CB
:10A09000E62903EB10E4D80112966D917C91139799
:10A0A0008D919C910F947958D0D56DEF7CE3C801C8
:10A0B0000E94CB58F8014285538564857585C80197
:10A0C0000F944F5D81E010C080E00EC080E00CC0B6
:10A0D00080E00AC080E008C00F2EFAE6CF2EFCE137
:10A0E000DF2EF02D10E08FCCE196CDBFDEBFDF91EB
:10A0F000CF911F910F91FF90EF90DF90CF90BF9085
:10A10000AF909F908F907F906F905F904F903F9017
:10A110002F900895CF92DF92EF92FF920F931F93AB
:10A12000CF93DF931F921F92CDB7DEB7009709F44C
:10A1300057C06115710509F453C07B018C01AE0154
:10A140004F5F5F4FBC018DEE94E10E945341882325
:10A1500009F446C089819A816C012FEFC21AD20A94
:10A16000F801E80FF91F20E22083B8016C0D7D1D76
:10A17000AE014F5F5F4F86ED94E10E94534188230B
:10A1800079F189819A81C80ED91EF801EC0DFD1D67
:10A190008DE0808382E0C80ED11C8AE08183B80103
:10A1A0006C0D7D1DAE014F5F5F4F88EA94E10E9408
:10A1B00053418823A9F089819A81C80ED91EF801DC
:10A1C000EC0DFD1D8DE0808322E0C20ED11C8AE0E3
:10A1D0008183F801EC0DFD1D1082F701C082D18250
:10A1E0000F900F90DF91CF911F910F91FF90EF9003
:10A1F000DF90CF900895EF92FF920F931F93CF932C
:10A20000DF93CDB7DEB7A297CDBFDEBF009709F4CD
:10A2100051C06115710509F44FC07B018C0160E0EC
:10A22000CE01039615D7882309F44BC0B701C801A6
:10A2300071DFF701408151819E012F5F3F4FB801CF
:10A24000CE0103960F944F5BCE0103960F94FD5CF5
:10A25000F7012081318189819A812817390771F5A9
:10A26000BE016D5F7F4FC80179DAA701B80182EAAC
:10A270009CE10E945341813099F4F7014081518162
:10A280009E012F5F3F4FB801CE0103960F944F5BA5
:10A29000F7012081318189819A812817390781F45A
:10A2A000CE0103960F94445D81E012D70F944A2C9F
:10A2B00081E007C080E005C080E003C080E001C00D
:10A2C00080E0A296CDBFDEBFDF91CF911F910F91AD
:10A2D000FF90EF9008950F931F93CF93DF931F92FA
:10A2E0001F92CDB7DEB70F944A2C8091393F823050
:10A2F00009F462C028F4882359F0813081F1D6C076
:10A30000843009F485C008F464C08A30E1F0CEC01E
:10A3100060E083E990E47FD5811107C060913A3F06
:10A3200087EF9CE30E94AC14C9C00F94991181116E
:10A3300004C081E08093393FC1C08AE08093393FF7
:10A340000F945B2ABBC00F94722A6C3D7540810547
:10A35000910508F4B3C081E08093393FAFC040E07D
:10A360006BE27DE38DE29DE30E94B94107EF1CE3C0
:10A37000F80144A955A99E012F5F3F4F6DE27DE38F
:10A3800083E990E40F944F5B83E990E40F94FD5CC4
:10A39000F80124A935A989819A812817390741F044
:10A3A0001092393F60913A3FC8010E94AC1486C0B8
:10A3B00082E08093393F82C000E021E043E950E42D
:10A3C0006BE27DE38DE29DE36ED983E08093393FBC
:10A3D00075C04BE25DE36DE27DE382EA9CE10E94A1
:10A3E0005341813069F440912B3D50912C3D9E01A9
:10A3F0002F5F3F4F6DE27DE383E990E40F944F5B65
:10A4000083E990E40F94445D84E08093393F56C023
:10A410000E94A9E2882381F10F94A52B8823C9F01B
:10A420000E94BA1F882309F449C087EF9CE30E9469
:10A43000992281110F94B32987EF9CE30E94E629AA
:10A440001092393F60913A3F87EF9CE30E94AC1431
:10A4500035C087EF9CE30E94992281110F94B329A4
:10A4600087EF9CE30E94E6291092393F61E087EF75
:10A470009CE30E94AC1422C00F94ED29672B682B3B
:10A48000692BE1F487EF9CE30E94992281110F94DC
:10A49000B32987EF9CE30E94E6291092393F60912F
:10A4A0003A3F87EF9CE30E94AC1408C01092393FFA
:10A4B00060913A3F87EF9CE30E94AC140F900F909D
:10A4C000DF91CF911F910F9108959F92AF92BF920C
:10A4D000CF92DF92EF92FF920F931F93CF93DF9370
:10A4E00000D0CDB7DEB7009709F471C061157105D2
:10A4F00009F46DC0A42E6B017C018EE0E8EFF3E25D
:10A50000D70101900D928A95E1F7F70101900020A3
:10A51000E9F73197EE19FF09E983AF0155279E014D
:10A520002E5F3F4FB701C6010F944F5BB12C0F2E2A
:10A53000FCE29F2EF02D8B2D0E9425D88B019C01D3
:10A5400048E0BE016F5F7F4FC7010F94743982E00E
:10A550008B1550F08981F701E80FF11D90828F5F14
:10A56000F701E80FF11D1082F70101900020E9F7D3
:10A570003197EE19FF09E983AF0155279E012E5F40
:10A580003F4FB701C6010F944F5B898190E02A814C
:10A590003B818217930721F4B394E4E0BE12CBCF42
:10A5A000AA2081F08DE0F70180838AE0818382E038
:10A5B00089839E012E5F3F4F42E050E0B701C60104
:10A5C0000F944F5BC6010F94FD5C0F944A2C2396A9
:10A5D000CDBFDEBFDF91CF911F910F91FF90EF9024
:10A5E000DF90CF90BF90AF909F9008959F92AF92D1
:10A5F000BF92CF92DF92EF92FF920F931F93CF9370
:10A60000DF931F921F92CDB7DEB7009709F4E1C028
:10A610006115710509F4DFC04115510509F4DDC06C
:10A62000902E122F5A016B017C010F944A2C41E0AD
:10A63000B601C7010E94B941F601408151819E01D6
:10A640002F5F3F4FB701C5010F944F5BC5010F94BA
:10A65000FD5CF6012081318189819A8128173907B3
:10A6600009F0BDC08DE0E6E0F4E2D70101900D9263
:10A670008A95E1F7F70101900020E9F73197AF01E2
:10A680004E195F0955279E012F5F3F4FB701C50146
:10A690000F944F5BC5010F94FD5CB501C7015ED8F7
:10A6A0008DE0F70180838AE081839E012F5F3F4F19
:10A6B00042E050E0B701C5010F944F5BC5010F9414
:10A6C000FD5C41E0B501C70100DFA601B70187EFDE
:10A6D0009CE30E947842F601408151819E012F5FE8
:10A6E0003F4FB701C5010F944F5BC5010F94FD5C4F
:10A6F000F6012081318189819A812817390709F073
:10A7000070C0B601C7010E94C442F6014081518168
:10A710009E012F5F3F4FB701C5010F944F5BC501ED
:10A720000F94FD5CF6012081318189819A8128177F
:10A73000390709F058C001E021E0A501B601C701C1
:10A740000E94534B21E0A501B601C7010E94AE450E
:10A750000E945044882331F0492DB601C7010E9460
:10A76000584406C0292D412FB601C7010E946243FB
:10A77000F601408151819E012F5F3F4FB701C50116
:10A780000F944F5BC5010F94FD5CF6012081318170
:10A7900089819A812817390741F5B601C7010E94BE
:10A7A000C844F601408151819E012F5F3F4FB701A0
:10A7B000C5010F944F5BC5010F94FD5C81E0F6016C
:10A7C0004081518129813A814217530779F080E015
:10A7D0000DC080E00BC080E009C080E007C080E0D1
:10A7E00005C080E003C080E001C080E00F900F90C2
:10A7F000DF91CF911F910F91FF90EF90DF90CF905D
:10A80000BF90AF909F9008952F923F924F925F928A
:10A810006F927F928F929F92AF92BF92CF92DF9270
:10A82000EF92FF920F931F93CF93DF93CDB7DEB7D5
:10A83000A897CDBFDEBF4115510509F4D7C1211539
:10A84000310509F4D5C16115710509F4D3C1280199
:10A8500069011A017B0188A70F944A2CA60166E8BA
:10A8600073E3CE010796A7D6882309F4C5C141E05A
:10A87000BE016B5F7F4FC1010E94B9414D815E8176
:10A880009E012B5F3F4FB101CE0107960F944F5BA6
:10A89000CE0107960F94FD5CBE01695F7F4FC10139
:10A8A0000E94AE4B1DE0F10110830AE001839E017E
:10A8B0002B5F3F4F42E050E0B101CE0107960F946D
:10A8C0004F5BCE0107960F94FD5CE6E8F3E3118B36
:10A8D000028B9E012B5F3F4F43E150E0BF01CE0151
:10A8E00007960F944F5BCE0107960F94FD5C0F2ED9
:10A8F000FAE6CF2EFCE1DF2EF02D10E001E021E0A2
:10A90000A101612FC6010E940B46882381F0F1014D
:10A9100001900020E9F73197AF01421953099E01D8
:10A920002B5F3F4FB101CE0107960F944F5BF2E0D2
:10A93000CF0ED11C1F5F133009F70F2EFCE7CF2E6F
:10A94000FCE1DF2EF02D19E001E021E0A101612FF3
:10A95000C6010E940B46882381F0F101019000207E
:10A96000E9F73197AF01421953099E012B5F3F4F21
:10A97000B101CE0107960F944F5B22E0C20ED11CAD
:10A980001F5F1B3009F70F2EF2E18F2E912CA12CA7
:10A99000B12CF02D88E188169104A104B10491F442
:10A9A00001E021E0A10169E18CE99CE10E940B46F4
:10A9B000811116C00F2EFCE18F2E912CA12CB12CF1
:10A9C000F02D31C001E021E0A101682DC401880F04
:10A9D000991F8659934E0E940B468823C1F007C0E9
:10A9E0000F2EF9E18F2E912CA12CB12CF02DF1011D
:10A9F00001900020E9F73197AF01421953099E01F8
:10AA00002B5F3F4FB101CE0107960F944F5B93E050
:10AA1000890E911CA11CB11CEAE18E169104A104BF
:10AA2000B10408F4B7CF1F92F8A5FF9383E194E235
:10AA30009F938F933F922F920F945867F10101904B
:10AA40000020E9F73197AF01421953099E012B5FAE
:10AA50003F4FB101CE0107960F944F5BCE01079691
:10AA60000F94FD5C612C712C0F900F900F900F9044
:10AA70000F900F90411451046104710409F4A7C0B0
:10AA8000870175016401812C912C5401F8014191D9
:10AA90005191619171918F019E012F5F3F4F88A568
:10AAA0000E94D02E882309F482C08C818F938B81E1
:10AAB0008F938A818F9389818F93BF92AF929F9258
:10AAC0008F928FEB93E29F938F933F922F920F94ED
:10AAD0005867F10101900020E9F73197AF01421961
:10AAE00053099E012B5F3F4FB101CE0107960F9492
:10AAF0004F5B8FA3CDBFDEBF9FA1992309F457C041
:10AB00000E944E2A81111FC0FF92EF92DF92CF92D6
:10AB10001F92EFA1EF9389EC93E29F938F933F9263
:10AB20002F920F945867F10101900020E9F73197B7
:10AB3000AF014219530920E0B1018AEA99E30F9469
:10AB4000F031CDBFDEBFF10101900020E9F7319770
:10AB5000AF01421953099E012B5F3F4FB101CE0156
:10AB600007960F944F5B8FA30E944E2A81111FC03E
:10AB7000FF92EF92DF92CF921F929FA19F93EAEDF7
:10AB8000F3E2FF93EF933F922F920F945867F101F6
:10AB900001900020E9F73197AF014219530920E0F5
:10ABA000B1018AEA99E30F94F031CDBFDEBF9FEF88
:10ABB000891A990AA90AB90AEFEFCE1ADE0AEE0A33
:10ABC000FE0A84149504A604B70408F45FCFCE01EE
:10ABD00007960F94FD5CCE0107960F94445D10928A
:10ABE000973386E893E39ED281E007C080E005C0FA
:10ABF00080E003C080E001C080E0A896CDBFDEBF4A
:10AC0000DF91CF911F910F91FF90EF90DF90CF9048
:10AC1000BF90AF909F908F907F906F905F904F907C
:10AC20003F902F900895089580919B330895089543
:10AC300010929B3380919A33882331F010929A338B
:10AC400083EB90E40D94445D089583EB90E40D94C0
:10AC5000445D089580919A330895CF92DF92EF92E8
:10AC6000FF921F93CF93DF93CDB7DEB76897CDBF29
:10AC7000DEBF6C017B0184E1EEE1F4E2DE011596BA
:10AC800001900D928A95E1F7DA01C9010196A11DA3
:10AC9000B11D883E23E09207A105B1050CF460C008
:10ACA0001F921F921F9281E08F938EEE91E29F93ED
:10ACB0008F93CE0101969F938F930F94586789814C
:10ACC000898B8A818A8B8B818B8B80E38D838AE34E
:10ACD0008E83CDBFDEBFE114F10459F0D701FE0130
:10ACE00038969E01245F3F4F8D918193E217F307C1
:10ACF000D9F710E346E0BE016B5F7F4F83EB90E432
:10AD00000F94B15899EF980F9230C8F48B8989331A
:10AD100099F48A89893361F48989893321F41092FD
:10AD20009A3380E03CC08F5F898B1A8B1B8BE2CFFC
:10AD30001B8B8F5F8A8BDECF8F5F8B8BDBCF882364
:10AD400021F010929A3380E02AC081E080939A33F8
:10AD5000BE01695F7F4FC6010F943A6781E01FC053
:10AD6000BF93AF939F938F938EEE91E29F938F93B8
:10AD7000CE0101969F938F930F9458678981898B99
:10AD80008A818A8B8B818B8B80E38D838AE38E8390
:10AD9000CDBFDEBFE114F10409F0A0CFAACF6896C1
:10ADA000CDBFDEBFDF91CF911F91FF90EF90DF907D
:10ADB000CF90089580E00F94E011882361F08250D5
:10ADC000823030F580919B33882311F110929B33B0
:10ADD00010929A33089580919B33811119C081E0BC
:10ADE00080939B338EE292E0ECE9F3E3DF019C0178
:10ADF0001D9221503040E1F7BF0180E00F9493583D
:10AE00008B3019F410929A33089581E080939A332D
:10AE100008958AE00895CF93DF93CDB7DEB76097AA
:10AE2000CDBFDEBF009719F120E329832AE32A83EF
:10AE30002BE0E2E3F4E2DE01139601900D922A95F5
:10AE4000E1F7613041F441E0BE016F5F7F4F0F9445
:10AE5000B158982F07C04AE0BE016F5F7F4F0F9433
:10AE6000B158982F81E0992319F080E001C080E06B
:10AE70006096CDBFDEBFDF91CF910895DF92EF9254
:10AE8000FF920F931F93CF93DF93CDB7DEB76497F5
:10AE9000CDBFDEBF8C0184E1EDE3F4E2DE0111966B
:10AEA00001900D928A95E1F70115110509F449C049
:10AEB0006115710509F447C080E389838AE38A83B9
:10AEC0004115510559F0DA01FE0134969E01285FC3
:10AED0003F4F9D919193E217F307D9F77B010F2E16
:10AEE000F0E3DF2EF02D46E0BE016F5F7F4FC8011B
:10AEF0000F94B15899EF980F9230A8F49F85993329
:10AF000079F48E85893341F48D858933F1F08F5F33
:10AF10008D87DE86DF86E7CFDF868F5F8E87E3CF84
:10AF20009F5F9F87E0CF811112C081E1FE013396C0
:10AF3000D70101900D928A95E1F7F701118A81E01E
:10AF400007C080E005C080E003C080E001C080E071
:10AF50006496CDBFDEBFDF91CF911F910F91FF901F
:10AF6000EF90DF900895DF92EF92FF920F931F937F
:10AF7000CF93DF93CDB7DEB76497CDBFDEBF8C0133
:10AF800084E1E1E5F4E2DE01119601900D928A95EB
:10AF9000E1F70115110509F449C06115710509F4BE
:10AFA00047C080E389838AE38A834115510559F0BC
:10AFB000DA01FE0134969E01285F3F4F9D919193E7
:10AFC000E217F307D9F77B010F2EF0E3DF2EF02D08
:10AFD00046E0BE016F5F7F4FC8010F94B15899EFF3
:10AFE000980F9230A8F49F85993379F48E85893330
:10AFF00041F48D858933F1F08F5F8D87DE86DF86A2
:10B00000E7CFDF868F5F8E87E3CF9F5F9F87E0CF9D
:10B01000811112C081E1FE013396D70101900D929A
:10B020008A95E1F7F701118A81E007C080E005C049
:10B0300080E003C080E001C080E06496CDBFDEBF49
:10B04000DF91CF911F910F91FF90EF90DF900895C6
:10B050000F931F93CF93DF93CDB7DEB76097CDBF2C
:10B06000DEBF009761F18C0180E389838AE38A83E4
:10B070008BE0E5E6F4E2DE01139601900D928A95ED
:10B08000E1F7613049F441E0BE016F5F7F4FC801D5
:10B090000F94B158982F0EC041E060E0CE010396A6
:10B0A0000F94215F4AE0BE016F5F7F4FC8010F948C
:10B0B000B158982F81E0992319F080E001C080E019
:10B0C0006096CDBFDEBFDF91CF911F910F910895A4
:10B0D000CF93DF93CDB7DEB76097CDBFDEBF9BE0E8
:10B0E000E5E6F4E2DE01119601900D929A95E1F702
:10B0F000813041F441E061E0CE0101960F94215F7F
:10B10000982F07C041E060E0CE0101960F94215FC7
:10B11000982F81E0911180E06096CDBFDEBFDF9176
:10B12000CF910895009721F041E061E00D94215FF7
:10B1300008951F93CF93DF93CDB7DEB76497CDBF4C
:10B14000DEBF009701F1162FBC0180E389838AE3FB
:10B150008A83CE0103960F943A67113041F441E09F
:10B1600061E0CE0101960F94215F982F07C041E066
:10B1700060E0CE0101960F94215F982F81E0992322
:10B1800019F080E001C080E06496CDBFDEBFDF91A2
:10B19000CF911F910895EF92FF920F931F93CF933A
:10B1A000DF93CDB7DEB76497CDBFDEBF6115710504
:10B1B00089F1009789F18B017C0180E389838AE31F
:10B1C0008A83CE0103960F943A6743E0BE016F5F16
:10B1D0007F4FC7010F94B158873069F460E0C80110
:10B1E000A8DF982F8823D9F043E0BE016F5F7F4F1F
:10B1F000C7010F94B158811111C0F70142855385E1
:10B2000064857585C7010F944F5D91E0882339F0FF
:10B2100090E005C090E003C090E001C090E0892F6D
:10B220006496CDBFDEBFDF91CF911F910F91FF904C
:10B23000EF900895CF93DF93CDB7DEB76097CDBF82
:10B24000DEBF0097C1F020E329832AE32A832AE0A6
:10B25000E0E7F4E2DE01139601900D922A95E1F702
:10B2600041E0BE016F5F7F4F0F94B15891E088239A
:10B2700019F090E001C090E0892F6096CDBFDEBF4D
:10B28000DF91CF9108953F924F925F926F927F929C
:10B290008F929F92AF92BF92CF92DF92EF92FF92E6
:10B2A0000F931F93CF93DF93CDB7DEB76197CDBFD9
:10B2B000DEBF6115710509F470C0009709F46FC015
:10B2C0004115510509F46DC03FEF320F383008F0D9
:10B2D0006AC0322E7A018C01FB01138A41E00F947F
:10B2E000B158811162C0F801428553856485758526
:10B2F000483EF3E05F076105710508F458C0413B23
:10B3000084E058076105710508F053C0C32CD12CA7
:10B310005601E6E0AE0EB11C25010B2C000C6608B0
:10B3200077084419550966097709C8010F944F5DDC
:10B33000811141C0A50160E070E0CE0103960F9439
:10B3400033679E012F5F3F4FA501BE016D5F7F4FA9
:10B35000C8010F94035AC8010F94445DFE01EC0D1F
:10B36000FD1D12868E010D5F1F4F812C912C540103
:10B37000A601B801C7010F941D67892BF1F0FFEFFB
:10B380008F1A9F0AAF0ABF0A0F5F1F4F4814590454
:10B390006A047B0468F780E011C080E00FC080E0A1
:10B3A0000DC080E00BC080E009C080E007C081E0F4
:10B3B00005C080E003C080E001C081E06196CDBFA0
:10B3C000DEBFDF91CF911F910F91FF90EF90DF9043
:10B3D000CF90BF90AF909F908F907F906F905F9035
:10B3E0004F903F9008954F925F926F927F92AF92ED
:10B3F000BF92CF92DF92EF92FF920F931F93CF9362
:10B40000DF93CDB7DEB76897CDBFDEBF680114E12B
:10B41000EEE1F4E2DE01159601900D921A95E1F746
:10B42000009709F491C0C114D10409F48FC0EFEF63
:10B43000EE0DE83008F08CC0860129013A015B016D
:10B440006C01283E83E03807410551050CF482C0A9
:10B450001F921F921F9281E08F938EEE91E29F9335
:10B460008F93CE0101969F938F930F945867898194
:10B47000898B8A818A8B8B818B8B80E38D838AE396
:10B480008E83CDBFDEBFA114B10459F0D501FE01FA
:10B4900038969E01245F3F4F8D918193E217F30709
:10B4A000D9F70F2EF0E3FF2EF02D46E0BE016B5FC3
:10B4B0007F4F83EB90E40F94B15899EF980F92303F
:10B4C00090F52E2DA801BE016B5F7F4F83EB90E4BA
:10B4D000DADE882379F060E0C6012BDE882351F0A4
:10B4E0004AE0BE016B5F7F4F83EB90E40F94B1584D
:10B4F0008823F9F09B89993399F48A89893361F417
:10B500008989893321F410929A3380E042C08F5F99
:10B51000898BFA8AFB8AC9CFFB8A8F5F8A8BC5CF5A
:10B520009F5F9B8BC2CF882321F010929A3380E0DB
:10B5300030C081E080939A33BE01695F7F4FC601BE
:10B540000F943A6781E025C080E023C080E021C0ED
:10B5500080E01FC07F926F925F922F938EEE91E2F8
:10B560009F938F93CE0101969F938F930F9458676B
:10B570008981898B8A818A8B8B818B8B80E38D83F8
:10B580008AE38E83CDBFDEBFA114B10409F07ECF64
:10B5900088CF6896CDBFDEBFDF91CF911F910F910D
:10B5A000FF90EF90DF90CF90BF90AF907F906F9023
:10B5B0005F904F900895DF92EF92FF920F931F9349
:10B5C000CF93DF93CDB7DEB76497CDBFDEBF8C01DD
:10B5D00084E1EAE7F4E2DE01119601900D928A958A
:10B5E000E1F70115110509F449C06115710509F468
:10B5F00047C080E389838AE38A834115510559F066
:10B60000DA01FE0134969E01285F3F4F9D91919390
:10B61000E217F307D9F77B010F2EF0E3DF2EF02DB1
:10B6200046E0BE016F5F7F4FC8010F94B15899EF9C
:10B63000980F9230A8F49F85993379F48E858933D9
:10B6400041F48D858933F1F08F5F8D87DE86DF864B
:10B65000E7CFDF868F5F8E87E3CF9F5F9F87E0CF47
:10B66000811112C081E1FE013396D70101900D9244
:10B670008A95E1F7F701118A81E007C080E005C0F3
:10B6800080E003C080E001C080E06496CDBFDEBFF3
:10B69000DF91CF911F910F91FF90EF90DF90089570
:10B6A0008091CA3508950895089581E08093CA3540
:10B6B00008951092CA350895CF92DF92EF92FF92CB
:10B6C0000F931F936623B9F081111DC0C12CD12C9B
:10B6D000760100E010E62AEE30E040E06CE170E236
:10B6E00080EB98E00F9411456CE170E280EB98E0FC
:10B6F0000F945B4508C0811106C06CE170E280EBDD
:10B7000098E00F9471451F910F91FF90EF90DF909B
:10B71000CF900895CF93DF931F921F92CDB7DEB7DE
:10B720008091CB359091CC35A091CD35B091CE356F
:10B73000072E75E1B695A795979587957A95D1F7D8
:10B74000702D61E0B9DF87ED8A8341E050E0BE01F2
:10B750006E5F7F4F80EB98E00F942C4541E050E006
:10B76000BE016F5F7F4F80EB98E00F944345898166
:10B770008823A4F78091CB359091CC35A091CD351D
:10B78000B091CE35072E75E1B695A795979587951B
:10B790007A95D1F7702D60E08FDF0F900F90DF91D9
:10B7A000CF91089580EB98E00F94DA441092CF3552
:10B7B00081E008951F93CF93DF93CDB7DEB72C9729
:10B7C000CDBFDEBF6115710520E28207910508F04B
:10B7D000A1C0DC01CB018093CB359093CC35A093F5
:10B7E000CD35B093CE358091CF35811193DF109256
:10B7F000CF358091CB359091CC35A091CD35B0919E
:10B80000CE35072E75E1B695A795979587957A95CC
:10B81000D1F7702D61E050DF82ED8C8741E050E080
:10B82000BE01645F7F4F80EB98E00F942C458091C0
:10B83000CB359091CC35A091CD35B091CE35AC01C2
:10B84000BD01032E39E076956795579547953A9552
:10B85000D1F7302D032E3AE0440F551F661F771F96
:10B860003A95D1F7302D9170AA27BB27842B952BC1
:10B87000A62BB72B89839A83AB83BC838B818D8363
:10B8800041E050E0BE016B5F7F4F80EB98E00F948A
:10B890002C458A818E8341E050E0BE016A5F7F4F74
:10B8A00080EB98E00F942C4589818F8341E050E034
:10B8B000BE01695F7F4F80EB98E00F942C4515E542
:10B8C000188741E050E0BE01685F7F4F80EB98E051
:10B8D0000F942C45198741E050E0BE01675F7F4F10
:10B8E00080EB98E00F942C451A8741E050E0BE01B0
:10B8F000665F7F4F80EB98E00F942C451B8741E0FB
:10B9000050E0BE01655F7F4F80EB98E00F942C45BF
:10B9100081E001C080E02C96CDBFDEBFDF91CF91EA
:10B920001F910895052E59E0660F771F881F991FF4
:10B930005A95D1F7502D6115710520E282079105C6
:10B9400010F438CF089580E008958091CB35909120
:10B95000CC35A091CD35B091CE350097A105B1057C
:10B9600069F00197A109B109072E75E1B695A79570
:10B97000979587957A95D1F7702D01C080E060E0AA
:10B980009BDE1092CF350895CF93DF93CDB7DEB70E
:10B990002897CDBFDEBF6115710520E282079105B2
:10B9A00008F078C0DC01CB018093CB359093CC3587
:10B9B000A093CD35B093CE358091CF358111AADEDD
:10B9C0001092CF358091CB359091CC35A091CD356B
:10B9D000B091CE35072E75E1B695A79597958795C9
:10B9E0007A95D1F7702D61E067DE82E8888741E0C3
:10B9F00050E0BE01685F7F4F80EB98E00F942C45CC
:10BA00008091CB359091CC35A091CD35B091CE358C
:10BA1000AC01BD01032E39E07695679557954795A2
:10BA20003A95D1F7302D032E3AE0440F551F661F8B
:10BA3000771F3A95D1F7302D9170AA27BB27842B19
:10BA4000952BA62BB72B89839A83AB83BC838B81E1
:10BA50008D8341E050E0BE016B5F7F4F80EB98E04B
:10BA60000F942C458A818E8341E050E0BE016A5FCD
:10BA70007F4F80EB98E00F942C4589818F8341E0C4
:10BA800050E0BE01695F7F4F80EB98E00F942C453A
:10BA900081E001C080E02896CDBFDEBFDF91CF916D
:10BAA0000895CF93DF931F92CDB7DEB78091CB354A
:10BAB0009091CC35A091CD35B091CE35AC01BD0182
:10BAC000517066277727452B462B472B31F119827A
:10BAD00041E050E0BE016F5F7F4F80EB98E00F9434
:10BAE0002C458091CB359091CC35A091CD35B0913E
:10BAF000CE350196A11DB11D8093CB359093CC35E9
:10BB0000A093CD35B093CE35AC01BD015170662701
:10BB10007727452B462B472BD1F60097A105B1057A
:10BB200069F00197A109B109072E75E1B695A795AE
:10BB3000979587957A95D1F7702D01C080E060E0E8
:10BB4000BBDD81E08093CF350F90DF91CF910895D9
:10BB50000F931F93CF93DF931F92CDB7DEB78091E2
:10BB6000CF358823B1F01092CF358091CB359091AD
:10BB7000CC35A091CD35B091CE35BC01CD01052E8F
:10BB800059E096958795779567955A95D1F7502DF9
:10BB9000C9DE41E050E0BE016F5F7F4F80EB98E06F
:10BBA0000F9443458091CB359091CC35A091CD3504
:10BBB000B091CE35AC01BD014F5F5F4F6F4F7F4FEE
:10BBC0004093CB355093CC356093CD357093CE35C3
:10BBD0008A019B01117022273327012B022B032B93
:10BBE000A1F4452B462B472B51F0072E75E1B69556
:10BBF000A795979587957A95D1F7702D01C080E02C
:10BC000060E05ADD81E08093CF3589810F90DF912C
:10BC1000CF911F910F9108950F931F93CF93DF93AF
:10BC20001F92CDB7DEB7182F8091CF35882349F00A
:10BC30006091CB357091CC358091CD359091CE35DA
:10BC4000A3DE198341E050E0BE016F5F7F4F80EBC0
:10BC500098E00F942C458091CB359091CC35A091F4
:10BC6000CD35B091CE35AC01BD014F5F5F4F6F4F09
:10BC70007F4F4093CB355093CC356093CD35709347
:10BC8000CE358A019B01117022273327012B022B0D
:10BC9000032BA1F4452B462B472B51F0072E75E1C2
:10BCA000B695A795979587957A95D1F7702D01C090
:10BCB00080E060E001DD81E08093CF3581E00F908E
:10BCC000DF91CF911F910F910895CF93DF931F9232
:10BCD0001F92CDB7DEB78091CF35882309F440C0DD
:10BCE0008091CB359091CC35A091CD35B091CE35AA
:10BCF000072E75E1B695A795979587957A95D1F713
:10BD0000702D61E0D9DC87ED8A8341E050E0BE010F
:10BD10006E5F7F4F80EB98E00F942C4541E050E040
:10BD2000BE016F5F7F4F80EB98E00F944345809199
:10BD3000CB359091CC35A091CD35B091CE35072E35
:10BD400075E1B695A795979587957A95D1F7702D5A
:10BD500060E0B2DC89818095881F8827881F01C038
:10BD600080E00F900F90DF91CF910895CF93DF93F4
:10BD7000EC01803C28E0920729F468E083E00F940E
:10BD80005B4410C0803C29E0920729F468E084E01D
:10BD90000F945B4407C0803C9A4021F468E085E042
:10BDA0000F945B44888180618883DF91CF910895EF
:10BDB000EF92FF920F931F93CF937C01C42FB90191
:10BDC000A80100E010E62AEE30E00E940C6988230A
:10BDD00044F0F7018081CC0FCC0FCC70837FC82B4F
:10BDE000C083CF911F910F91FF90EF90089580E055
:10BDF000089591E0811101C090E09093D34081E0DB
:10BE00008093442008950F931F9307ED10E62FE1D0
:10BE100030E040E156E361E082E00E948F798111D9
:10BE200005C063E07FE582E00E94DF7A1F910F91F9
:10BE30000895CF93DF931092F3351092F4350F9459
:10BE40008745811104C010920C36D0E012C0815099
:10BE500080930C362ADCD82F882359F0C0E060E0AC
:10BE60008C2F0F949D45CF5F80910C368C17B8F7BF
:10BE7000CADF8D2FDF91CF910895C5CF08950F931D
:10BE80001F930DE31FE52DE030E048E450E260E051
:10BE900081E80E948F79811105C06FE37FE581E819
:10BEA0000E94DF7A1F910F9108958091F4358823C5
:10BEB00041F082E00E94B87A65E57FE582E00C946B
:10BEC000DF7A08958091F435882341F081E80E945B
:10BED000B87A62E67FE581E80C94DF7A0895809174
:10BEE000502090915120A0915220B0915320892B45
:10BEF0008A2B8B2B59F080911C36882324F481E8FF
:10BF00000E94B87A03C082E00E94B87A8091143609
:10BF100090911536A0911636B091173680934C202B
:10BF200090934D20A0934E20B0934F20A8CF08951A
:10BF3000E8EFF5E382E1DF011D928A95E9F780EFF2
:10BF400080838AE087830895DF92EF92FF920F93B8
:10BF50001F93CF93DF93D82EC62FD72F122F032FE7
:10BF6000F42EE52EE5DF81E080935420E8EFF5E341
:10BF7000D282E382F48205831683D487C587DF915A
:10BF8000CF911F910F91FF90EF90DF90089520E0E7
:10BF900030E0A90160E074E285E0D6CF08950F9308
:10BFA0001F9320911C3642276CF000915020109175
:10BFB000512020915220309153200617170728074F
:10BFC000390720F4E4DF8BDF80E001C081E01F91BE
:10BFD0000F91089520E030E0A90160E070E084E076
:10BFE000B3CF08950F931F93262F30E008E110E69A
:10BFF000AC0161E081E80E948F79811102C0EADF23
:10C000006EDF1F910F91089520E030E0A90160E0FC
:10C0100078E286E099CF089520E030E0A90160E061
:10C020007AE382E091CF089583DF1092542008953F
:10C03000CF93DF93811111C0EB01F6DFE8E4F0E26A
:10C0400080859185A285B3858C1B9D0BA109B109C3
:10C0500080879187A287B38742DFDF91CF910895D0
:10C060001F93CF93DF93D82F84E1E8EDF5E3DF0151
:10C070001D928A95E9F7DD2331F090912736E0EEA5
:10C08000F5E318E005C090912336ECEDF5E314E0FC
:10C09000809121368F738C3111F08F3339F48CE11C
:10C0A00080838AE0818385E08383145FC12F9117A9
:10C0B00008F4C92F8C2F90E0A0E0B0E040E8BC016C
:10C0C000CD016DDF882309F180911D360F94A445C1
:10C0D000811102C020E001C020E8DD2361F0E8ED1D
:10C0E000F5E3812F90E0029798278927982780838E
:10C0F0009183238306C0E8EDF5E38FEF810F808302
:10C1000022836C2F88ED95E36DDFDF91CF911F9136
:10C110000895CF93C82F81110FC080911D360F94C1
:10C12000A445882349F020E030E0A90160E077E2EF
:10C1300087E00ADFD4DE39C0AEEEB5E3E0E1F6E336
:10C14000818913968C931397828912968C931297F8
:10C15000838911968C93119784898C93ACEEB5E307
:10C16000868911968C93119787898C936091EC3511
:10C170007091ED35CB01A0E0B0E0BC01CD01052E02
:10C1800059E0660F771F881F991F5A95D1F7502DD8
:10C19000C11102C040E001C040E801DF882329F05E
:10C1A000C093F23581E08093F335CF9108950F93DA
:10C1B0001F93CF93DF93811132C16F31710569F401
:10C1C0008091103690911136A0911236B0911336AD
:10C1D00085359345A244B34431F081E08093F43532
:10C1E00064DE70DE1CC1E0E1F6E395859F70958703
:10C1F00080910C36891718F4CADE71DE10C1E0E1B7
:10C20000F6E34085518562857385409350205093B5
:10C2100051206093522070935320478550E04B3556
:10C22000510508F0EEC0FA018827E958FE4F8F4FFC
:10C230000D942B65C0912336C33108F0C2E18C2FD9
:10C2400090E0A0E0B0E040E8BC01CD01A8DE88238A
:10C2500009F4E5C06C2F88EF95E3C4DEE0C0C0911F
:10C260002336C53208F0C4E28C2F90E0A0E0B0E0A5
:10C2700040E8BC01CD0193DE882309F4D0C0809151
:10C280002036837021F4D0912136DD2319F07FDE32
:10C2900026DEC5C080911D360F94AB458111D0E8D4
:10C2A00000E210E2F801D18380911D360F94B2456F
:10C2B00020E1FC013196A0E3B0E201900D922A95B5
:10C2C000E1F7F8018089882309F4A4C0823209F4D7
:10C2D000A3C0E1E3F0E281E09191992309F49DC0CC
:10C2E000923209F49AC08F5F8031B1F708C0E82F0D
:10C2F000F0E0E05EFF4D908B8F5F8031C1F76C2FD7
:10C3000080E290E26FDE8BC080E0AADE88C081E030
:10C31000A7DE85C0892F0F948945823039F083309C
:10C3200019F0811105C006C06FDE05C075DE03C0BF
:10C3300051DE01C079DED3DD72C040E868E070E014
:10C3400080E090E02CDE882309F469C060ED75E39D
:10C3500080911D360F949045823041F0833019F062
:10C36000811107C009C050DEBADD59C055DEB7DD06
:10C3700056C030DEB4DD53C0E0EDF5E380E090E080
:10C38000A2E0B0E084839583A683B7838081918106
:10C39000A281B3815A2F4B2F60E070E09827892744
:10C3A0009827A0E0B0E0DC0199278827842B952B03
:10C3B000A62BB72B80839183A283B38368E0CF0140
:10C3C00011DE2DC08091233681FF06C08095682F35
:10C3D0006170892F0F949D4527DE81DD20C08091FB
:10C3E0002336811102C020DE01C0D1DD78DD17C007
:10C3F0001BDE75DD14C081E08CDE11C080E089DEBB
:10C400000EC020E030E0A90160E070E285E09CDD34
:10C4100066DD05C080E001C080E090E268CFDF917A
:10C42000CF911F910F9108951092F33542C908954D
:10C430008091DC408823F4F480768032D9F58091B5
:10C44000DD408E3FC9F58091E2409091E340019735
:10C45000A9F58091DE409091DF40892B89F5ECEDC4
:10C46000F0E48CE096E38087918781E090E082871A
:10C47000938708958076803229F58091DD408F3F43
:10C4800019F58091E2409091E340892BF9F4809175
:10C49000DE409091DF40892BD9F41092F435109250
:10C4A000F33582E00E944D7A81E80E944D7AABDC40
:10C4B00081E0089580E0089580E0089580E0089587
:10C4C00080E0089580E0089580E0089580E0089578
:10C4D00080E00895CF93C091F335CC23A9F1109259
:10C4E000F3358091F235882389F02091EC35309135
:10C4F000ED354091EE355091EF356091F03570910A
:10C50000F13580911D360F94BA4510C02091EC355D
:10C510003091ED354091EE355091EF356091F03529
:10C520007091F13580911D360F94DE45823041F0D7
:10C53000833021F0811106C077DD05C065DD03C0C1
:10C540006BDD01C047DDCBDC8C2FCF910895EF92DE
:10C55000FF920F931F93CF93DF93982F80914420E6
:10C56000882309F448C0109244202115310511F0A8
:10C57000890102C009EF1EE5911102C082E001C0ED
:10C5800081E8E9017A01AB01970160E00E948F79AF
:10C59000811104C091E0909344202DC0CD2BD9F49B
:10C5A000809144208823E1F38091D340811122C0FF
:10C5B000E8E4F0E280859185A285B3858E199F0914
:10C5C000A109B10980879187A287B3879091D34051
:10C5D00081E0892710C0E8E4F0E24085518562855A
:10C5E00073854E195F096109710940875187628718
:10C5F000738701C080E0DF91CF911F910F91FF9071
:10C60000EF900895E0913536F09136360190F08143
:10C61000E02D228133812E0F3F1FFC014081E40F6A
:10C62000F11DE217F307A0F481818430A1F0861395
:10C6300006C014C081818430A1F08617A9F08081E2
:10C64000E80FF11DE217F307A8F380E090E00895EA
:10C6500080E090E0089580E090E008958E2F9F2F75
:10C66000089580E090E008958E2F9F2F0895809187
:10C67000DE408F770C94AA780895909137369923ED
:10C6800081F1E0913536F09136360190F081E02D60
:10C690009481891740F5E0933336F0933436228144
:10C6A00033812E0F3F1FE217F307F8F49181943086
:10C6B00061F49281891309C09381961306C0E093B7
:10C6C0003336F093343681E008959081E90FF11DFF
:10C6D000E217F30758F3E0933336F093343680E0F3
:10C6E000089580E0089580E0089580E00895EF9235
:10C6F000FF921F93CF93DF93C82F60E0BEDF182F08
:10C70000882381F1A0913536B0913636EC2FF0E0D8
:10C71000EE0FFF1F12968D919C911397E80FF91F52
:10C72000E080F180D7011696ED91FC91179719954D
:10C73000682F8C2FA2DF182F8823A1F0C0913336E9
:10C74000D091343665E0CE015DDFEC01892B21F01C
:10C750008A810E949C7AF6CFD7011296ED91FC91C6
:10C7600013971995812FDF91CF911F91FF90EF9033
:10C7700008951F93CF93DF93182F7FDF882341F114
:10C78000C0913336D091343665E0CE013BDFEC0109
:10C79000892B49F04C815D816B818A810E94B77839
:10C7A0008111F2CF15C0A0913536B0913636E12F08
:10C7B000F0E0EE0FFF1F12968D919C911397E80FFA
:10C7C000F91F0190F081E02D0190F081E02D199585
:10C7D000DF91CF911F9108950C9442780895CF93E3
:10C7E000809137368823C1F0E0913536F0913636A6
:10C7F0000190F081E02D8481882371F0C0E08C2FBE
:10C8000076DFCF5FE0913536F09136360190F081DA
:10C81000E02D8481C81798F31092373681E090E0BC
:10C820008093383690933936CF9108950E940E78D0
:10C83000D6CF0895CF9380913736882349F1A091C0
:10C840003536B0913636ED91FC911197848188236D
:10C85000F9F0C0E0EC2FF0E0EE0FFF1F12968D9183
:10C860009C911397E80FF91F0190F081E02D00844F
:10C87000F185E02D309709F01995CF5FA0913536FD
:10C88000B0913636ED91FC9111978481C81710F361
:10C89000CF9108950F931F93CF93DF93ECEDF0E4C6
:10C8A000128613861486158616861786808188233D
:10C8B0000CF060C22091E2403091E3402115310537
:10C8C00009F05DC24FC28F7109F097C09091DD40B1
:10C8D000963081F0983009F485C091118EC02230D5
:10C8E000310509F0FBC162E070E088E396E30E9445
:10C8F000B0784EC28091DE409091DF40292F3327DF
:10C900002230310589F02330310579F121303105AC
:10C9100009F0A6C18091622090916320DC016C91A6
:10C9200070E00E94B0784FC0E0916220F0916320E7
:10C930002189821708F0D2C19927880F991F880F83
:10C94000991FE0916420F0916520E80FF91F808124
:10C950009181FC01628173810E94B078E091E44092
:10C96000F091E54082E081832EC0992781309105C6
:10C9700099F058F08230910509F406C2039709F046
:10C9800078C13CE0EEE8F4E20AC064E070E088ECD4
:10C9900090E20E94B07817C0EEEBF0E239E0A2EA34
:10C9A000B0E220E0819190E08D939D932F5F23175B
:10C9B000C8F3632F660F6E5F6093A02070E080EA7B
:10C9C00090E20E94B078ECEDF0E4868197812285B8
:10C9D00033858217930708F0DBC18093E64090937C
:10C9E000E740D6C12130310509F078C161E070E03F
:10C9F00087E396E30E94B078CBC18130E9F590914E
:10CA0000DD409A30C9F52130310509F037C18091F8
:10CA10003736882309F432C1C091E040D091E1401B
:10CA20000091353610913636D801ED91FC91848114
:10CA3000C81708F023C160E08C2F1FDE882309F49B
:10CA400018C1CE019927880F991FD8011296ED9130
:10CA5000FC911397E80FF91F0190F081E02D86817A
:10CA60009781FC0119958093323661E070E082E392
:10CA700096E30E94B0788CC1823009F0FAC08091B0
:10CA8000DD408111EFC02230310509F027C18091CE
:10CA9000E0400E943F7990E08093303690933136A9
:10CAA00062E070E080E396E30E94B07871C18F711C
:10CAB00009F084C09091DD40933009F4D5C018F49A
:10CAC0009130A1F07BC0953019F0993039F176C0E2
:10CAD0008091E2409091E340892B09F0FFC087E309
:10CAE00093E68093E8409093E94052C18091E24000
:10CAF0009091E340892B09F0F1C08091DE40909144
:10CB0000DF40019709F0EAC08091383690913936BC
:10CB10008D7F80933836909339363AC18091E240C8
:10CB20009091E340892B09F0D9C00E94AD78882309
:10CB300009F49FC02091DE403091DF403327E0911F
:10CB40006220F0916320818990E08217930708F4B6
:10CB500090C045DE8091DE409091DF408093373673
:10CB6000882309F415C199278150904C880F991F8B
:10CB7000880F991FE0916420F0916520E80FF91F5C
:10CB8000E0933536F09336360190F081E02D8481C4
:10CB9000882309F4FDC0C0E060E08C2FEADD882323
:10CBA00009F467C0CF5FE0913536F09136360190D9
:10CBB000F081E02D8481C81778F3EAC08130E9F470
:10CBC0009091DD409B30C9F48091E2409091E34028
:10CBD000892B09F053C080913736882309F44EC061
:10CBE000ECEDF0E4C481D2818C2F81DD882309F43F
:10CBF00040C06D2F8C2FBDDD3AC08230D1F58091C1
:10CC0000DD40813019F08330A1F030C08091E240E6
:10CC10009091E340892B09F061C08091DE409091B2
:10CC2000DF40892B09F05AC08091E0400E945A7978
:10CC30001EC08091E2409091E340892B09F04EC0E4
:10CC40008091DE409091DF40892B09F047C0CCED08
:10CC5000D0E48C810E944D7A8C810E94B87A07C002
:10CC600080E005C080E003C080E001C080E0811169
:10CC700090C08091DC408F71813081F58091373692
:10CC8000882309F471C00091E0401091E140C09107
:10CC90003536D0913636E881F9818481081708F05D
:10CCA00065C060E0802FE9DC8823C1F0F801FF2730
:10CCB000CF01880F991FEA81FB81E80FF91FC0811E
:10CCC000D181EE81FF811995682F802FD6DC8823D2
:10CCD00029F0EC81FD81199581115BC08091DC40C8
:10CCE0008F71823009F044C0809137368823B1F1CA
:10CCF000A0913536B0913636ED91FC911197848133
:10CD0000882371F1C0E0EC2FF0E0EE0FFF1F1296C8
:10CD10008D919C911397E80FF91F00811181D80123
:10CD20001696ED91FC9117971995682F8C2FA5DC1D
:10CD3000882379F1D8011496ED91FC9115971995F6
:10CD4000811127C0CF5FA0913536B0913636ED9175
:10CD5000FC9111979481C917B0F21BC080E019C0F3
:10CD600080E017C080E015C080E013C080E011C0F3
:10CD700080E00FC0982F907609F07BCF98CE982F47
:10CD8000907609F076CF9FCD33E0EAEBF0E207CE64
:10CD900081E0DF91CF911F910F9108958038910527
:10CDA00058F1672B21F4873C910571F41CC08F3F2B
:10CDB000910509F0F8F49C01220F331FF901E55A9F
:10CDC000F84D808191810895EDE5F8E221E030E0B1
:10CDD000419151918417950741F02F5F3F4F2038C3
:10CDE0003105B1F702C020E030E020583F4FC901C3
:10CDF0009927089580E090E008958136910589F0A3
:10CE0000EDE7F6E240E050E04F5F5F4F2191319156
:10CE10002115310591F028173907B1F7892B19F43D
:10CE20000AC040E050E0440F551FFA01E556FB4DA3
:10CE300080819181089580E090E0089543E050E082
:10CE400060E880E096E00F94B34443E050E064E093
:10CE500080E296E00F94B34443E050E062E080E269
:10CE600096E00F94B34440E058E160E280EA96E037
:10CE70000F94B34441E050E062E080EA96E00F9402
:10CE8000B34443E050E060E180E896E00F94B3449F
:10CE900043E050E060E180E496E00F94B34441E069
:10CEA00050E061E080E496E00F94B34441E050E04C
:10CEB00062E080E496E00F94B34441E050E060E229
:10CEC00080E696E00F94B34441E050E062E080E0F9
:10CED00096E00F94B34443E050E062E080E696E0D1
:10CEE0000F94B34440E050E061E080EA96E00F9494
:10CEF000B34440E050E061E080E096E00F94B3443A
:10CF000040E050E068E080E096E00F94B34441E0F8
:10CF100050E060E480E096E00F94B34440E058E1D4
:10CF200061E080E896E00F94B34440E050E061E0B7
:10CF300080E096E00F94B34440E050E060E280E08F
:10CF400096E00F94B34440E050E064E080E096E067
:10CF50000F94B34440E050E061E080EA96E00F9423
:10CF6000B34443E050E060E880E496E00F94B344BB
:10CF700043E050E060E280E496E00F94B34440E088
:10CF800050E060E480E496E00F94B34441E050E068
:10CF900060E880E896E00F94B34441E050E060E23E
:10CFA00080E896E00F94B34440E050E060E480E80D
:10CFB00096E00F94B34443E050E068E080E496E0EC
:10CFC0000F94B34440E050E064E080E496E00F94B6
:10CFD000B34443E050E068E080E696E00F94B34449
:10CFE00040E050E064E080E696E00F94B34443E014
:10CFF00050E068E080E896E00F94B34440E050E0F1
:10D0000064E080E896E00F94B34443E050E068E0C9
:10D0100080EA96E00F94B34440E050E064E080EA98
:10D0200096E00F94B34440E058E160E480EA96E073
:10D030000F94B34440E058E160E180E696E00F943D
:10D04000B34440E058E161E080E296E00F94B344DD
:10D0500043E050E060E880E496E00F94B34443E09E
:10D0600050E060E280E496E00F94B34440E050E08A
:10D0700060E480E496E00F94B34443E050E060E85D
:10D0800080EA96E00F94B34443E050E060E880E427
:10D0900096E00F94B34443E050E060E280E496E011
:10D0A0000F94B34440E050E060E480E496E00F94D5
:10D0B000B34443E050E068E080E296E00F94B3446C
:10D0C00041E050E062E080E896E00F94B34440E035
:10D0D00050E061E080E696E00F94B34440E050E019
:10D0E00060E180E096E00D94B34408951F920F92A2
:10D0F0000FB60F9211240BB60F928F939F93EF935D
:10D10000FF93E4EDF0E48081918101968083918327
:10D11000FF91EF919F918F910F900BBE0F900FBEDB
:10D120000F901F9018951F920F920FB60F92112417
:10D130000BB60F92CF92DF92EF92FF920F931F9355
:10D140002F933F934F935F936F937F938F939F930F
:10D15000AF93BF93EF93FF93E4EDF0E4808191816F
:10D160002281338182179307F0F121E0209302049A
:10D17000E091DA40F091DB403097A9F1609108042A
:10D1800070910904A0E0B0E0DC0199278827AB0189
:10D1900060E070E08C019D01042B152B262B372BB2
:10D1A000C901B801A4EDB0E412960D911C9113973A
:10D1B00020E030E09801112700271496CD90DC90F4
:10D1C0001597E12CF12C0C291D292E293F29061732
:10D1D00017072807390730F0C901B8016F5F7F4F83
:10D1E0008F4F9F4F1995FF91EF91BF91AF919F91F5
:10D1F0008F917F916F915F914F913F912F911F91EF
:10D200000F91FF90EF90DF90CF900F900BBE0F909B
:10D210000FBE0F901F901895CF92DF92EF92FF9262
:10D220000F931F93CF93DF93EC016A017B01DB0126
:10D23000CA010197A109B109BC01CD01600F711F9D
:10D24000821F931FA70196010F94ED6421383105C9
:10D2500041055105F8F4213460F4213260F42131A4
:10D2600060F4293060F4253060F4233060F490E8F5
:10D270000BC093E009C092E007C092E805C091E0BE
:10D2800003C091E801C090E088818C77892B888366
:10D2900081E001C08FEFDF91CF911F910F91FF903F
:10D2A000EF90DF90CF9008951F920F920FB60F92DC
:10D2B00011240BB60F922F933F934F935F936F936D
:10D2C0007F938F939F93AF93BF93EF93FF93E091DF
:10D2D0008036F0918136309709F01995FF91EF91E2
:10D2E000BF91AF919F918F917F916F915F914F917E
:10D2F0003F912F910F900BBE0F900FBE0F901F907C
:10D3000018951F920F920FB60F9211240BB60F9221
:10D310002F933F934F935F936F937F938F939F933D
:10D32000AF93BF93EF93FF93E0917E36F0917F36FA
:10D33000309709F01995FF91EF91BF91AF919F91AF
:10D340008F917F916F915F914F913F912F910F90AE
:10D350000BBE0F900FBE0F901F9018951F920F924B
:10D360000FB60F9211240BB60F922F933F934F934A
:10D370005F936F937F938F939F93AF93BF93EF933D
:10D38000FF93E0917C36F0917D36309709F0199546
:10D39000FF91EF91BF91AF919F918F917F916F918D
:10D3A0005F914F913F912F910F900BBE0F900FBE49
:10D3B0000F901F9018951F920F920FB60F92112485
:10D3C0000BB60F922F933F934F935F936F937F937F
:10D3D0008F939F93AF93BF93EF93FF93E0917A3630
:10D3E000F0917B36309709F01995FF91EF91BF913D
:10D3F000AF919F918F917F916F915F914F913F91ED
:10D400002F910F900BBE0F900FBE0F901F9018958D
:10D410001F920F920FB60F9211240BB60F922F93FB
:10D420003F934F935F936F937F938F939F93AF93AC
:10D43000BF93EF93FF93E0917836F0917936309770
:10D4400009F01995FF91EF91BF91AF919F918F9145
:10D450007F916F915F914F913F912F910F900BBEF4
:10D460000F900FBE0F901F9018951F920F920FB63E
:10D470000F9211240BB60F922F933F934F935F930C
:10D480006F937F938F939F93AF93BF93EF93FF938C
:10D49000E0917636F0917736309709F01995FF9143
:10D4A000EF91BF91AF919F918F917F916F915F911C
:10D4B0004F913F912F910F900BBE0F900FBE0F9089
:10D4C0001F9018951F920F920FB60F9211240BB652
:10D4D0000F922F933F934F935F936F937F938F930D
:10D4E0009F93AF93BF93EF93FF93E0917436F091C6
:10D4F0007536309709F01995FF91EF91BF91AF9173
:10D500009F918F917F916F915F914F913F912F915B
:10D510000F900BBE0F900FBE0F901F9018951F928B
:10D520000F920FB60F9211240BB60F922F933F93C9
:10D530004F935F936F937F938F939F93AF93BF931B
:10D54000EF93FF93E0917236F0917336309709F0C4
:10D550001995FF91EF91BF91AF919F918F917F911D
:10D560006F915F914F913F912F910F900BBE0F9054
:10D570000FBE0F901F9018951F920F920FB60F922B
:10D5800011240BB60F922F933F934F935F936F939A
:10D590007F938F939F93AF93BF93EF93FF93E0910C
:10D5A0007036F0917136309709F01995FF91EF912F
:10D5B000BF91AF919F918F917F916F915F914F91AB
:10D5C0003F912F910F900BBE0F900FBE0F901F90A9
:10D5D00018951F920F920FB60F9211240BB60F924F
:10D5E0002F933F934F935F936F937F938F939F936B
:10D5F000AF93BF93EF93FF93E0916E36F0916F3648
:10D60000309709F01995FF91EF91BF91AF919F91DC
:10D610008F917F916F915F914F913F912F910F90DB
:10D620000BBE0F900FBE0F901F9018951F920F9278
:10D630000FB60F9211240BB60F922F933F934F9377
:10D640005F936F937F938F939F93AF93BF93EF936A
:10D65000FF93E0916C36F0916D36309709F0199593
:10D66000FF91EF91BF91AF919F918F917F916F91BA
:10D670005F914F913F912F910F900BBE0F900FBE76
:10D680000F901F9018951F920F920FB60F921124B2
:10D690000BB60F922F933F934F935F936F937F93AC
:10D6A0008F939F93AF93BF93EF93FF93E0916A366D
:10D6B000F0916B36309709F01995FF91EF91BF917A
:10D6C000AF919F918F917F916F915F914F913F911A
:10D6D0002F910F900BBE0F900FBE0F901F901895BB
:10D6E0001F920F920FB60F9211240BB60F922F9329
:10D6F0003F934F935F936F937F938F939F93AF93DA
:10D70000BF93EF93FF93E0916836F09169363097BD
:10D7100009F01995FF91EF91BF91AF919F918F9172
:10D720007F916F915F914F913F912F910F900BBE21
:10D730000F900FBE0F901F9018951F920F920FB66B
:10D740000F9211240BB60F922F933F934F935F9339
:10D750006F937F938F939F93AF93BF93EF93FF93B9
:10D76000E0916636F0916736309709F01995FF9190
:10D77000EF91BF91AF919F918F917F916F915F9149
:10D780004F913F912F910F900BBE0F900FBE0F90B6
:10D790001F9018951F920F920FB60F9211240BB67F
:10D7A0000F922F933F934F935F936F937F938F933A
:10D7B0009F93AF93BF93EF93FF93E0916436F09103
:10D7C0006536309709F01995FF91EF91BF91AF91B0
:10D7D0009F918F917F916F915F914F913F912F9189
:10D7E0000F900BBE0F900FBE0F901F9018951F92B9
:10D7F0000F920FB60F9211240BB60F922F933F93F7
:10D800004F935F936F937F938F939F93AF93BF9348
:10D81000EF93FF93E0916236F0916336309709F011
:10D820001995FF91EF91BF91AF919F918F917F914A
:10D830006F915F914F913F912F910F900BBE0F9081
:10D840000FBE0F901F9018951F920F920FB60F9258
:10D8500011240BB60F922F933F934F935F936F93C7
:10D860007F938F939F93AF93BF93EF93FF93E09139
:10D870006036F0916136309709F01995FF91EF917C
:10D88000BF91AF919F918F917F916F915F914F91D8
:10D890003F912F910F900BBE0F900FBE0F901F90D6
:10D8A00018951F920F920FB60F9211240BB60F927C
:10D8B0002F933F934F935F936F937F938F939F9398
:10D8C000AF93BF93EF93FF93E0915E36F0915F3695
:10D8D000309709F01995FF91EF91BF91AF919F910A
:10D8E0008F917F916F915F914F913F912F910F9009
:10D8F0000BBE0F900FBE0F901F9018951F920F92A6
:10D900000FB60F9211240BB60F922F933F934F93A4
:10D910005F936F937F938F939F93AF93BF93EF9397
:10D92000FF93E0915C36F0915D36309709F01995E0
:10D93000FF91EF91BF91AF919F918F917F916F91E7
:10D940005F914F913F912F910F900BBE0F900FBEA3
:10D950000F901F9018951F920F920FB60F921124DF
:10D960000BB60F922F933F934F935F936F937F93D9
:10D970008F939F93AF93BF93EF93FF93E0915A36AA
:10D98000F0915B36309709F01995FF91EF91BF91B7
:10D99000AF919F918F917F916F915F914F913F9147
:10D9A0002F910F900BBE0F900FBE0F901F901895E8
:10D9B0001F920F920FB60F9211240BB60F922F9356
:10D9C0003F934F935F936F937F938F939F93AF9307
:10D9D000BF93EF93FF93E0915836F091593630970B
:10D9E00009F01995FF91EF91BF91AF919F918F91A0
:10D9F0007F916F915F914F913F912F910F900BBE4F
:10DA00000F900FBE0F901F9018951F920F920FB698
:10DA10000F9211240BB60F922F933F934F935F9366
:10DA20006F937F938F939F93AF93BF93EF93FF93E6
:10DA3000E0915636F0915736309709F01995FF91DD
:10DA4000EF91BF91AF919F918F917F916F915F9176
:10DA50004F913F912F910F900BBE0F900FBE0F90E3
:10DA60001F9018951F920F920FB60F9211240BB6AC
:10DA70000F922F933F934F935F936F937F938F9367
:10DA80009F93AF93BF93EF93FF93E0915436F09140
:10DA90005536309709F01995FF91EF91BF91AF91ED
:10DAA0009F918F917F916F915F914F913F912F91B6
:10DAB0000F900BBE0F900FBE0F901F9018951F92E6
:10DAC0000F920FB60F9211240BB60F922F933F9324
:10DAD0004F935F936F937F938F939F93AF93BF9376
:10DAE000EF93FF93E0915236F0915336309709F05F
:10DAF0001995FF91EF91BF91AF919F918F917F9178
:10DB00006F915F914F913F912F910F900BBE0F90AE
:10DB10000FBE0F901F9018951F920F920FB60F9285
:10DB200011240BB60F922F933F934F935F936F93F4
:10DB30007F938F939F93AF93BF93EF93FF93E09166
:10DB40005036F0915136309709F01995FF91EF91C9
:10DB5000BF91AF919F918F917F916F915F914F9105
:10DB60003F912F910F900BBE0F900FBE0F901F9003
:10DB700018951F920F920FB60F9211240BB60F92A9
:10DB80002F933F934F935F936F937F938F939F93C5
:10DB9000AF93BF93EF93FF93E0914E36F0914F36E2
:10DBA000309709F01995FF91EF91BF91AF919F9137
:10DBB0008F917F916F915F914F913F912F910F9036
:10DBC0000BBE0F900FBE0F901F9018951F920F92D3
:10DBD0000FB60F9211240BB60F922F933F934F93D2
:10DBE0005F936F937F938F939F93AF93BF93EF93C5
:10DBF000FF93E0914C36F0914D36309709F019952E
:10DC0000FF91EF91BF91AF919F918F917F916F9114
:10DC10005F914F913F912F910F900BBE0F900FBED0
:10DC20000F901F9018951F920F920FB60F9211240C
:10DC30000BB60F922F933F934F935F936F937F9306
:10DC40008F939F93AF93BF93EF93FF93E0914A36E7
:10DC5000F0914B36309709F01995FF91EF91BF91F4
:10DC6000AF919F918F917F916F915F914F913F9174
:10DC70002F910F900BBE0F900FBE0F901F90189515
:10DC80001F920F920FB60F9211240BB60F922F9383
:10DC90003F934F935F936F937F938F939F93AF9334
:10DCA000BF93EF93FF93E0914836F0914936309758
:10DCB00009F01995FF91EF91BF91AF919F918F91CD
:10DCC0007F916F915F914F913F912F910F900BBE7C
:10DCD0000F900FBE0F901F9018951F920F920FB6C6
:10DCE0000F9211240BB60F922F933F934F935F9394
:10DCF0006F937F938F939F93AF93BF93EF93FF9314
:10DD0000E0914636F0914736309709F01995FF912A
:10DD1000EF91BF91AF919F918F917F916F915F91A3
:10DD20004F913F912F910F900BBE0F900FBE0F9010
:10DD30001F9018951F920F920FB60F9211240BB6D9
:10DD40000F922F933F934F935F936F937F938F9394
:10DD50009F93AF93BF93EF93FF93E0914436F0917D
:10DD60004536309709F01995FF91EF91BF91AF912A
:10DD70009F918F917F916F915F914F913F912F91E3
:10DD80000F900BBE0F900FBE0F901F9018951F9213
:10DD90000F920FB60F9211240BB60F922F933F9351
:10DDA0004F935F936F937F938F939F93AF93BF93A3
:10DDB000EF93FF93E0914236F0914336309709F0AC
:10DDC0001995FF91EF91BF91AF919F918F917F91A5
:10DDD0006F915F914F913F912F910F900BBE0F90DC
:10DDE0000FBE0F901F9018951F920F920FB60F92B3
:10DDF00011240BB60F922F933F934F935F936F9322
:10DE00007F938F939F93AF93BF93EF93FF93E09193
:10DE10004036F0914136309709F01995FF91EF9116
:10DE2000BF91AF919F918F917F916F915F914F9132
:10DE30003F912F910F900BBE0F900FBE0F901F9030
:10DE400018951F920F920FB60F9211240BB60F92D6
:10DE50002F933F934F935F936F937F938F939F93F2
:10DE6000AF93BF93EF93FF93E0913E36F0913F362F
:10DE7000309709F01995FF91EF91BF91AF919F9164
:10DE80008F917F916F915F914F913F912F910F9063
:10DE90000BBE0F900FBE0F901F9018951F920F9200
:10DEA0000FB60F9211240BB60F922F933F934F93FF
:10DEB0005F936F937F938F939F93AF93BF93EF93F2
:10DEC000FF93E0913C36F0913D36309709F019957B
:10DED000FF91EF91BF91AF919F918F917F916F9142
:10DEE0005F914F913F912F910F900BBE0F900FBEFE
:10DEF0000F901F9018951F920F920FB60F9211243A
:10DF00000BB60F922F933F934F935F936F937F9333
:10DF10008F939F93AF93BF93EF93FF93E0913A3624
:10DF2000F0913B36309709F01995FF91EF91BF9131
:10DF3000AF919F918F917F916F915F914F913F91A1
:10DF40002F910F900BBE0F900FBE0F901F90189542
:10DF5000CF93CFB7F894282F392F211588E03807B1
:10DF600049F461E083E00F945B4464E083E00F9444
:10DF70005B444FC0203488E0380749F462E083E016
:10DF80000F945B4464E083E00F945B4442C021152E
:10DF900089E0380749F461E084E00F945B4464E071
:10DFA00084E00F945B4435C0203489E0380749F49D
:10DFB00062E084E00F945B4464E084E00F945B448F
:10DFC00028C021158AE0380749F461E085E00F9404
:10DFD0005B4464E085E00F945B441BC020348AE01E
:10DFE000380749F462E085E00F945B4464E085E023
:10DFF0000F945B440EC021153B4049F461E086E07C
:10E000000F945B4464E086E00F945B4402C0CFBF92
:10E0100001C0CFBFCF910895CF93CFB7F894282FE9
:10E02000392F211588E0380749F461E083E00F9427
:10E03000674464E083E00F9467444FC0203488E075
:10E04000380749F462E083E00F94674464E083E0BA
:10E050000F94674442C0211589E0380749F461E014
:10E0600084E00F94674464E084E00F94674435C013
:10E07000203489E0380749F462E084E00F94674473
:10E0800064E084E00F94674428C021158AE03807D3
:10E0900049F461E085E00F94674464E085E00F9403
:10E0A00067441BC020348AE0380749F462E085E009
:10E0B0000F94674464E085E00F9467440EC0211517
:10E0C0003B4049F461E086E00F94674464E086E0F9
:10E0D0000F94674402C0CFBF01C0CFBFCF91089556
:10E0E000811528E0920729F4609380367093813679
:10E0F0000895803428E0920729F460937436709371
:10E1000075360895811529E0920729F460936C36DD
:10E1100070936D360895803429E0920729F4609356
:10E12000603670936136089581152AE0920729F4CC
:10E130006093583670935936089580342AE09207D8
:10E1400029F460934C3670934D36089581159B40A9
:10E1500021F460934436709345360895FC01918113
:10E1600095FFFDCF608380E090E008954F925F922D
:10E170006F927F928F929F92AF92BF92EF92FF9297
:10E180000F931F93CF937C014A015B012801390152
:10E19000FC01848182FF16C0D901C801689412F87D
:10E1A000B695A795979587951694D1F7B901A801CB
:10E1B000032E36E176956795579547953A95D1F7B1
:10E1C000302D15C0D901C801689413F8B695A795EC
:10E1D000979587951694D1F7B901A801032E37E1D9
:10E1E00076956795579547953A95D1F7302D8815CF
:10E1F0009905AA05BB0508F4A6C084169506A606CF
:10E20000B70608F4A2C0F701848182FD04C0880C1F
:10E21000991CAA1CBB1CC301B201A50194010F9457
:10E22000ED642F3F31054105510508F490C08FEF93
:10E2300090E0A0E0B0E0C9EF05C0281739074A0711
:10E240005B0758F0880F991FAA1FBB1FCD3F0CF426
:10E250008160CF5FC73089F74FC0CC230CF04CC032
:10E26000D501C401880F991FAA1FBB1F880F991FD2
:10E27000AA1FBB1F880F991FAA1FBB1F481A590A44
:10E280006A0A7B0ACE3FF4F48DEF9FEF8C1B910955
:10E29000C7FD939504C0440C551C661C771C8A95D9
:10E2A000D2F7D501C401B695A79597958795BC017E
:10E2B000CD01640D751D861D971DA50194010F9458
:10E2C000ED6437C083E08C0FA501940104C0220FD8
:10E2D000331F441F551F8A95D2F7DA01C901B6953D
:10E2E000A79597958795BC01CD01640D751D861D79
:10E2F000971D0F94ED641DC083E08C0FA501940160
:10E3000004C0220F331F441F551F8A95D2F7DA012C
:10E31000C901B695A79597958795BC01CD01640D68
:10E32000751D861D971D0F94ED642150310941091B
:10E330005109832F8F70C295C07FC82BF701C78307
:10E34000268381E018C080E016C080E014C0D501AB
:10E35000C401880F991FAA1FBB1F880F991FAA1FEE
:10E36000BB1F880F991FAA1FBB1F481A590A6A0AA8
:10E370007B0AC9EF89CFCF911F910F91FF90EF904A
:10E38000BF90AF909F908F907F906F905F904F90D5
:10E3900008950F931F93CF93DF93EC018B010097A8
:10E3A00009F41EC1803C910529F460E180E00F94DE
:10E3B0005B4416C1C11584E0D80729F464E080E00D
:10E3C0000F945B440DC1C038E1E0DE0729F462E040
:10E3D00080E00F945B4404C1C115F1E0DF0729F42C
:10E3E00061E080E00F945B44FBC0C03883E0D80755
:10E3F00029F461E081E00F945B44F2C0C039E3E0AE
:10E40000DE0729F461E082E00F945B44E9C0C115A6
:10E41000F2E0DF0729F462E081E00F945B44E0C0A2
:10E42000C03482E0D80729F462E082E00F945B44B4
:10E43000D7C0C032E3E0DE0729F464E082E00F9445
:10E440005B44CEC0C115F8E0DF0729F461E083E04A
:10E450000F945B44C5C0C11589E0D80729F461E079
:10E4600084E00F945B44BCC0C115EAE0DE0729F4E8
:10E4700061E085E00F945B44B3C0C115FBE0DF07AA
:10E4800029F461E086E00F945B44AAC0C03488E0C0
:10E49000D80729F462E083E00F945B44A1C0C03444
:10E4A000E9E0DE0729F462E084E00F945B4498C061
:10E4B000C034FAE0DF0729F462E085E00F945B44A2
:10E4C0008FC0C03988E0D80729F464E083E00F9456
:10E4D0005B4486C0C039E9E0DE0729F464E084E0EB
:10E4E0000F945B447DC0C039FAE0DF0729F464E093
:10E4F00085E00F945B4474C0C0398BE0D80729F4E1
:10E5000064E086E00F945B446BC0C03CE8E0DE074B
:10E5100029F468E083E00F945B4462C0C03CF9E0FA
:10E52000DF0729F468E084E00F945B4459C0C03CE5
:10E530008AE0D80729F468E085E00F945B4450C076
:10E54000C03AE8E0DE0729F460E183E00F945B4421
:10E5500047C0C03AF9E0DF0729F460E184E00F9496
:10E560005B443EC0C03A8AE0D80729F460E185E008
:10E570000F945B4435C0C03AEBE0DE0729F460E15C
:10E5800086E00F945B442CC0C03BF8E0DF0729F421
:10E5900060E283E00F945B4423C0C03B89E0D8076E
:10E5A00029F460E284E00F945B441AC0C03BEAE0C7
:10E5B000DE0729F460E285E00F945B4411C0C038A7
:10E5C000F4E0DF0729F460E483E00F945B4408C0C3
:10E5D000C03A84E0D80721F460E485E00F945B44FE
:10E5E0008D818F738D83F80195818481892B96812C
:10E5F000911198E0892B8D83F801408151816281CE
:10E60000738100E010E62AEE30E0CE01AFDD9C81A0
:10E6100098609C839C8190619C83DF91CF911F9136
:10E620000F910895CF92DF92EF92FF920F931F9375
:10E63000CF93DF93EC01D901C801B695A7959795C3
:10E640008795481759076A077B0778F46A017B01A9
:10E65000CC0CDD1CEE1CFF1CC901B801A701960102
:10E660000F94ED642150310902C020E030E0832F87
:10E670008F708F832E83DF91CF911F910F91FF9029
:10E68000EF90DF90CF900895EF92FF920F931F933A
:10E69000CF93DF93EC017B01009709F4B9C1803C73
:10E6A000910529F460E180E00F945B44B1C18115CC
:10E6B000944029F464E080E00F945B44A9C1C03821
:10E6C00081E0D80729F462E080E00F945B44A0C1A8
:10E6D000C115E1E0DE0729F461E080E00F945B44BE
:10E6E00097C1C038F3E0DF0729F461E081E00F94BF
:10E6F0005B448EC1C03933E0D30729F461E082E086
:10E700000F945B4485C1C11582E0D80729F462E00B
:10E7100081E00F945B447CC1C034E2E0DE0729F461
:10E7200062E082E00F945B4473C1C032F3E0DF0724
:10E7300029F464E082E00F945B446AC1C11538E0BB
:10E74000D30729F461E083E00F945B4461C1C115F4
:10E7500089E0D80729F461E084E00F945B4458C154
:10E76000C115EAE0DE0729F461E085E00F945B441F
:10E770004FC1C115FBE0DF0729F461E086E00F948B
:10E780005B4446C1C03438E0D30729F462E083E03B
:10E790000F945B443DC1C03489E0D80729F462E09E
:10E7A00084E00F945B4434C1C034EAE0DE0729F40E
:10E7B00062E085E00F945B442BC1C039F8E0DF07CD
:10E7C00029F464E083E00F945B4422C1C03939E04E
:10E7D000D30729F464E084E00F945B4419C1C03985
:10E7E0008AE0D80729F464E085E00F945B4410C107
:10E7F000C039EBE0DE0729F464E086E00F945B4467
:10E8000007C1C03CF8E0DF0729F468E083E00F941B
:10E810005B44FEC0C03C39E0D30729F468E084E0E3
:10E820000F945B44F5C0C03C8AE0D80729F468E047
:10E8300085E00F945B44ECC0C03AE8E0DE0769F481
:10E8400060E183E00F945B44E0EAF8E084818F7E2E
:10E850008483F7012481225053C0C03AF9E0DF07D6
:10E8600029F460E184E00F945B44D2C0C03A3AE0FE
:10E87000D30729F460E185E00F945B44C9C0C03A36
:10E880008BE0D80729F460E186E00F945B44C0C0B8
:10E89000C03BE8E0DE0729F460E283E00F945B44CC
:10E8A000B7C0C03BF9E0DF0729F460E284E00F94D1
:10E8B0005B44AEC0C03B3AE0D30729F460E285E098
:10E8C0000F945B44A5C0C03884E0D80729F460E405
:10E8D00083E00F945B449CC0C03AE4E0DE0729F477
:10E8E00060E485E00F945B4493C08C818F7E8C83C1
:10E8F000FB0124812250CE01C03AF8E0DF0731F459
:10E9000080914E0684FD8CC011E18BC0803B38E0C5
:10E91000930779F0803AE9E09E0731F430916E0672
:10E9200034FD82C019E110C0803BF9E09F0789F0F7
:10E9300001C015E1803A3AE0930731F480918E06E8
:10E9400084FD74C011E212C0803BEAE09E0759F0DA
:10E9500001C01DE1803A9B4049F48091AE0684FDE0
:10E9600004C019E203C015E201C01DE2E12FE695E3
:10E97000E695E69530E2E39FF0011124FA5F177007
:10E9800081E090E0012E02C0880F991F0A94E2F7FF
:10E990008183223010F040E001C040E4DF01509656
:10E9A000A10FB11D3FB7F8942C9127702C939C9127
:10E9B000942B9C933FBF85838D81806C8D83F70161
:10E9C00084818D7F813021F48D8182608D8303C0AD
:10E9D0008D818D7F8D83F7018581882321F08D8145
:10E9E00084608D8303C08D818B7F8D83F70140818F
:10E9F00051816281738100E010E62AEE30E0CE01A1
:10EA000011DE8C8188608C838C8180618C8310C046
:10EA10008C818F7E8C83F70124812250CE0176CFAA
:10EA200015E180EA98E080CF1DE18ECF15E29ECF00
:10EA3000DF91CF911F910F91FF90EF9008950F9369
:10EA4000E8ECF4E080818F7D808380818F7D8083FE
:10EA5000E0E8F7E302E005931092823710928337E3
:10EA600000E2069300E40693E8E7F7E300E206938A
:10EA700000E40693ECEDF0E41486158616861786FE
:10EA80001286138610926B370F9108950F9385E0CD
:10EA900080936B37E1E8F7E304E00593E9E7F7E3F8
:10EAA00004E005930F9108950F9383E080936B37F3
:10EAB0001092823710928337E0E8F7E302E0069382
:10EAC0000F910895E091E840F091E940309709F006
:10EAD000199508950F93CF93DF9380916B3783300F
:10EAE00019F4F0DFACDF5EC0809167379091683732
:10EAF000C091E640D091E740C81BD90B71F5209139
:10EB0000693730916A37820F931F809369379093EA
:10EB10006A372091E2403091E3408217930721F059
:10EB200080918236882341F084E080936B37E8E758
:10EB3000F7E302E0069336C0E091EA40F091EB4043
:10EB4000309799F01995882381F0109267371092C9
:10EB50006837C091E640D091E740C034D10528F035
:10EB600010928236C0E4D0E003C081E08093823608
:10EB7000ECE6F7E3C68BD78B8091673790916837C7
:10EB80002091E4403091E540280F391F208F318FCC
:10EB9000C80FD91FC0936737D0936837E0E8F7E311
:10EBA00002E00693DF91CF910F910895FC018181DE
:10EBB000E82FE7708E2F90E0FC013197E730F105E8
:10EBC000D8F48827EE52FE4F8F4F0D942B6580E1CD
:10EBD00090E0089580E290E0089580E490E0089548
:10EBE00080E890E0089580E091E0089580E092E070
:10EBF00008958FEF93E0089588E090E00895282F1E
:10EC00002F7030E0220F331F082E000C990B88273D
:10EC1000990F881F9927820F931F02979C01220F3B
:10EC2000331F220F331F220F331F820F931F8D5F5D
:10EC3000984C08950F93CF938091CC0480FF63C0CC
:10EC400081E08093CC04E8E7F7E300E80693E0E88E
:10EC5000F7E300E806938093CA04E8E7F7E300E1EE
:10EC6000069380916B37882329F08350823008F413
:10EC700029DFE5DE80917A3790917B37089709F09C
:10EC800044C088E0E7E2F7E3ACEDB0E401900D9218
:10EC90008A95E1F7E8ECF4E08081806280838081EE
:10ECA000806280830E944A64C82F811103C0EEDE17
:10ECB000C1E02CC08091DC4088236CF4109269374D
:10ECC00010926A37109267371092683782E080930B
:10ECD0006B3700DF1BC08091E2409091E340892BAD
:10ECE00011F4E2DE13C01092693710926A37109265
:10ECF00067371092683781E080936B37E8E7F7E376
:10ED000002E0069303C0C0E001C0C1E08C2FCF91A8
:10ED10000F9108958F929F92AF92BF92DF92EF92E0
:10ED2000FF920F931F93CF93DF93D82E68DF8C0150
:10ED3000CD2DCF70D0E0CE01880F991FCD2D0D2C99
:10ED4000000CDD0BCC27DD0FCC1FDD27C80FD91F32
:10ED5000CE01880F991F880F991F880F991F9C015A
:10ED60002858384C7901C90121DF4C01DD200CF015
:10ED70007BC0FE01EE0FFF1FEE0FFF1FEE0FFF1F08
:10ED8000E459F84C22893389D80115968D919C91CC
:10ED90001697820F931F15968D939C931697139633
:10EDA0002D913C9114978217930709F447C0281BB3
:10EDB000390B2115B4E03B0740F02FEF33E0C901D8
:10EDC000B4010F94C664281B390BF801808181FFC0
:10EDD0000AC0C901B4010F94C66441E0892B09F04F
:10EDE00040E0842F01C080E0D8019C9180FB91F924
:10EDF0009C93FE01EE0FFF1FEE0FFF1FEE0FFF1F94
:10EE0000E459F84C128A138A2687378711962D9178
:10EE10003C91129715968D919C911697820F931F96
:10EE2000CC0FDD1FCC0FDD1FCC0FDD1FC458D84C1D
:10EE300088839983F70102E00693E4C0D8018C919E
:10EE400081FFCDC08D7F8C93CC0FDD1FCC0FDD1FDC
:10EE5000CC0FDD1FC459D84C1A8A1B8A1E861F8608
:10EE6000F70102E00693CEC0FE01EE0FFF1FEE0F8A
:10EE7000FF1FEE0FFF1FE459F84CA684B784D8019A
:10EE80008C9182FF1BC01196ED91FC911297159603
:10EE90002D913C91169713968D919C911497B401E6
:10EEA0000F94C664B0E4DB9EB00111246D5B794C15
:10EEB000AC01CF01820F931F0F942A67F8012581BF
:10EEC00036812A0D3B1D25833683838194818217E9
:10EED000930768F485839683CC0FDD1FCC0FDD1F6D
:10EEE000CC0FDD1FC459D84C8A899B8978C0FE019C
:10EEF000EE0FFF1FEE0FFF1FEE0FFF1FE459F84C40
:10EF000042895389A416B50609F069C02817390744
:10EF100009F465C0AC01421B530B9A01211554E062
:10EF2000350748F02FEF33E0C901B4010F94C664F0
:10EF3000281B390B06C0C901B4010F94C664281BF5
:10EF4000390BFE01EE0FFF1FEE0FFF1FEE0FFF1F2D
:10EF5000E459F84C168617862815390500F5D801AE
:10EF60008C9184608C93B0E4DB9EC00111248D5B96
:10EF7000994CFE01EE0FFF1FEE0FFF1FEE0FFF1F5C
:10EF8000E458F84C80839183CC0FDD1FCC0FDD1F3C
:10EF9000CC0FDD1FC459D84C8A8A9B8A1CC0F8014B
:10EFA0004181528185819681840F951FFE01EE0F6C
:10EFB000FF1FEE0FFF1FEE0FFF1FE458F84C80837A
:10EFC0009183CC0FDD1FCC0FDD1FCC0FDD1FC4598B
:10EFD000D84C2A8B3B8BF70102E0069313C0D80173
:10EFE0008C9180FF0FC08E7F8C931796ED91FC91D2
:10EFF0001897309739F015966D917C9116974D2D95
:10F0000080E01995DF91CF911F910F91FF90EF90C4
:10F01000DF90BF90AF909F908F900895CF93CFB720
:10F02000F894E1ECF4E080818E7F80831092C0043C
:10F0300010820F94AA441092AC37CFBFCF9108959D
:10F040009FB7F89481E08093AC37EAECF4E080E479
:10F05000808380E28083E1ECF4E0808181608083C2
:10F06000A9ECB4E08C9182608C93E8ECF4E08081B0
:10F07000806480838C9181608C93808180688083A0
:10F080009FBF0895CF93DF93C0E6D0E0188280E35E
:10F090000F947244E0ECF4E080818064808381E02E
:10F0A0008883CFB7F894ECE6F7E31586158A158EBA
:10F0B00015A215A615AAE3E0F7E380818E7F808371
:10F0C000ECE0F7E380818E7F8083E5E1F7E38081E8
:10F0D0008E7F8083EEE1F7E380818E7F80836AE11B
:10F0E00070E082E00F9486628F3F19F08093FA04FB
:10F0F00003C08FE18093FA046BE170E082E00F942B
:10F1000086628F3F19F08093FB0403C08FE18093E8
:10F11000FB04E0ECF4E08081826080838081806881
:10F12000808380818061808388E797E386839783EB
:10F130008081806280838FEF8093C504E8ECF4E0E7
:10F140008081816080831092AC377ADFCFBFDF91FE
:10F15000CF9108958093C30408958091C3040895C6
:10F16000ECEDF0E480879187628773870895282FFC
:10F170002F7030E0220F331F082E000C990B8827C8
:10F18000990F881F9927820F931FFC01EE0FFF1F15
:10F19000EE0FFF1FEE0FFF1FE459F84C2585207C72
:10F1A00009F069C06370613011F018F404C060ECBC
:10F1B00003C060E801C060E440385105E9F050F454
:10F1C00040325105A9F040345105A1F040315105BC
:10F1D000D9F40CC0411522E0520791F04F3F23E0D3
:10F1E000520781F04115514079F408C021E00DC06B
:10F1F00022E00BC023E009C024E007C025E005C0E1
:10F2000026E003C027E001C020E0FC01EE0FFF1F55
:10F21000EE0FFF1FEE0FFF1FE459F84C158636E086
:10F220003487262B2587FC01EE0FFF1FEE0FFF1FF3
:10F23000EE0FFF1FE459F84C2585207C203C69F433
:10F24000FC01EE0FFF1FEE0FFF1FEE0FFF1FE45933
:10F25000F84C25852770273081F0880F991F880F7B
:10F26000991F880F991FFC01E459F84C858580622D
:10F27000858781E0089580E0089581E00895E82F72
:10F28000EF70F0E0EE0FFF1F082E000C990B88279F
:10F29000990F881F9927E80FF91FEE0FFF1FEE0F38
:10F2A000FF1FEE0FFF1FE459F84C858582FB88276E
:10F2B00080F90895282F2F7030E0A901440F551FC1
:10F2C000282F082E000C330B2227330F221F332741
:10F2D000240F351FF901EE0FFF1FEE0FFF1FEE0F7A
:10F2E000FF1FE459F84C958592FF17C0220F331F7A
:10F2F000220F331F220F331FF901E459F84C958573
:10F300009B7F95877CDCFC01808180FF06C08E7F1F
:10F3100080830780F085E02D199581E008958F9214
:10F320009F92AF92BF92CF92DF92EF92FF920F9394
:10F330001F93CF93DF93982E862E6A0179015FDCAD
:10F340005C01292DC92DCF70D0E0CE01880F991F07
:10F35000C92D092C000CDD0BCC27DD0FCC1FDD27C0
:10F36000C80FD91FFE01EE0FFF1FEE0FFF1FEE0F9C
:10F37000FF1FE459F84C8585807C09F47EC0FE01AE
:10F38000EE0FFF1FEE0FFF1FEE0FFF1FE459F84CAB
:10F390008585807C803C61F0FE01EE0FFF1FEE0F43
:10F3A000FF1FEE0FFF1FE459F84C858582FD67C0F3
:10F3B0008FB7F894F501908190FF03C08FBF80E074
:10F3C0005FC0F5019081916090838FBFC182D2822E
:10F3D000E382F4821582168207831087811006C0AB
:10F3E00091E0E114F10419F090E001C091E0F50121
:10F3F000808190FB81F98B7F808322235CF4CC0F8A
:10F40000DD1FCC0FDD1FCC0FDD1FC459D84C1A8A6D
:10F410001B8A2FC0FE01EE0FFF1FEE0FFF1FEE0F26
:10F42000FF1FE459F84C8585807C803CB1F4CE0107
:10F43000880F991F880F991F880F991F8858984C1B
:10F44000B5DBBC01C7010F94C664892B31F0F5010F
:10F4500080818E7F808380E013C0CC0FDD1FCC0FB6
:10F46000DD1FCC0FDD1FC459D84C1E861F861A8A9B
:10F470001B8A892D4FDC81E003C080E001C080E061
:10F48000DF91CF911F910F91FF90EF90DF90CF9080
:10F49000BF90AF909F908F900895FF920F931F930E
:10F4A000CF93DF93182FC82FCF70D0E0CE01880FF5
:10F4B000991FC12F012E000CDD0BCC27DD0FCC1FB7
:10F4C000DD27C80FD91F812F9ADBDC01FE01EE0F6B
:10F4D000FF1FEE0FFF1FEE0FFF1FE858F84C02E072
:10F4E00005938C9180FF22C08E7F8C931796ED91AF
:10F4F000FC9118973097D1F011235CF4CC0FDD1FED
:10F50000CC0FDD1FCC0FDD1FC459D84C6A897B8915
:10F510000AC0CC0FDD1FCC0FDD1FCC0FDD1FC4597F
:10F52000D84C6E857F85412F81E01995DF91CF9171
:10F530001F910F91FF900895CF93C82FAEDFEC2F4E
:10F54000EF70F0E0EE0FFF1F8C2FCC0F990B882788
:10F55000990F881F9927E80FF91FEE0FFF1FEE0F75
:10F56000FF1FEE0FFF1FE459F84C1586CF91089549
:10F570000F93E82FEF70F0E0EE0FFF1F282F082EFB
:10F58000000C330B2227330F221F3327E20FF31F08
:10F59000EE0FFF1FEE0FFF1FEE0FFF1FDF01A4593D
:10F5A000B84C1D969C911D9794601D969C93E858AD
:10F5B000F84C01E0069371DF81E00F9108950F93FD
:10F5C0001F93CF93DF938B01C82FCF70D0E0CC0F68
:10F5D000DD1F282F082E000C330B2227330F221F8C
:10F5E0003327C20FD31F0BDBCC0FDD1FCC0FDD1F6A
:10F5F000CC0FDD1FC459D84C2D8522FF0AC0FC0159
:10F60000208120FD0AC0216020830783108781E0CC
:10F6100005C0F801199581E001C080E0DF91CF912C
:10F620001F910F9108951F920F920FB60F92112400
:10F630000BB60F920F932F933F934F935F936F935C
:10F640007F938F939F93AF93BF93EF93FF9380919B
:10F65000CB04882344F480E88093CA040E941A648F
:10F660000E94505B87C08091CB0482FF20C084E061
:10F670008093CA048091803786FF7CC08091CC043F
:10F6800081FD78C0D7DA811175C080916B378130E8
:10F6900011F40ADA6FC0843009F06CC0E1E8F7E3D6
:10F6A00004E00593E9E7F7E304E0059363C0809184
:10F6B000CB0481FF5AC082E08093CA0480917837DE
:10F6C00086FF58C08091CC0481FD54C0B3DA81110B
:10F6D00051C080916B37823041F484E080936B3766
:10F6E000E8E7F7E302E0069345C0833009F042C043
:10F6F000E1E8F7E304E00593E9E7F7E304E00593C5
:10F7000039C080E18093CA0481E0C7DE81E8C5DEAC
:10F710000E94EF631092C304ECE6F7E3158696E0CF
:10F72000948783E48587158A948B858B87E297E39A
:10F73000808B918B84D91EC08091CB0486FF08C03A
:10F7400080E48093CA041092AC370E94535B12C0CD
:10F750008091CB0485FF0EC080E28093CA0481E0D3
:10F760008093AC370E94545B05C08091CB0484FF2A
:10F77000E3CFC7CFFF91EF91BF91AF919F918F9151
:10F780007F916F915F914F913F912F910F910F90CA
:10F790000BBE0F900FBE0F901F9018951F920F92E7
:10F7A0000FB60F9211240BB60F920F931F932F9346
:10F7B0003F934F935F936F937F938F939F93AF93F9
:10F7C000BF93CF93DF93EF93FF938091CC0481FDA0
:10F7D00003C030DA8111C2C082E08093CC048091F2
:10F7E000C5048195880FE8E7F7E3E81BF10920815C
:10F7F0003181285737433695279536952795369585
:10F800002795822F869520FD02C090E001C090E8E8
:10F81000890FE82FEF70F0E0EE0FFF1F282F082E62
:10F82000000C330B2227330F221F3327E20FF31F65
:10F83000DF01AA0FBB1FAA0FBB1FAA0FBB1FA45932
:10F84000B84C1C969C9195FF89C0EE0FFF1FEE0FE0
:10F85000FF1FEE0FFF1FE858F84C00E206938111DE
:10F8600078C080916B37843019F42CD9E8D876C0F1
:10F8700000917A3710917B378091E6409091E74074
:10F88000C0916737D091683798012C0F3D1F8217C0
:10F89000930718F48C010C1B1D0B8091E440909190
:10F8A000E540A80167E277E38C0F9D1F0F942A675C
:10F8B000C00FD11FC0936737D0936837003411054C
:10F8C00069F48091693790916A378C0F9D1F209160
:10F8D000E2403091E3408217930780F0ECEDF0E4D2
:10F8E000C287D3870684F785E02D309729F01995D4
:10F8F000811102C0CBD832C0D7D830C08091E64049
:10F900009091E740C817D907F9F4E091EA40F091E7
:10F91000EB40309711F4BAD821C01995811102C07B
:10F92000B5D81CC02091693730916A37809167370C
:10F9300090916837820F931F8093693790936A374D
:10F940001092673710926837E8E7F7E302E0069312
:10F9500005C0803811F4BED801C0DCD9FF91EF9109
:10F96000DF91CF91BF91AF919F918F917F916F91D7
:10F970005F914F913F912F911F910F910F900BBE6F
:10F980000F900FBE0F901F9018959091800024E06B
:10F99000829FB00111246C7392709160692B80E892
:10F9A00090E00F942762E0E8F0E0828180FDFDCFD7
:10F9B0000895609180006C73636080E890E00F941C
:10F9C0002762E0E8F0E0828180FDFDCF0895CF92CC
:10F9D000DF92EF92FF92CF93DF93EC016B01E12C6A
:10F9E000F12C60E070E68AEE90E0A70196010F949A
:10F9F000ED64CA01B9012FEF3FEF40E050E00F94F2
:10FA0000ED642115310529F481E08C8321E030E09B
:10FA10002DC02230310528F482E08C8322E030E0D2
:10FA200025C02430310528F483E08C8324E030E0C5
:10FA30001DC02830310528F484E08C8328E030E0B4
:10FA400015C02034310528F485E08C8320E430E0B3
:10FA50000DC02F3F310509F028F486E08C8320E0AB
:10FA600031E004C087E08C8320E034E040E050E0E7
:10FA700060E070E68AEE90E00F94ED64CA01B9018F
:10FA8000A70196010F94ED642D833E832436310542
:10FA900018F41C821D821E82DF91CF91FF90EF909F
:10FAA000DF90CF9008950F931F93CF93DF93EC01D6
:10FAB0008901862F90E08730910508F08BC0FC010A
:10FAC0008827E752FE4F8F4F0D942B6580E098E01A
:10FAD00088839983E0E4F6E0308181E090E02FEFC5
:10FAE000240F02C0880F991F2A95E2F7832B808389
:10FAF00071C080E498E088839983E0E4F6E0308187
:10FB000081E090E023E0240F02C0880F991F2A951E
:10FB1000E2F7832B80835EC080E099E0888399833D
:10FB2000E0E6F6E0308181E090E02FEF240F02C0A4
:10FB3000880F991F2A95E2F7832B80834BC080E4BE
:10FB400099E088839983E0E6F6E0308181E090E0F7
:10FB500023E0240F02C0880F991F2A95E2F7832B18
:10FB6000808338C080E09AE088839983E0E8F6E0FB
:10FB7000308181E090E02FEF240F02C0880F991FA1
:10FB80002A95E2F7832B808325C080E49AE088835E
:10FB90009983E0E8F6E0308181E090E023E0240FF3
:10FBA00002C0880F991F2A95E2F7832B808312C029
:10FBB00080E09BE088839983E0EAF6E0308181E091
:10FBC00090E02FEF240F02C0880F991F2A95E2F7CB
:10FBD000832B80834A83423061F018F4413031F046
:10FBE00010C0433049F0443051F00BC080E18B83AA
:10FBF00008C080E28B8305C080E48B8302C080E86C
:10FC00008B83888199810E94A86FE881F981818125
:10FC1000887F836081831D821E821C82E881F98136
:10FC20008081807F8083B801CE01D1DEDF91CF91CA
:10FC30001F910F910895CF93DF93EC012D813E81A9
:10FC4000A62FB0E00F94336524E630E040E050E0AA
:10FC50000F94ED648A81E881F981E6FD17C0823056
:10FC600061F018F4813031F01BC0833049F08430EA
:10FC700051F016C020AF31AF13C022AF33AF10C068
:10FC800024AF35AF0DC026AF37AF0AC0813019F0B1
:10FC9000823021F005C020AF31AF02C022AF33AFB8
:10FCA0008D819E81E881F98186A397A38B81E8816C
:10FCB000F981E6FD04C09181892B818304C0918183
:10FCC0008073892B8183E881F9818081807F9C8189
:10FCD000892B8083DF91CF910895CF93DF93EC013F
:10FCE0004115510509F443C0A9E4B3E420E030E034
:10FCF000922FF901E45FFA4EE491ED932F5F3F4FAD
:10FD000027303105A9F7FA01DE01C9E4D3E4808187
:10FD10008B8381818C83F901E75BFC4B8CE28083D0
:10FD2000E2E0E90FF0E0E75BFC4B6083C4E0C90F61
:10FD30009D5FE92FF0E0E75BFC4B8DE78083D0E02F
:10FD4000FE01E75BFC4B108221E0AE0169E473E445
:10FD5000CD010F94F0310E944E2A811108C021E09C
:10FD6000AE0169E473E48AEA99E30F94F031DF911C
:10FD7000CF9108954F925F926F927F928F929F9250
:10FD8000AF92BF92DF92EF92FF920F931F93CF93A8
:10FD9000DF931F92CDB7DEB77C014115510509F401
:10FDA00066C188E08983A9E4B3E420E030E0922FC3
:10FDB000F901E45FFA4EE491ED932F5F3F4F273056
:10FDC0003105A9F7FA01162FA9E4B3E4808113964F
:10FDD0008C931397818114968C9302E0090FF9019B
:10FDE000E75BFC4B8CE28083623088F5862F0F94B2
:10FDF00077188823B1F0812F0F943C189F938F932D
:10FE00001F921F938BE599E29F938F93E02FF0E071
:10FE1000E75BFC4BFF93EF930F945867CDBFDEBFBA
:10FE200008C1812F0E942FD19F938F931F921F9300
:10FE30008BE599E29F938F93E02FF0E0E75BFC4B1B
:10FE4000FF93EF930F945867CDBFDEBFF2C06631CA
:10FE500009F078C086E10F9480172B013C010F94C4
:10FE60000A0F4B015C01672B682B692BF1F4C3016E
:10FE7000B20120E13EE040E050E00F940F655F9357
:10FE80004F933F932F931F9286E18F9382E699E2DF
:10FE90009F938F93E02FF0E0E75BFC4BFF93EF9392
:10FEA0000F945867CDBFDEBFC4C0802F0E94CAD058
:10FEB000992334F5C301B20120E13EE040E050E077
:10FEC0000F940F65CA01B9010F946D37BF92AF92BD
:10FED0009F928F929F938F937F936F931F9286E150
:10FEE0008F938AE699E29F938F93E02FF0E0E75B90
:10FEF000FC4BFF93EF930F945867CDBFDEBF99C0C3
:10FF0000BF92AF929F928F92C301B20120E13EE077
:10FF100040E050E00F940F655F934F933F932F9312
:10FF20001F9286E18F9387E799E29F938F93E02F4B
:10FF3000F0E0E75BFC4BFF93EF930F945867CDBF66
:10FF4000DEBF77C0663071F5E02FF0E0E75BFC4B79
:10FF500086E380836894DD24D2F8D90E9D5FE92F73
:10FF6000F0E0E75BFC4B8CE2808386E00F94801727
:10FF70008B019C018D2D90E04BE0BE016F5F7F4FA8
:10FF8000875B9C4B0F94C637E981ED0DAE2FB0E037
:10FF9000A75BBC4B8DE78C93EF5FF0E0E75BFC4B1E
:10FFA000108247C0653071F5E02FF0E0E75BFC4B55
:10FFB00085E380836894DD24D2F8D90E9D5FE92F14
:10FFC000F0E0E75BFC4B8CE2808385E00F948017C8
:10FFD0008B019C018D2D90E04BE0BE016F5F7F4F48
:10FFE000875B9C4B0F941239E981ED0DAE2FB0E089
:10FFF000A75BBC4B8DE78C93EF5FF0E0E75BFC4BBE
:020000021000EC
:10000000108217C0862F0F9480179F938F937F9332
:100010006F931F921F9382E699E29F938F93802F95
:1000200090E0875B9C4B9F938F930F945867CDBF55
:10003000DEBFE9E4F3E401900020E9F73197E954E9
:10004000F344E983AF01552721E069E473E4C70174
:100050000F94F0310E944E2A811109C0498150E06D
:1000600021E069E473E48AEA99E30F94F0310F9098
:10007000DF91CF911F910F91FF90EF90DF90BF9094
:10008000AF909F908F907F906F905F904F9008956A
:10009000AC016115710571F1E5E1F5E1A9E4B3E4A5
:1000A00021E533E494919D933196A217B307D1F7DC
:1000B000FB01CA01A9E4B3E4208113962C931397A2
:1000C000218114962C93149718961C92189721E06E
:1000D00048E050E0BD010F94F0310E944E2A81119A
:1000E00009C021E048E050E069E473E48AEA99E35A
:1000F0000D94F0310895EF92FF920F931F93CF93D9
:10010000DF938C016115710509F47FC0411551051C
:1001100009F47BC0E3E0F5E1A9E4B3E4C1E5D3E48D
:1001200094919D933196AC17BD07D1F7FA017B01ED
:10013000C9E4D3E480818B8381818C831F922F93C8
:1001400083E899E29F938F9381E593E49F938F9344
:100150000F94586709900020E9F72197C954D344B8
:10016000F70181810F900F900F900F900F900F90DB
:10017000811115C080811F928F9380E791E29F9338
:100180008F93DD27C75BDC4BDF93CF930F945867CA
:100190000F900F900F900F900F900F9016C01F921E
:1001A0008F93F70180811F928F938DE691E29F9349
:1001B0008F93DD27C75BDC4BDF93CF930F9458679A
:1001C000EDB7FEB73896EDBFFEBFE9E4F3E401906A
:1001D0000020E9F73197E954F344EF01DD2721E0EE
:1001E000AE0169E473E4C8010F94F0310E944E2A15
:1001F00081110BC00A5A194341F021E0AE0169E4B4
:1002000073E48AEA99E30F94F031DF91CF911F9163
:100210000F91FF90EF900895CF93DF93EC0141157C
:10022000510509F43FC0662361F0E5E1F5E1A9E479
:10023000B3E490E024912D939F5F31969730D1F7EE
:100240000BC0ECE0F5E1A9E4B3E490E024912D9338
:100250009F5F31969730D1F7DA01CE01E9E4F3E4FC
:100260002C91238311962C9124832CE227833CE448
:100270003087218720E322872DE72387148621E01A
:100280004CE050E0BF010F94F0310E944E2A8111E2
:1002900009C021E04CE050E069E473E48AEA99E3A4
:1002A0000F94F031DF91CF910895EF92FF920F9369
:1002B0001F93CF93DF9300D01F92CDB7DEB7009787
:1002C000C9F166307105C0F1FC0120812035B1F51E
:1002D00021812C32A9F524812C32A1F57A018C01DF
:1002E0000B5F1F4FAB01455051099E012F5F3F4FE0
:1002F000B8018CE20F949D37882349F149815A81D6
:100300004B5F5F4F49835A8346305105E8F04550B3
:100310009E012D5F3F4F60E0C8010F942536882372
:10032000B1F08B819C818C31910580F4F701808341
:1003300081E00DC080E00BC080E009C080E007C014
:1003400080E005C080E003C080E001C080E024962A
:10035000CDBFDEBFDF91CF911F910F91FF90EF9046
:100360000895CF92DF92EF92FF920F931F93CF9356
:10037000DF93CDB7DEB72C97CDBFDEBF009709F472
:1003800031C16630710508F42FC1FC012081203590
:1003900009F02CC121812C3209F02AC124812C3290
:1003A00009F028C17B018C016C01F5E0CF0ED11C56
:1003B000AB01455051099E012F5F3F4FB6018CE2C2
:1003C0000F949D37982F882309F423C149815A81BE
:1003D0004B5F5F4F49835A834630510508F40CC187
:1003E00045509E012D5F3F4F60E0C6010F942536BA
:1003F000982F882309F40DC12B813C812C313105C4
:1004000008F0FCC049815A81DA011196AE15BF058A
:1004100008F0F6C02C31310508F0F4C0F901882746
:10042000E052FE4F8F4F0D942B65C8018A0F9B1F22
:10043000FC0160816D3241F4FA013296EE15FF0540
:1004400008F0E2C040E002C0FD0141E02631310584
:1004500059F46E2D6E1B9E01275F3F4FC8018E0F12
:100460009F1F0F94760512C02630310541F46E2D82
:100470006A1BAE01475F5F4F0F94430807C06E2DA4
:100480006A1BAE01475F5F4F0F945F09882309F431
:10049000BDC049855A856B857C858B810E941ED69F
:1004A000982F882309F4B5C049855A856B857C85CA
:1004B0008B810F94931791E0ACC04E2D4A1B9E0187
:1004C0002B5F3F4F60E0C8018A0F9B1F0F94B0362F
:1004D000982F882309F49DC04D815E816F817885B6
:1004E00049875A876B877C878B810E941ED6982FFD
:1004F000882309F48EC089859A85AB85BC858B30AD
:100500009105A105B10549F487EF9CE30E94DF2E18
:10051000982F882309F47DC00CC00C97A105B10564
:1005200044F087EF9CE30E94DF2E982F882309F484
:1005300070C049855A856B857C858B810F94931794
:1005400091E067C04E2D4A1B9E012B5F3F4F60E03C
:10055000C8018A0F9B1F0F94B036982F882309F487
:1005600058C04D815E816F81788549875A876B8736
:100570007C878B810E941ED6982F882349F049855D
:100580005A856B857C858B810F94931791E041C0D0
:100590002B813C81A9014C50510946305105C8F5C9
:1005A00049855A856B857C85452B462B472B89F5DC
:1005B00040E050E0BA01822F0F94931791E029C0D8
:1005C000C7018A1B9B0B899718F56E2D6A1B422F5A
:1005D000C8018A0F9B1F0F94FE1791E0811119C06B
:1005E00090E017C090E015C090E013C090E011C0FB
:1005F00090E00FC090E00DC090E00BC090E009C00B
:1006000090E007C090E005C090E003C090E001C01A
:1006100090E0892F2C96CDBFDEBFDF91CF911F9147
:100620000F91FF90EF90DF90CF9008950F931F935D
:10063000CF93DF931F921F92CDB7DEB7009741F1A2
:100640006630710538F1FC012081203529F52181C2
:100650002C3221F524812C3219F58C01AB01455047
:100660005109BC016B5F7F4F9E012F5F3F4F8CE2B2
:100670000F949D378823B9F089819A810596069752
:1006800088F081E0F8019581963469F080E00BC034
:1006900080E009C080E007C080E005C080E003C0C2
:1006A00080E001C080E00F900F90DF91CF911F910B
:1006B0000F910895EF92FF920F931F93CF93DF93C3
:1006C00000D000D0CDB7DEB7009709F453C0663034
:1006D000710508F451C0FC012081203509F04EC09D
:1006E00021812C3209F04CC024812C3209F04AC0FF
:1006F0007B018C01AB0145505109BC016B5F7F4F01
:100700009E012F5F3F4F8CE20F949D37882309F4A1
:1007100042C089819A819C012B5F3F4F29833A8394
:100720002630310588F1F8012581263479F50696C1
:100730008E159F0568F54E2D481B9E012D5F3F4F7E
:1007400060E0800F911F0F94B036882321F16B81F8
:100750007C818D819E818B019C01015011092109B1
:100760003109073E134021053105A0F40E94B3D1A1
:1007700081E011C080E00FC080E00DC080E00BC0C0
:1007800080E009C080E007C080E005C080E003C0D1
:1007900080E001C080E02696CDBFDEBFDF91CF9123
:1007A0001F910F91FF90EF9008950F931F93CF9398
:1007B000DF93EC016115710509F444C0A9E4B3E4C9
:1007C00020E030E0922FF901E45FFA4EE491ED93DE
:1007D0002F5F3F4F27303105A9F7FB01A9E4B3E4B0
:1007E000808113968C931397818114968C93149720
:1007F000F901E75BFC4B8CE280839E5FE92FF0E020
:10080000E75BFC4B86E49DE7808391831282FD01C8
:1008100001900020E9F73197E954F3448F01112743
:1008200021E0A801BD01CE010F94F0310E944E2AB3
:10083000811108C021E0A80169E473E48AEA99E320
:100840000F94F031DF91CF911F910F910895FC012A
:10085000892B61F06530710558F08081803551F445
:1008600081E091819C3239F080E0089580E0089524
:1008700080E0089580E00895009799F06330710555
:1008800090F0FC012081203581F421812C3279F413
:1008900024812C3271F485818354823060F080E0B1
:1008A000089580E0089580E0089580E0089580E054
:1008B000089580E0089581E00895009791F06330F5
:1008C000710588F0FC012081203579F421812C32DA
:1008D00071F424812C3269F485818F3461F080E0D9
:1008E000089580E0089580E0089580E0089580E014
:1008F000089580E0089581E00895009791F06330B5
:10090000710588F0FC012081203579F421812C3299
:1009100071F424812C3269F48581873561F080E09F
:10092000089580E0089580E0089580E0089580E0D3
:10093000089580E0089581E00895CF92DF92EF92CC
:10094000FF920F931F93CF93DF934115510509F445
:10095000AFC0009709F4AEC06630710508F4ACC0B2
:10096000FC012081203509F0A9C021812C3209F039
:10097000A7C024812C3209F0A5C08581873509F0F4
:10098000A3C0EA0187EF9CE30E94BF14883009F4FA
:100990009DC087EF9CE30E94BF14863009F498C085
:1009A0000F9491290E94255661E08DEF9CE30E94EF
:1009B00099580F94BB180E94D11C813079F582E0C0
:1009C0000E94D8D06B017C01DD24EE24FF24B70106
:1009D000A60182E00F949317B701A60182E00E945E
:1009E000C0D00E944E2A811119C084E1E7E8F9E2E3
:1009F000A0EDB4E401900D928A95E1F7E0EDF4E406
:100A000001900020E9F73197AF01405D544420E0A8
:100A100060ED74E48AEA99E30F94F031CE010E940C
:100A2000201C80E00E94A6D09B01AC016894EE24BB
:100A3000E2F801ED12E2BE01685E7F4FCE0106963C
:100A40000E94F3598D8340E050E0BA01CE010E942C
:100A50008F2E8D81882351F182E00E94CAD0062F0B
:100A60008BE00E94CAD021E0611120E043EB50E40A
:100A7000BE016C5C7F4FCE01C6960E94F652CE013D
:100A80000E94F61B9E01265A3D4FAE01475A5D4F0C
:100A9000BE016C5A7D4FCE018D5A9D4F0E94162D7E
:100AA0000E94153468E0CE010E94AC148D8111C003
:100AB00080E00FC080E00DC080E00BC080E009C086
:100AC00080E007C080E005C080E003C080E001C096
:100AD00080E0DF91CF911F910F91FF90EF90DF9019
:100AE000CF900895CF92DF92EF92FF920F93CF9322
:100AF000DF934115510509F4B0C0009709F4AFC068
:100B00006630710508F4ADC0FC012081203509F084
:100B1000AAC021812C3209F0A8C024812C3209F00E
:100B2000A6C0EA018581833409F493C0843409F0B6
:100B3000A0C00E9468D10F94591887EF9CE30E94CF
:100B4000BF14883009F497C087EF9CE30E94BF145C
:100B5000863009F492C00F9491290E94255661E0D5
:100B60008DEF9CE30E9499580F94BB180E94D11CF2
:100B7000813079F582E00E94D8D06B017C01DD24C0
:100B8000EE24FF24B701A60182E00F949317B7016A
:100B9000A60182E00E94C0D00E944E2A811119C095
:100BA00084E1E7E8F9E2A0EDB4E401900D928A95C2
:100BB000E1F7E0EDF4E401900020E9F73197AF01AF
:100BC000405D544420E060ED74E48AEA99E30F94B8
:100BD000F03180E00E94A6D09B01AC01BE01685EAE
:100BE0007F4FCE0106960E942D568D8340E050E047
:100BF000BA01CE010E948F2E8D81882341F182E0BF
:100C00000E94CAD0062F8BE00E94CAD021E0611159
:100C100020E043EB50E4BE016C5C7F4FCE01C696F2
:100C20000E94F652CE010E94F61B9E01265A3D4FAD
:100C3000AE01475A5D4FBE016C5A7D4FCE018D5AB1
:100C40009D4F0E94162D68E0CE010E94AC148D814C
:100C500015C00F94591881E011C080E00FC080E0EA
:100C60000DC080E00BC080E009C080E007C080E0DC
:100C700005C080E003C080E001C080E0DF91CF913B
:100C80000F91FF90EF90DF90CF900895BF92CF9299
:100C9000DF92EF92FF920F931F93CF93DF931F92F8
:100CA000CDB7DEB76115710509F464C0DB017C01C5
:100CB000E9E4F3E48BE7808380E781838CE282833D
:100CC0009C91938311969C91948385839FE4968352
:100CD000878380E00E9425D88B019C0148E0BE01FB
:100CE0006F5F7F4F81E593E40F947439E981E85F8A
:100CF000D12C0F2EFCE2BF2EF02DCC24C394CE0EAF
:100D0000F0E0E75BFC4BB082D3948D2D0E9425D898
:100D10008B019C018C2D90E048E0BE016F5F7F4FFE
:100D2000875B9C4B0F947439E981EC0D83E0D812FA
:100D3000E4CF81E08E0FF0E0E75BFC4B9DE7908312
:100D4000482F50E0FA01E75BFC4B1082898321E0D9
:100D500069E473E4C7010F94F0310E944E2A8111B7
:100D600009C0498150E021E069E473E48AEA99E32B
:100D70000F94F0310F90DF91CF911F910F91FF9061
:100D8000EF90DF90CF90BF900895CF93DF93411500
:100D90005105A9F10097A9F165307105A0F1FC0199
:100DA0002081203591F521812C3289F5228126344C
:100DB00081F5EA0184818235E9F0833531F08434AC
:100DC00051F50E9492D181E027C00F949129BE0174
:100DD0006C5C7F4FCE01C6960E94FB5087EF9CE370
:100DE0000E94992281110F94B329CE010E94E62915
:100DF0008D8112C0CA01C6960F94640E0DC080E0AA
:100E00000BC080E009C080E007C080E005C080E042
:100E100003C080E001C080E0DF91CF910895FC0124
:100E2000892B79F06630710570F08081833569F423
:100E300081818C3261F481E094819C3249F080E0C0
:100E4000089580E0089580E0089580E0089580E0AE
:100E500008950F93CF93DF93009709F476C066301F
:100E6000710508F474C0FC016081633509F071C03C
:100E700061816C3209F06FC064816C3209F06DC021
:100E80004115510509F46BC02115310509F469C0FC
:100E90008581813309F067C0B901EA01F901108247
:100EA000CA010E948020882309F45FC0CE010E94FD
:100EB000612081112BC0CE010E94E62961E0CE01A4
:100EC0000E94112764E0CE010E94AC1461E0CE01C3
:100ED0000E94462019820E94FBA8E5E8F3E4808185
:100EE00090E0DC01AB57BC4B25853685880F991FF8
:100EF000FC01EB57FC4B418152811F960C9161E044
:100F000087EF9CE30E94002581E032C00E944E2AB8
:100F100081112DC084E1EBE9F9E2A9E4B3E4019089
:100F20000D928A95E1F7E9E4F3E401900020E9F7F6
:100F30003197AF014954534421E069E473E48AEAEC
:100F400099E30F94F03181E013C080E011C080E09C
:100F50000FC080E00DC080E00BC080E009C080E0E1
:100F600007C080E005C080E003C081E001C081E0EF
:100F7000DF91CF910F9108950F931F93CF93009717
:100F800009F4C5C16630710508F4C3C1DC012C91B8
:100F9000233509F0C0C111962C9111972C3209F01C
:100FA000BCC114962C9114972C3209F0B8C141158C
:100FB000510509F4B6C11596EC918E2F90E0FC0115
:100FC000F097E734F10508F0AEC18A018827E450B4
:100FD000FE4F8F4F0D942B65CA010E94BF148430C1
:100FE00031F0C8010E94BF14893009F09EC1C801C8
:100FF0000E94D21FC8010F94721BC8010E94E629EB
:101000000F94912960E087EF9CE30E94112763E031
:10101000C8010E94AC14F80111820E94E8A8E5E81A
:10102000F3E4808190E0DC01AB57BC4B258536852D
:10103000880F991FFC01EB57FC4B418152811F9691
:101040000C9161E087EF9CE30E940025C1E07CC128
:10105000CA010E946120882309F469C181E0D80196
:1010600011968C9360E0C8010E94D81460E0C8011A
:101070000E94C6140E944E2A81115BC180E1EFEAF2
:10108000F9E2A9E4B3E401900D928A95E1F7E9E46D
:10109000F3E401900020E9F73197AF01495453443C
:1010A00021E069E473E48AEA99E30F94F031C1E046
:1010B0004BC1CA010E946120882309F43CC160E051
:1010C000C8010E94D81460E0C8010E94C614F8014B
:1010D000ED5AFD4FD801A75ABD4F8C9180833196B0
:1010E00011968C918083F80111820E944E2A811101
:1010F00024C180E1EFEBF9E2A9E4B3E401900D92A1
:101100008A95E1F7E9E4F3E401900020E9F73197EB
:10111000AF014954534421E069E473E48AEA99E356
:101120000F94F031C1E010C1CA010E946120C82FA4
:10113000882309F409C1C8010E94AE27C1E08111CA
:1011400003C1C0E001C1CA010E946120882329F0C7
:10115000C8010E943827C82FF7C00E9477D8C1E085
:10116000F3C0CA010E946120C82F882309F4ECC093
:101170000F94912960E087EF9CE30E94112769E0BA
:10118000C8010E94AC14D80111961C92C8010F949A
:10119000821BC8010E948A1CC8010F941C200F9456
:1011A000952C61E0C8010E944620C1E0CDC0CA0173
:1011B0000E946120C82F811106C0C8010E94BF147F
:1011C0008A3009F0C1C00F9491290F94C82760E0BC
:1011D000C8010E9411276AE0C8010E94AC1481E096
:1011E000F8018183C8010E9475B3C8010E94BC3513
:1011F000C8010E9409B30F945A2E0E944BB361E0BC
:10120000C8010E944620C1E09FC0CA010E9461201F
:10121000882309F494C00F94912960E0C8010E94CA
:10122000D81460E0C8010E94C614F801E45AFD4FCA
:101230001082C8010E9449B46AE0C8010E94AC143F
:1012400081E0D80111968C93C1E07EC0CA010E9452
:10125000BF148930A9F463EB70E4C8010F94B91F7F
:10126000C8010F94791B843109F06BC0C8010F9439
:10127000821BC8010F941C200F94952CC1E064C000
:10128000C8010E94BF148A3009F05DC0E3EBF0E4AE
:1012900062817381808191810F94795863EB70E44E
:1012A000C8010E94A6B2C1E04FC0CA010F94721BD0
:1012B000C8010E94F0ADC8010E94E62961E0C801A2
:1012C0000E94112764E0C8010E94AC1461E0C801CB
:1012D0000E944620F80111820E94FBA8E5E8F3E491
:1012E000808190E0DC01AB57BC4B25853685880FAB
:1012F000991FFC01EB57FC4B418152811F960C91C9
:1013000061E087EF9CE30E940025C1E01DC0C0E0C2
:101310001BC0C0E019C0C0E017C0C0E015C0C0E0ED
:1013200013C0C0E011C0C0E00FC0C1E00DC0C1E0FB
:101330000BC0C1E009C0C1E007C0C1E005C0C1E009
:1013400003C0C1E001C0C0E08C2FCF911F910F916D
:101350000895FC01892B61F06630710558F0808199
:101360008D3451F481E091819C3239F080E0089510
:1013700080E0089580E0089580E00895FC01892BC5
:1013800061F06630710558F08081823551F481E05A
:1013900091819C3239F080E0089580E0089580E0EA
:1013A000089580E00895FC01892B61F06530710596
:1013B00058F080818A3551F481E091819C3239F076
:1013C00080E0089580E0089580E0089580E0089529
:1013D000CF92DF92EF92FF920F931F93CF93DF9301
:1013E000CDB7DEB72897CDBFDEBF009709F457C051
:1013F0006530710508F455C0FC0120812A3509F0DB
:1014000052C021812C3209F050C07B018C016C014B
:10141000F2E0CF0ED11CAB01425051099E012F5F6B
:101420003F4FB6018CE20F949D37882309F446C0E4
:1014300049815A814E5F5F4F49835A83433051053A
:10144000B0F142509E012D5F3F4F60E0C6010F9406
:101450002536882399F18B819C81039750F58981EA
:101460009A8101968E159F0530F54E2D481B9E01E1
:101470002B5F3F4F60E0800F911F0F94B0368823A1
:10148000E9F06D817E818F819885623071058105DB
:10149000910598F48B810E9465EE81E00FC080E099
:1014A0000DC080E00BC080E009C080E007C080E094
:1014B00005C080E003C080E001C080E02896CDBF79
:1014C000DEBFDF91CF911F910F91FF90EF90DF90E2
:1014D000CF9008952F923F924F925F926F927F929A
:1014E0008F929F92AF92BF92CF92DF92EF92FF9234
:1014F0000F931F93CF93DF93CDB7DEB76397CDBF25
:10150000DEBF8C01F62E81E08D830115110509F4F3
:1015100023C38093CE2089E10E94CAD0672B682B19
:10152000692B09F025C30F949911B82E811103C0BE
:10153000F11020C385C387EF9CE30E94D320B82E0F
:10154000882309F47DC387EF9CE30E94BF148F8733
:10155000F11004C08150823008F400C32F8524307C
:1015600031F487EF9CE30E942C2A33E03F870F94ED
:101570005C190F94451987EF9CE30E949922811111
:101580000F94B32987EF9CE30E94E62982E00E9432
:10159000CAD0E62E8FEF8E0D8A3008F0E1C2AE0180
:1015A0004A5F5F4FBE016B5F7F4F8E2D0E940E2200
:1015B0008E810E94D0ED8E8184700E9444EE8D81D8
:1015C0000F94B7130F2EF9E4CF2EF3E4DF2EF02D96
:1015D0008BE7D6018C938DE611968C9311978CE254
:1015E00012968C93129787E713968C9320E044E031
:1015F00050E0B601C8010F94F0311F92EF928FECCA
:1016000099E29F938F93DF92CF920F945867F601E0
:1016100001900020E9F73197AF014954534420E08D
:10162000B601C8010F94F031E8E2F4E587858F93A5
:1016300086858F9385858F9384858F930F2EF3ED09
:10164000AF2EF9E2BF2EF02DBF92AF92DF92CF9274
:101650000F945867F60101900020E9F73197AF0128
:101660004954534420E0B601C8010F94F0318AE098
:101670000E94CAD09F938F937F936F93BF92AF9234
:10168000DF92CF920F945867F60101900020E9F79E
:101690003197AF014954534420E0B601C8010F947B
:1016A000F0318BE00E94CAD09F938F937F936F930A
:1016B000BF92AF92DF92CF920F945867F6010190DC
:1016C0000020E9F73197AF014954534420E0B601B7
:1016D000C8010F94F0310F2EF2E4CF2EF4E5DF2E87
:1016E000F02DCDBFDEBF412C512C320145010F2E14
:1016F000F9E4AF2EF3E4BF2EF02D2BC0D6018C9170
:1017000011969C91119712962C91129713963C91D9
:10171000B4E0CB0ED11C3F932F939F938F939F9256
:101720008F92BF92AF920F945867F50101900020FD
:10173000E9F73197AF014954534420E0B501C8019E
:101740000F94F031EFEF4E1A5E0A6E0A7E0ACDBF9B
:10175000DEBF0F94922C90E0A0E0B0E0481659064E
:101760006A067B0658F28DE78093494321E041E009
:1017700050E069E473E4C8010F94F03165E087EF4D
:101780009CE30E94AC140F94912987EF9CE30E9484
:10179000EB240E94D25B60E072E080E090E00E9467
:1017A000C45C1092EC401092ED4086EC93E40E94F1
:1017B00052B70E94655E8111FCCFB82EF11004C0B3
:1017C0000E94BA1F8823E1F389E00E94CAD06F31DA
:1017D00071058105910508F59B01AC01012E1CE006
:1017E000220F331F441F551F1A95D1F7102D2B8739
:1017F0003C874D875E87CA01B9010F94FE180F948C
:101800005B2A81E00F94AB2C80E090E1A0E0B0E097
:101810008F839887A987BA873FC09B01AC01012EAF
:1018200019E0220F331F441F551F1A95D1F7102DB1
:101830002B873C874D875E87CA01B9010F94FE183C
:101840000F945B2A0F94DB2C80E092E0A0E0B0E0E4
:101850008F839887A987BA871FC0412C512C3201EA
:101860009F2CCB84DC84ED84FE840F94182D882378
:10187000E1F08D810F94852866EC73E40E94B5B782
:10188000A82E0F94072D9FEF491A590A690A790A61
:10189000A1100BC0F92C0FC02B853C854D855E85B2
:1018A000232B242B252BC9F606C04C145D046E0493
:1018B0007F04D8F2F92C0F94022D86EC93E40E9459
:1018C00019B8E82E0E94515D0F944526EE2031F0A4
:1018D0006F8587EF9CE30E94AC14B2C18FEE95E454
:1018E0000E9467DE882351F0F11008C06091EE4637
:1018F00070E08FEE95E40E9479B809C0E9E4F3E462
:101900001082118262E070E0CF010E9479B860E03D
:1019100072E080E090E00E94DA5B0E94655E8111D7
:10192000FCCF8B859C85AD85BE85892B8A2B8B2B27
:1019300009F4F3C0C12CD12C76010F2EF9E42F2E1F
:10194000F3E43F2EF02D4F80588469847A8491E02F
:10195000491A5108610871080E9468B88093EC40E8
:101960009093ED40AE014F5F5F4FBC018D810E94AF
:10197000EA14882309F463C1C701B6012F813885B1
:1019800049855A850F94ED644B015C01672B682BE8
:10199000692BA1F5C701B6012F81388549855A8584
:1019A0000F94ED64288B398B4A8B5B8B89E00E9406
:1019B000CAD0AB89AF93BA89BF93E989EF93F8890D
:1019C000FF939F938F937F936F9328ED39E23F931B
:1019D0002F933F922F920F945867F10101900020AE
:1019E000E9F73197AF014954534420E0B101C801F0
:1019F0000F94F0311092CE20CDBFDEBF2F813885FD
:101A000049855A85211582E038074105510509F4B9
:101A1000BAC0211530414105510509F4DDC0D70197
:101A2000C60187709927AA27BB27892B8A2B8B2B66
:101A300009F043C08C818F938B818F938A818F9320
:101A400089818F93A1E5BBE2BF93AF933F922F9221
:101A50000F945867F10101900020E9F73197AF0129
:101A60004954534420E0B101C8010F94F031C7013B
:101A7000B6012F81388549855A850F94ED642F5F13
:101A80003F4F4F4F5F4F6F81788589859A850F94BF
:101A9000AB64CDBFDEBFA7019601285F3F4F4F4F1C
:101AA0005F4F621773078407950719F41092CE20D1
:101AB000C0C031E03093CE20BCC01092CE20841440
:101AC0009504A604B70479F4EDE7D101EC9321E085
:101AD00041E050E0B101C8010F94F0310FC0ECE2D9
:101AE000D101EC9304C08091CE20882339F020E00E
:101AF00041E050E0B101C8010F94F031FFEFCF1A7F
:101B0000DF0AEF0AFF0A2B853C854D855E85C216EC
:101B1000D306E406F50609F01FCF0E94A55C0F94DA
:101B200045260F941D3B83EB90E40F94FD5C6F857D
:101B300087EF9CE30E94AC140F94D31987EF9CE3CA
:101B40000E94992281110F94B32987EF9CE30E9490
:101B5000E629BB24B39474C0B12C72C0B12C70C000
:101B6000B12C6EC087EF9CE30E94BF148F87F6CC28
:101B7000FF24F39487EF9CE30E94D320B82E8823A0
:101B800009F45EC0EFCF8C818F938B818F938A8114
:101B90008F9389818F9341E55BE25F934F933F92EF
:101BA0002F920F945867F10101900020E9F73197C7
:101BB000AF014954534420E0B101C8010F94F03102
:101BC00091E09093CE20CDBFDEBF481459046A0443
:101BD0007B0409F084CF78CF8C818F938B818F9396
:101BE0008A818F9389818F93E1E5FBE2FF93EF93E5
:101BF0003F922F920F945867F10101900020E9F76E
:101C00003197AF014954534420E0B101C8010F940A
